S01B0000636F756E7465725F68616E645F646973635F742E737265633A
S3150802000000000A2021AD0308297C0308317C030875
S31508020010397C0308417C0308497C030871AD03084F
S3150802002000000000000000000000000071AD030897
S31508020030517C03080000000035030208E1020208A9
S3150802004071AD030871AD030871AD030871AD0308FC
S3150802005071AD030871AD030871AD030871AD0308EC
S3150802006071AD030871AD030871AD030871AD0308DC
S315080200705F7C030871AD030871AD030871AD03080F
S3150802008071AD030871AD030871AD030871AD0308BC
S3150802009071AD030871AD030871AD030871AD0308AC
S315080200A071AD030871AD030871AD030871AD03089C
S315080200B071AD030871AD030871AD030871AD03088C
S315080200C071AD030871AD030871AD030871AD03087C
S315080200D00000000071AD030871AD03086D7C0308CA
S315080200E071AD030871AD030871AD030871AD03085C
S315080200F071AD030871AD030871AD0308817C03086D
S31508020100957C030871AD030871AD030871AD030848
S3150802011071AD030871AD030871AD030871AD03082B
S3150802012071AD030871AD0308A97C030871AD030814
S3150802013071AD030871AD030871AD030871AD03080B
S3150802014071AD030871AD030871AD030871AD0308FB
S3150802015071AD030871AD030871AD030871AD0308EB
S3150802016071AD030871AD030871AD030871AD0308DB
S3150802017071AD030871AD030871AD030871AD0308CB
S3150802018071AD030871AD030871AD030871AD0308BB
S3150802019071AD030871AD030871AD030871AD0308AB
S315080201A071AD030871AD030871AD030871AD03089B
S315080201B071AD030871AD030871AD030871AD03088B
S315080201C071AD030871AD030871AD030871AD03087B
S315080201D071AD030871AD030871AD030871AD03086B
S315080201E071AD030871AD030871AD030871AD03085B
S315080201F071AD030871AD030871AD030871AD03084B
S3150802020071AD030871AD030871AD03080000000063
S315080202100000000071AD03080000000071AD03087C
S3150802022071AD030871AD0308BD7C030871AD0308FF
S3150802023071AD030871AD030871AD030871AD03080A
S3150802024071AD030871AD030871AD03080000000023
S3150802025010B5054C237833B9044B13B10448AFF3F0
S3150802026000800123237010BDB01800200000000092
S31508020270F44A050808B5034B1BB103490348AFF313
S31508020280008008BD00000000B4180020F44A0508E2
S3150802029072B64FF0E0201749C0F8081D16480168E3
S315080202A041F00101016015481249096801604FF0E1
S315080202B0E020134941614FF0070101614FF0000147
S315080202C0C0F8181D4FF07F41C0F81C1D0D49C0F833
S315080202D0201D7047FFF7FEBF01B5BDE80140704714
S315080202E001B500F097F8BDE801407047FFF7FEBF79
S315080202F0FFF7FEBF00000208001000E08CFD002098
S315080203008FD003000000FF404FF000002D4A106016
S31508020310EFF3148020F0040080F3148862B64FF0DD
S3150802032080504FF0E021C1F8040DBFF34F8FBFF3A1
S315080203306F8FFEE72448254A4FF00003016891B102
S315080203400360EFF3098C2CE9F00F1EF0100F01D1B0
S315080203502CED108A1E4C4CF804EDC1F808C025682D
S315080203600DB18D61236072B61168D1B1016062B6B2
S315080203704F68174C8D6907F101074F602560D1F860
S315080203800CC08CF30B88D1F808C05CF804EB1EF09D
S31508020390100F01D1BCEC108ABCE8F00F8CF3098867
S315080203A0704772B61168016009B962B6F9E74FF08B
S315080203B000674FF0E028C8F8047D62B6D8E700BFA8
S315080203C07047000028FE002090FD002094FD0020C2
S315080203D094030120026922F00702A2F144026FF097
S315080203E0430313604FF0000353609360D3601361B5
S315080203F053619361D361136253629362D362136347
S3150802040053634FF0FF339363D1634FF080731364E2
S31508020410826070472249086800F101000860214B92
S315080204201A683AB1A2F101021A601AB91E4B4FF0C4
S31508020430010018601D490868026822B11C4B4FF07A
S3150802044001021A6008E000F104001A4B1A68904289
S3150802045001D1194B18680860134B1A6812B9144966
S315080204600868C8B101B51249086808B127F078FDCD
S315080204700D4B1A6872B127F0E5FC1048016849B9B4
S315080204800F4801680F4A13680F484FF08052994285
S3150802049000D00260BDE80140BFF34F8F70470000ED
S315080204A034FE00209403012038FE0020C4FE0020FA
S315080204B0C8FE0020C0FE0020BCFE002028FE002048
S315080204C090FD002094FD002004ED00E0034613F899
S315080204D0012B002AFBD1181A0138704781F0004116
S315080204E002E000BF83F0004330B54FEA41044FEA09
S315080204F0430594EA050F08BF90EA020F1FBF54EAA4
S31508020500000C55EA020C7FEA645C7FEA655C00F03F
S31508020510E2804FEA5454D4EB5555B8BF6D420CDD10
S315080205202C4480EA020281EA030382EA000083EA93
S31508020530010180EA020281EA0303362D88BF30BD33
S3150802054011F0004F4FEA01314FF4801C4CEA113189
S3150802055002D0404261EB410113F0004F4FEA0333E8
S315080205604CEA133302D0524263EB430394EA050F73
S3150802057000F0A780A4F10104D5F1200E0DDB02FAE2
S315080205800EFC22FA05F2801841F1000103FA0EF276
S31508020590801843FA05F359410EE0A5F120050EF13C
S315080205A0200E012A03FA0EFC28BF4CF0020C43FA6D
S315080205B005F3C01851EBE37101F0004507D54FF07A
S315080205C0000EDCF1000C7EEB00006EEB0101B1F5CA
S315080205D0801F1BD3B1F5001F0CD349085FEA300010
S315080205E04FEA3C0C04F101044FEA445212F5800F1B
S315080205F080F09A80BCF1004F08BF5FEA500C50F1B8
S31508020600000041EB045141EA050130BD5FEA4C0C9A
S31508020610404141EB0101013C28BFB1F5801FE9D2F7
S3150802062091F0000F04BF01460020B1FA81F308BF1A
S315080206302033A3F10B03B3F120020CDA0C3208DDE6
S3150802064002F1140CC2F10C0201FA0CF021FA02F1C1
S315080206500CE002F11402D8BFC2F1200C01FA02F131
S3150802066020FA0CFCDCBF41EA0C019040E41AA2BF56
S3150802067001EB0451294330BD6FEA04041F3C1CDA1E
S315080206800C340EDC04F11404C4F1200220FA04F03E
S3150802069001FA02F340EA030021FA04F345EA0301E8
S315080206A030BDC4F10C04C4F1200220FA02F001FAAA
S315080206B004F340EA0300294630BD21FA04F029462C
S315080206C030BD94F0000F83F4801306BF81F48011C5
S315080206D00134013D4EE77FEA645C18BF7FEA655C38
S315080206E029D094EA050F08BF90EA020F05D054EA0A
S315080206F0000C04BF1946104630BD91EA030F1EBF0F
S315080207000021002030BD5FEA545C05D14000494112
S3150802071028BF41F0004130BD14F580043CBF01F505
S31508020720801130BD01F0004545F0FE4141F47001EB
S315080207304FF0000030BD7FEA645C1ABF19461046C6
S315080207407FEA655C1CBF0B46024650EA013406BFC7
S3150802075052EA033591EA030F41F4002130BD00BF86
S3150802076090F0000F04BF0021704730B54FF4806443
S3150802077004F132044FF000054FF0000150E700BFC4
S3150802078090F0000F04BF0021704730B54FF4806423
S3150802079004F1320410F0004548BF40424FF0000110
S315080207A03EE700BF42004FEAE2014FEA31014FEA53
S315080207B002701FBF12F07F4393F07F4F81F06051A2
S315080207C0704732F07F4208BF704793F07F4F04BFED
S315080207D041F40021704730B54FF4607401F00045CA
S315080207E021F000411CE700BF50EA010208BF70472A
S315080207F030B54FF000050AE050EA010208BF70471B
S3150802080030B511F0004502D5404261EB41014FF483
S31508020810806404F132045FEA915C3FF4D8AE4FF08B
S3150802082003025FEADC0C18BF03325FEADC0C18BF6E
S31508020830033202EBDC02C2F1200300FA03FC20FABF
S3150802084002F001FA03FE40EA0E0021FA02F114440C
S31508020850BDE600BF70B54FF0FF0C4CF4E06C1CEA25
S3150802086011541DBF1CEA135594EA0C0F95EA0C0F96
S3150802087000F0DEF82C4481EA030621EA4C5123EA09
S315080208804C5350EA013518BF52EA033541F4801138
S3150802089043F4801338D0A0FB02CE4FF00005E1FBEB
S315080208A002E506F00042E0FB03E54FF00006E1FB35
S315080208B003569CF0000F18BF4EF0010EA4F1FF0478
S315080208C0B6F5007F64F5407404D25FEA4E0E6D41B8
S315080208D046EB060642EAC62141EA55514FEAC520C9
S315080208E040EA5E504FEACE2EB4F1FD0C88BFBCF545
S315080208F0E06F1ED8BEF1004F08BF5FEA500E50F1F6
S31508020900000041EB045170BD06F0004646EA0101BB
S3150802091040EA020081EA0301B4EB5C04C2BFD4EBED
S315080209200C0541EA045170BD41F480114FF0000EE6
S31508020930013C00F3AB8014F1360FDEBF002001F054
S31508020940004170BDC4F10004203C35DA0C341BDCCE
S3150802095004F11404C4F1200500FA05F320FA04F0A0
S3150802096001FA05F240EA020001F0004221F00041D4
S3150802097010EBD37021FA04F642EB06015EEA430E47
S3150802098008BF20EAD37070BDC4F10C04C4F1200577
S3150802099000FA04F320FA05F001FA04F240EA02002A
S315080209A001F0004110EBD37041F100015EEA430EFB
S315080209B008BF20EAD37070BDC4F1200500FA05F21B
S315080209C04EEA020E20FA04F301FA05F243EA02039A
S315080209D021FA04F001F0004121FA04F220EA0200A9
S315080209E000EBD3705EEA430E08BF20EAD37070BDEF
S315080209F094F0000F0FD101F00046400041EB0101CF
S31508020A0011F4801F08BF013CF7D041EA060195F0B0
S31508020A10000F18BF704703F00046520043EB03036A
S31508020A2013F4801F08BF013DF7D043EA0603704757
S31508020A3094EA0C0F0CEA135518BF95EA0C0F0CD062
S31508020A4050EA410618BF52EA4306D1D181EA0301A8
S31508020A5001F000414FF0000070BD50EA410606BFA2
S31508020A601046194652EA430619D094EA0C0F02D1E7
S31508020A7050EA013613D195EA0C0F05D152EA03362C
S31508020A801CBF104619460AD181EA030101F000414A
S31508020A9041F0FE4141F470014FF0000070BD41F093
S31508020AA0FE4141F4780170BD70B54FF0FF0C4CF46D
S31508020AB0E06C1CEA11541DBF1CEA135594EA0C0F8C
S31508020AC095EA0C0F00F0A7F8A4EB050481EA030ED9
S31508020AD052EA03354FEA013100F088804FEA0333C0
S31508020AE04FF0805545EA131343EA12634FEA02228E
S31508020AF045EA111545EA10654FEA00260EF000414F
S31508020B009D4208BF964244F1FD0404F5407402D2A0
S31508020B105B084FEA3202B61A65EB03055B084FEA31
S31508020B2032024FF480104FF4002CB6EB020E75EB2E
S31508020B30030E22BFB61A754640EA0C005B084FEA56
S31508020B403202B6EB020E75EB030E22BFB61A7546D3
S31508020B5040EA5C005B084FEA3202B6EB020E75EB1E
S31508020B60030E22BFB61A754640EA9C005B084FEA96
S31508020B703202B6EB020E75EB030E22BFB61A7546A3
S31508020B8040EADC0055EA060E18D04FEA051545EA92
S31508020B9016754FEA06164FEAC30343EA52734FEA3B
S31508020BA0C2025FEA1C1CC0D111F4801F0BD141EAB4
S31508020BB000014FF000004FF0004CB6E711F4801F19
S31508020BC004BF01430020B4F1FD0C88BFBCF5E06FF9
S31508020BD03FF6AFAEB5EB030C04BFB6EB020C5FEA09
S31508020BE0500C50F1000041EB045170BD0EF0004E5E
S31508020BF04EEA113114EB5C04C2BFD4EB0C0541EA90
S31508020C00045170BD41F480114FF0000E013C90E68C
S31508020C1045EA060E8DE60CEA135594EA0C0F08BF50
S31508020C2095EA0C0F3FF43BAF94EA0C0F0AD150EA4F
S31508020C3001347FF434AF95EA0C0F7FF425AF1046E2
S31508020C4019462CE795EA0C0F06D152EA03353FF40A
S31508020C50FDAE1046194622E750EA410618BF52EA87
S31508020C6043067FF4C5AE50EA41047FF40DAF52EA5B
S31508020C7043057FF4EBAE12E74FF0FF3C06E000BFF8
S31508020C804FF0010C02E000BF4FF0010C4DF804CD05
S31508020C904FEA410C7FEA6C5C4FEA430C18BF7FEAC5
S31508020CA06C5C1BD001B050EA410C0CBF52EA430CF3
S31508020CB091EA030F02BF90EA020F0020704710F173
S31508020CC0000F91EA030F58BF994208BF90422CBF02
S31508020CD0D8176FEAE37040F0010070474FEA410CFB
S31508020CE07FEA6C5C02D150EA013C07D14FEA430C19
S31508020CF07FEA6C5CD6D152EA033CD3D05DF8040B8A
S31508020D00704700BF8446104662468C4619466346BB
S31508020D1000E000BF01B5FFF7B7FF002848BF10F192
S31508020D20000F01BD4DF808EDFFF7F4FF0CBF0120D7
S31508020D3000205DF808FB00BF4DF808EDFFF7EAFF53
S31508020D4034BF012000205DF808FB00BF4DF808ED0E
S31508020D50FFF7E0FF94BF012000205DF808FB00BF03
S31508020D604DF808EDFFF7CEFF94BF012000205DF88D
S31508020D7008FB00BF4DF808EDFFF7C4FF34BF01209A
S31508020D8000205DF808FB00BF4FEA410C7FEA6C5C65
S31508020D9002D150EA013C0AD14FEA430C7FEA6C5C65
S31508020DA002D152EA033C02D14FF0000070474FF0DD
S31508020DB0010070474FEA410212F5001215D211D509
S31508020DC06FF47873B3EB625212D94FEAC12343F038
S31508020DD0004343EA505311F0004F23FA02F018BFBA
S31508020DE0404270474FF00000704750EA013005D183
S31508020DF011F0004008BF6FF0004070474FF0000046
S31508020E00704700BF4A0011D212F5001211D20DD551
S31508020E106FF47873B3EB62520ED44FEAC12343F0F0
S31508020E20004343EA505323FA02F070474FF000009A
S31508020E30704750EA013002D14FF0FF3070474FF049
S31508020E40000070474FEA4102B2F1E04324BFB3F50E
S31508020E50001CDCF1FE5C0DD901F0004C4FEAC00221
S31508020E604CEA5070B2F1004F40EB830008BF20F005
S31508020E700100704711F0804F21D113F13872BCBFBF
S31508020E8001F00040704741F480114FEA5252C2F114
S31508020E901802C2F1200C10FA0CF320FA02F018BF5D
S31508020EA040F001004FEAC1234FEAD32303FA0CFCB0
S31508020EB040EA0C0023FA02F34FEA4303CCE77FEA3F
S31508020EC0625307D150EA01331EBF4FF0FE4040F489
S31508020ED04000704701F0004040F0FE4040F4000038
S31508020EE0704700BF53B94AB9002908BF00281CBF7A
S31508020EF04FF0FF314FF0FF3000F0B4B9ADF1080CF6
S31508020F006DE904CE00F03CF8DDF804E0DDE90223E1
S31508020F1004B0704738B50022002304460D46FFF791
S31508020F200BFF28B920462946BDE8384000F00AB822
S31508020F30204605F1004100F005F8404261EB410107
S31508020F4038BD00BFD0B500220B4B06460F46FFF749
S31508020F5081FCFFF757FF0446FFF702FC0022074B06
S31508020F60FFF778FC02460B4630463946FFF7BAFACF
S31508020F70FFF748FF2146D0BD0000F03D0000F041D2
S31508020F802DE9F04F099D0C46002B4DD18A420F469A
S31508020F9084469646B2FA82F360D94BB102FA03FE48
S31508020FA0C3F120029F4000FA03FC20FA02F217431B
S31508020FB04FEA1E461FFA8EF44FEA1C42B7FBF6F1B9
S31508020FC006FB117701FB04F042EA0742904208D970
S31508020FD01EEB020201F1FF3702D2904200F22D8186
S31508020FE03946121A1FFA8CFCB2FBF6F006FB1022DF
S31508020FF000FB04F44CEA024C644508D91EEB0C0CBF
S3150802100000F1FF3202D2644500F21A81104640EA24
S315080210100140ACEB040C002125B12CFA03F30022A3
S31508021020C5E90032BDE8F08F8B4205D90DB1C5E995
S31508021030000100210846F5E7B3FA83F100294DD1EC
S31508021040A342C0F0F280904280F0EF800646234623
S315080210500846002DE6D0C5E90063E3E7002B40F019
S31508021060A2808A1A4FEA1E471FFA8EF60121B2FBA0
S31508021070F7F407FB14204FEA1C4242EA004206FB39
S3150802108004F090420FD91EEB020204F1FF382CBF7E
S315080210904FF001094FF00009904203D9B9F1000F48
S315080210A000F0C8804446121A1FFA8CFCB2FBF7F00D
S315080210B007FB102200FB06F64CEA024C664508D9E5
S315080210C01EEB0C0C00F1FF3202D2664500F2BB8021
S315080210D01046ACEB060C40EA04409DE7C1F1200637
S315080210E08B4004FA01FE22FA06F720FA06FCF440BF
S315080210F08A401F434EEA0C0300FA01FE4FEA1748DC
S315080211004FEA13491FFA87FCB4FBF8F008FB1044B0
S3150802111049EA044400FB0CF9A1450ED93C1900F131
S31508021120FF3A2CBF4FF0010B4FF0000BA14503D934
S31508021130BBF1000F00F093805046A4EB09041FFA96
S3150802114083F9B4FBF8F308FB134403FB0CFC49EAE6
S315080211500444A44506D93C1903F1FF3801D2A44533
S315080211607AD8434643EA0040A4EB0C04A0FB029853
S315080211704445CC46434602D306D1CE4504D201386D
S31508021180B9EB020C68EB07035DB1BEEB0C0264EB2C
S31508021190030404FA06F622FA01F3CC401E43C5E913
S315080211A0006400213EE702FA03FEC3F1200104FAB5
S315080211B003F200FA03FCCC404FEA1E4720FA01F17B
S315080211C01FFA8EF6B4FBF7F00A4307FB1044110C1C
S315080211D041EA044100FB06F48C420ED91EEB0101DA
S315080211E000F1FF382CBF4FF001094FF000098C427D
S315080211F002D9B9F1000F2CD04046091B92B2B1FBB5
S31508021200F7F407FB141142EA014204FB06F1914284
S3150802121007D91EEB020204F1FF3801D2914215D812
S315080212204446521A44EA004121E7861A64EB03034C
S3150802123001200EE7023C724435E702397244D0E6D1
S31508021240F4440238E3E6F444023842E7023C7244C4
S31508021250E7E702387144D0E7023B3C4482E70238AA
S315080212603C446AE7704700BF80B586B002AF786033
S315080212700023FB60342300934FF4E8430B4A0C49DE
S315080212800C4827F017F90346002B0AD1094BBB6015
S31508021290B86802F0D7FFF860FB68002B01D000BFE0
S315080212A0FDE700BF1037BD4680BD00BFCC18002041
S315080212B0104B0508CC8C002090B589B000AF786039
S315080212C00023FB617B68BB61FE202BF0D3FA002367
S315080212D0FB611FE007F1080310220021184630F0CF
S315080212E045F9BB6907F10804186859689A68DB6802
S315080212F00FC4FB6903F1016303F57C2307F10802B6
S31508021300114618462BF09BFABB691033BB61FB6981
S315080213101033FB61FB691F2BDCD9012318462437DE
S31508021320BD4690BD80B483B000AF78607B685B68C9
S3150802133018460C37BD465DF8047B704780B483B007
S3150802134000AF786039607B683A685A6000BF0C372C
S31508021350BD465DF8047B704780B483B000AF786001
S315080213607B681B7A18460C37BD465DF8047B7047C6
S3150802137080B483B000AF78600B46FB707B68FA785E
S315080213801A7200BF0C37BD465DF8047B704780B4FD
S3150802139083B000AF78600B46FB70FB78042B04D849
S315080213A0FB787A6813449B7A00E0002318460C37C8
S315080213B0BD465DF8047B704780B483B000AF7860A1
S315080213C00B46FB701346BB70FB78042B0DD8BB7813
S315080213D0002B05D0FB787A68134401229A7204E03E
S315080213E0FB787A68134400229A7200BF0C37BD460E
S315080213F05DF8047B704780B483B000AF78607B6881
S31508021400DB7B18460C37BD465DF8047B704780B413
S3150802141083B000AF78600B46FB707B68FA78DA73A4
S3150802142000BF0C37BD465DF8047B704780B483B0B5
S3150802143000AF78607B681B7C18460C37BD465DF8A2
S31508021440047B704780B483B000AF78600B46FB70AC
S315080214507B68FA781A7400BF0C37BD465DF8047BC0
S315080214607047000080B483B000AF0346FB71044A9C
S31508021470FB79137000BF0C37BD465DF8047B7047D5
S31508021480E5A2002080B586B000AFF8600B467A6008
S31508021490FB720023FB752D4819F014FA0023FB751D
S315080214A04CE0FB7D2A4A4FF48E7101FB03F3134489
S315080214B01B78012B3FD1FB7D4FF48E7202FB03F39F
S315080214C0234A134402331946224819F0FBF92248E3
S315080214D019F0F8F9FB7D4FF48E7202FB03F3183309
S315080214E01B4A1344043319461A4819F0EBF91B48E8
S315080214F019F0E8F9FB7D164A4FF48E7101FB03F3E6
S3150802150013449C331B782D2B12D0154819F0DAF99F
S31508021510FB7D4FF48E7202FB03F398330C4A134495
S31508021520043319460B4819F0CDF90C4819F0CAF9D3
S315080215300A4819F0C7F9FB7D0133FB75FB7D132BAE
S31508021540AFD900BF00BF1837BD4680BD244B05087A
S31508021550000000204C4B0508504B0508544B050863
S31508021560584B050890B587B000AFF8600B467A600D
S31508021570FB7200237B6100233B617B6803F50073E2
S315080215801A78A14B1B78D31A002B0FD17B6803F567
S3150802159000731846FEF79AFF0346012B06D19B48AD
S315080215A019F090F99A4819F08DF92EE37B6803F53C
S315080215B000730322974918462FF0E0FF0346002BD3
S315080215C008D17B6803F500731846FEF77FFF0346CA
S315080215D0032B15D07B6803F5007307228E4918463C
S315080215E02FF0CCFF0346002B40F00C837B6803F5F3
S315080215F000731846FEF76AFF0346072B40F002837C
S315080216007B6803F580631A787F4B1B78D31A002B05
S3150802161024D17B6803F580631846FEF757FF034615
S31508021620012B1BD17D4819F04DF97D4819F04AF96D
S315080216307C4819F047F97C4819F044F97B4819F0B7
S3150802164041F97B4819F03EF97A4819F03BF97A488C
S3150802165019F038F9794819F035F9D6E27B6803F5B5
S3150802166080630822764918462FF088FF0346002B26
S3150802167008D17B6803F580631846FEF727FF034601
S31508021680082B11D07B6803F580631A786D4B1B789B
S31508021690D31A002B31D17B6803F580631846FEF70F
S315080216A015FF0346012B28D17B6803F5C06318464C
S315080216B02EF05AFE78617B69002B02DB7B690A2BC6
S315080216C003DD614819F0FEF89FE227F0DDF90346CB
S315080216D0184627F021FA03460133DBB219465B485E
S315080216E027F044FA7B69DBB21946584827F059FABB
S315080216F05749564827F0B6FA76E27B6803F58063BF
S315080217000C22544918462FF039FF0346002B08D1FC
S315080217107B6803F580631846FEF7D8FE03460C2B52
S3150802172011D07B6803F580631A784B4B1B78D31A62
S31508021730002B1AD17B6803F580631846FEF7C6FEAE
S315080217400346012B11D127F09FF90346184627F0C5
S31508021750E3F903460133DBB21946404827F03CFA5F
S315080217603B493E4827F0E1FA3EE27B6803F580638F
S3150802177008223B4918462FF001FF0346002B08D1E1
S315080217807B6803F580631846FEF7A0FE0346082B1E
S3150802179011D07B6803F580631A78324B1B78D31A0B
S315080217A0002B65D17B6803F580631846FEF78EFE2B
S315080217B00346012B5CD17B6803F5C06318462EF0FD
S315080217C0D3FD78617B69002B02DB7B69062B03DD7F
S315080217D0254819F077F818E227F056F9034618460D
S315080217E027F09AF903460133DBB219461F480BF074
S315080217F04BFF7B69DBB219461C480BF060FF1449A4
S315080218001A480CF0B0F8EFE1644B0508684B050876
S315080218107C4B0508944B0508984B0508A04B050810
S31508021820B04B0508D04B0508E84B0508084C0508D7
S31508021830284C0508484C0508744C0508944C0508BC
S31508021840B84C0508C44C0508C84C050800A3002076
S3150802185008A30020EC4C0508FC4C050804A300204C
S31508021860004D05080C4D0508104D0508E8A2002094
S315080218707B6803F580630622A24918462FF07EFE8E
S315080218800346002B08D17B6803F580631846FEF7EA
S315080218901DFE0346062B11D07B6803F580631A7872
S315080218A0994B1B78D31A002B31D17B6803F58063D9
S315080218B01846FEF70BFE0346012B28D17B6803F573
S315080218C0C06318462EF050FD78617B69002B02DD55
S315080218D07B69022B03DD8D4818F0F4FF95E127F0AA
S315080218E0D3F80346184627F017F903460133DBB245
S315080218F0194687480BF0FEFE7B69DBB21946844817
S315080219000BF013FF834982480CF090F86CE17B6870
S3150802191003F580630B22804918462FF02FFE0346F3
S31508021920002B08D17B6803F580631846FEF7CEFDC7
S3150802193003460B2B11D07B6803F580631A78774B25
S315080219401B78D31A002B31D17B6803F580631846BE
S31508021950FEF7BCFD0346012B28D17B6803F5C0635D
S3150802196018462EF001FD78617B69002B02DB7B6944
S31508021970062B03DD6A4818F0A5FF46E127F084F82E
S315080219800346184627F0C8F803460133DBB2194660
S3150802199064480BF0E5FE7B69DBB2194661480BF039
S315080219A0FAFE5C495F480CF0A4F81DE17B6803F572
S315080219B080630B225C4918462FF0E0FD0346002B94
S315080219C008D17B6803F580631846FEF77FFD034658
S315080219D00B2B11D07B6803F580631A78534B1B785F
S315080219E0D31A002B3ED17B6803F580631846FEF7AF
S315080219F06DFD0346012B35D17B6803F5C063184696
S31508021A002EF0B2FC78617B6803F5006318462EF067
S31508021A10ABFC38617B69002B02DB7B69022B03DD99
S31508021A20434818F04FFFF0E027F02EF80346184611
S31508021A3027F072F803460133DBB219463D480BF02C
S31508021A40C5FE7B69DBB219463A480BF0DAFE3B69FA
S31508021A50DBB2194637480BF0EFFE2E4935480CF033
S31508021A60ABF8C1E07B6803F580630A22324918465F
S31508021A702FF084FD0346002B08D17B6803F58063AB
S31508021A801846FEF723FD03460A2B11D07B6803F599
S31508021A9080631A78294B1B78D31A002B52D17B689C
S31508021AA003F580631846FEF711FD0346012B49D15B
S31508021AB07B6803F5C06318462EF056FC78617B698D
S31508021AC0002B02DB7B69042B03DD154818F0FAFEAE
S31508021AD09BE026F0D9FF0346184627F01DF8034671
S31508021AE00133DBB2194616480BF0C1FE7B69DBB23D
S31508021AF0194613480BF0D6FE064911480CF0D2F8DF
S31508021B0072E000BF304D0508384D05083C4D050802
S31508021B10ECA2002008A30020584D0508644D0508CC
S31508021B20104D0508F0A20020684D0508744D0508F9
S31508021B30784D0508F4A20020984D0508A44D05081D
S31508021B40F8A200207B6803F580630E223049184606
S31508021B502FF014FD0346002B08D17B6803F580633A
S31508021B601846FEF7B3FC03460E2B11D07B6803F525
S31508021B7080631A78274B1B78D31A002B31D17B68DE
S31508021B8003F580631846FEF7A1FC0346012B28D10C
S31508021B907B6803F5C06318462EF0E6FB78617B691D
S31508021BA0002B02DB7B69022B03DD1B4818F08AFE39
S31508021BB02BE026F069FF0346184626F0ADFF0346DA
S31508021BC00133DBB2194615480BF087FE7B69DBB297
S31508021BD0194612480BF09CFE114910480CF0C5F83C
S31508021BE002E0104818F06EFE0D482AF024FF04465B
S31508021BF00B482AF02CFF0346DBB2194620460CF0A6
S31508021C0097FA02E0084818F05DFE1C37BD4690BDFB
S31508021C10A84D0508B84D0508104D0508FCA2002078
S31508021C2008A30020BC4D0508D04D050880B586B02E
S31508021C3000AFF8600B467A60FB7200237B617B6813
S31508021C4003F500731A78634B1B78D31A002B2ED12F
S31508021C507B6803F500731846FEF738FC0346012B2A
S31508021C6025D17B6803F5806318462EF07DFB7861E3
S31508021C707B69642B17DC584B01221A70796957481D
S31508021C8018F020FE564B1B687A69DA63544B1B68B8
S31508021C9000229A630821524821F0EAF804215048A2
S31508021CA021F046FA93E04F4818F00CFE8FE07B6865
S31508021CB003F500731A784C4B1B78D31A002B2AD1DA
S31508021CC07B6803F500731846FEF700FC0346012BF2
S31508021CD021D17B6803F5806318462EF045FB7861AF
S31508021CE07B69642B13DC3C4B01221A7079693F48E5
S31508021CF018F0E8FD3A4B1B687A699A630821384856
S31508021D0021F016FA0421364821F0B2F85FE0354888
S31508021D1018F0D8FD5BE07B6803F500731A78344B3C
S31508021D201B78D31A002B1CD17B6803F5007318465F
S31508021D30FEF7CCFB0346012B13D1274B01221A705F
S31508021D40274B1B686322DA63254B1B6863229A6357
S31508021D500821234821F08CF80421214821F088F82B
S31508021D6035E07B6803F500730322224918462FF0F3
S31508021D7005FC0346002B1FD17B6803F50073184642
S31508021D80FEF7A4FB0346032B16D1134B00221A7047
S31508021D90134B1B680022DA63114B1B6800229A63F5
S31508021DA008210F4821F0C4F904210D4821F0C0F991
S31508021DB0114818F087FD0AE0074B00221A7008211D
S31508021DC0074821F0B5F90421054821F0B1F9183779
S31508021DD0BD4680BDE84D0508F8F20020EC4D050821
S31508021DE0ACE70020044E0508244E0508284E0508CF
S31508021DF0404E0508444E0508484E050880B598B079
S31508021E0000AFF8600B467A60FB72002387F85F30F2
S31508021E1040F61F03A7F85C30002387F85E307B681C
S31508021E2003F500730322BF4918462FF0A7FB0346A2
S31508021E30002B37D17B6803F500731846FEF746FB7D
S31508021E400346032B2ED17B6803F5806318462EF0D2
S31508021E508BFA034687F85F3097F85F301946B2481F
S31508021E6018F030FD97F85F30002B14D097F85F30E2
S31508021E70062B10D816F062F903460121184616F009
S31508021E80BAFB06F091FF024697F85F3019461046EC
S31508021E9006F0F1FF35E397F85F301946A34818F0C4
S31508021EA011FD2EE37B6803F500730922A049184643
S31508021EB02FF064FB0346002B10D17B6803F50073F1
S31508021EC01846FEF703FB0346092B07D106F0EEFF79
S31508021ED003461946974818F0F5FC12E37B6803F5A2
S31508021EE000730522944918462FF048FB0346002B37
S31508021EF054D17B6803F500731846FEF7E7FA0346E2
S31508021F00052B4BD17B6803F5806318462EF02CFA15
S31508021F10034687F85F3097F85F301946874818F006
S31508021F20D1FC97F85F30013B042B35D801A252F851
S31508021F3023F000BF491F0208591F0208691F020839
S31508021F40791F0208891F02082AF07CFB0123012255
S31508021F50662116F089FE20E02AF074FB012304228A
S31508021F60662116F081FE18E02AF06CFB01230A228C
S31508021F70662116F079FE10E02AF064FB01230B2293
S31508021F80662116F071FE08E02AF05CFB01231E2288
S31508021F90662116F069FE00E000BFB2E27B6803F52F
S31508021FA000730622664918462FF0E8FA0346002B04
S31508021FB021D17B6803F500731846FEF787FA0346B4
S31508021FC0062B18D17B6803F5806318462EF0CCF9E8
S31508021FD0034687F85F3097F85F301946594818F074
S31508021FE071FC16F0ABF8024697F85F3019461046B0
S31508021FF016F055FB85E27B6803F500730522524904
S3150802200018462FF0BBFA0346002B13D17B6803F55B
S3150802201000731846FEF75AFA0346052B0AD14B48AF
S3150802202018F050FC06F0C0FE03460121184606F0D9
S31508022030D1FE66E27B6803F5007305224449184619
S315080220402FF09CFA0346002B13D17B6803F5007325
S315080220501846FEF73BFA0346052B0AD13D4818F007
S3150802206031FC06F0A1FE03460821184606F0B2FE28
S3150802207047E27B6803F500730C22374918462FF0AE
S315080220807DFA0346002B13D17B6803F500731846C5
S31508022090FEF71CFA03460C2B0AD1304818F012FC3C
S315080220A006F082FE03460221184606F093FE28E24F
S315080220B07B6803F500730B22294918462FF05EFA4E
S315080220C00346002B52D17B6803F500731846FEF7C8
S315080220D0FDF903460B2B49D17B6803F58063184645
S315080220E02EF042F9034687F85F301E4818F0EAFBDD
S315080220F006F05AFE03460321184606F06BFE97F8C9
S315080221005F30012B03D097F85F30022B05D197F881
S315080221105F30184608F0DCFAF3E1134818F0D2FBF0
S31508022120EFE100BF544E0508584E0508684E0508EB
S31508022130884E0508944E0508AC4E0508B44E0508A7
S31508022140CC4E0508D44E0508E84E0508F04E05089B
S31508022150044F05080C4F0508204F0508304F05089F
S315080221604C4F0508584F05086C4F05087B6803F560
S3150802217000730722CB4918462FF000FA0346002BB4
S3150802218014D17B6803F500731846FEF79FF90346D8
S31508022190072B0BD1C44818F095FB27F041FC07F131
S315080221A05C03022219462DF09DF9AAE17B6803F524
S315080221B000730722BD4918462FF0E0F90346002BA3
S315080221C017D17B6803F500731846FEF77FF90346B5
S315080221D0072B0ED106F0E8FD03460321184606F042
S315080221E0F9FD06F0E1FD03460121184606F028FE30
S315080221F087E17B6803F500730722AD4918462FF07D
S31508022200BDF90346002B17D17B6803F50073184600
S31508022210FEF75CF90346072B0ED106F0C5FD034609
S315080222200321184606F0D6FD06F0BEFD0346022136
S31508022230184606F005FE64E17B6803F5007305227D
S315080222409C4918462FF09AF90346002B17D17B684A
S3150802225003F500731846FEF739F90346052B0ED126
S3150802226006F0A2FD03460321184606F0B3FD06F062
S315080222709BFD03460321184606F0E2FD41E17B6811
S3150802228003F5007308228C4918462FF077F903469E
S31508022290002B23D17B6803F500731846FEF716F95F
S315080222A00346082B1AD1854818F00CFB07F1580388
S315080222B00121184628F04DFE07F1140207F15803CA
S315080222C01146184629F0D5FB27F096FB3A7D07F109
S315080222D01403013319462DF0E7F912E17B6803F579
S315080222E000730A22764918462FF048F90346002B4E
S315080222F03FD17B6803F500731846FEF7E7F80346F5
S315080223000A2B36D16F4818F0DDFA15F017FF034687
S31508022310184616F0E7F803461A4607F1100311465F
S31508022320184628F008FD15F009FF0346184616F068
S31508022330F6F803461A4607F110031146184628F01E
S3150802234015FD07F110030221184628F02AFD07F1A8
S31508022350140207F110031146184629F09BFA27F0D2
S3150802236055FB3A7D07F11403013319462DF09CF902
S31508022370C7E07B6803F500730422534918462FF019
S31508022380FDF80346002B0CD17B6803F5007318464B
S31508022390FEF79CF80346042B03D101200EF06EF8D3
S315080223A0AFE07B6803F500731022484918462FF000
S315080223B0E5F80346002B21D17B6803F5007318461E
S315080223C0FEF784F80346102B18D1414818F07AFA1A
S315080223D006F0EAFC03460121184606F016FD06F049
S315080223E0E3FC03460321184606F0F4FC06F0DCFC7F
S315080223F003460221184606F023FD82E07B6803F5B0
S3150802240000730F22334918462FF0B8F80346002BFB
S3150802241013D17B6803F500731846FEF757F803468F
S315080224200F2B0AD12C4818F04DFA06F0BDFC0346CC
S315080224300021184606F0E9FC63E07B6803F50073A1
S315080224400822264918462FF099F80346002B54D13C
S315080224507B6803F500731846FEF738F80346082B1F
S315080224604BD17B6803F5806318462DF07DFF034642
S3150802247087F85F3097F85F301946194818F022FA3C
S3150802248097F85F30184609F069F9034687F85E300F
S3150802249097F85E30002B27D0124818F013FA00BFBF
S315080224A02FE000BF884F0508904F0508A84F05087A
S315080224B0B04F0508B84F0508C04F0508CC4F0508A8
S315080224C0F44F05080050050820500508285005084D
S315080224D03C5005085050050860500508705005081C
S315080224E07C5005088C500508084B1B78184618F0CE
S315080224F027FB642025F0D4F9C2E7054818F0E2F96B
S3150802250000BF00BF6037BD4680BD00BFE5A2002000
S315080225109C50050880B584B000AFF8600B467A6017
S31508022520FB727B6803F5007308222A4918462FF0C6
S3150802253025F80346002B10D17B6803F5007318466D
S31508022540FDF7C4FF0346082B07D10DF015FE034617
S31508022550012118460DF04DFE37E07B6803F500733E
S3150802256008221D4918462FF009F80346002B10D1F8
S315080225707B6803F500731846FDF7A8FF0346082B88
S3150802258007D10DF0F9FD0346022118460DF031FE7A
S315080225901BE07B6803F500730722104918462EF0E4
S315080225A0EDFF0346002B10D17B6803F5007318462E
S315080225B0FDF78CFF0346072B07D10DF0DDFD034619
S315080225C0032118460DF015FEFFE700BF1037BD467A
S315080225D080BD00BFAC500508B8500508C4500508B0
S315080225E080B584B000AFF8600B467A60FB7215F0CE
S315080225F0A5FD0346184615F00DFE00BF1037BD4669
S3150802260080BD000080B586B000AFF8600B467A60E0
S31508022610FB7200237B617B6803F5007303224C4936
S3150802262018462EF0ABFF0346002B22D17B6803F532
S3150802263000731846FDF74AFF0346032B19D17B6838
S3150802264003F5806318462DF08FFE78617B69002BAF
S3150802265007D015F073FD03460121184615F082FED0
S3150802266071E015F06BFD03460121184615F097FE39
S3150802267069E07B6803F500730522364918462EF091
S315080226807DFF0346002B22D17B6803F500731846AB
S31508022690FDF71CFF0346052B19D17B6803F58063FA
S315080226A018462DF061FE78617B69002B07D015F07C
S315080226B045FD03460421184615F054FE43E015F07D
S315080226C03DFD03460421184615F069FE3BE07B688A
S315080226D003F500730322204918462EF04FFF0346DE
S315080226E0002B30D17B6803F500731846FDF7EEFE22
S315080226F00346032B27D17B6803F5806318462DF022
S3150802270033FE78617B69002B0ED015F017FD034660
S315080227100121184615F026FE15F010FD0346042180
S31508022720184615F01FFE0EE015F008FD03460121B6
S31508022730184615F034FE15F001FD03460421184625
S3150802274015F02DFEFFE700BF1837BD4680BD00BF56
S31508022750CC500508D0500508D850050880B584B075
S3150802276000AFF8600B467A60FB727B6803F500736C
S315080227701A78B54B1B78D31A002B12D17B6803F54E
S3150802278000731846FDF7A2FE0346012B09D1AF488E
S3150802279018F098F8AE4818F095F8AE4818F092F87E
S315080227A04FE27B6803F500730B22AB4918462EF0FD
S315080227B0E5FE0346002B40F0C5817B6803F50073EE
S315080227C01846FDF783FE03460B2B40F0BB817B6858
S315080227D003F580630922A14918462EF0CFFE034667
S315080227E0002B6FD17B6803F580631846FDF76EFEF2
S315080227F00346092B66D17B6803F5C0631A78984BA2
S315080228001B78D31A002B08D17B6803F5C0631846D8
S31508022810FDF75CFE0346012B13D07B6803F5C06304
S315080228200222904918462EF0A9FE0346002B13D120
S315080228307B6803F5C0631846FDF748FE0346022B7C
S315080228400AD115F07BFC03460121184615F0C9FD8D
S31508022850854818F037F834E07B6803F5C0631A78C0
S31508022860824B1B78D31A002B08D17B6803F5C06309
S315080228701846FDF72BFE0346012B13D07B6803F59A
S31508022880C06303227A4918462EF078FE0346002BC7
S3150802289013D17B6803F5C0631846FDF717FE034696
S315080228A0032B0AD115F04AFC03460121184615F0F6
S315080228B0B5FD704818F006F803E06F4818F002F8FC
S315080228C0BFE13EE17B6803F5806309226B4918463E
S315080228D02EF054FE0346002B6FD17B6803F5806306
S315080228E01846FDF7F3FD0346092B66D17B6803F507
S315080228F0C0631A785A4B1B78D31A002B08D17B6807
S3150802290003F5C0631846FDF7E1FD0346012B13D014
S315080229107B6803F5C0630222524918462EF02EFE42
S315080229200346002B13D17B6803F5C0631846FDF7EF
S31508022930CDFD0346022B0AD115F000FC03460221FF
S31508022940184615F04EFD4E4817F0BCFF34E07B687A
S3150802295003F5C0631A78454B1B78D31A002B08D1A6
S315080229607B6803F5C0631846FDF7B0FD0346012BE5
S3150802297013D07B6803F5C06303223D4918462EF03F
S31508022980FDFD0346002B13D17B6803F5C063184689
S31508022990FDF79CFD0346032B0AD115F0CFFB034630
S315080229A00221184615F03AFD364817F08BFF03E068
S315080229B0314817F087FF44E1C3E07B6803F580637B
S315080229C00922314918462EF0D9FD0346002B40F05C
S315080229D095807B6803F580631846FDF777FD034605
S315080229E0092B40F08B807B6803F5C0631A781C4B71
S315080229F01B78D31A002B08D17B6803F5C0631846E7
S31508022A00FDF764FD0346012B13D07B6803F5C0630B
S31508022A100222144918462EF0B1FD0346002B37D17F
S31508022A207B6803F5C0631846FDF750FD0346022B83
S31508022A302ED115F083FB03460421184615F0D1FC66
S31508022A40124817F03FFF58E0644B0508DC500508AA
S31508022A50F4500508345105087851050884510508CB
S31508022A60FC4C05089051050894510508C44C050804
S31508022A70444E0508C4510508F451050808520508CC
S31508022A80145205084452050874520508805205086E
S31508022A907B6803F5C0631A786B4B1B78D31A002B35
S31508022AA008D17B6803F5C0631846FDF70FFD034698
S31508022AB0012B13D07B6803F5C063032263491846CA
S31508022AC02EF05CFD0346002B13D17B6803F5C06329
S31508022AD01846FDF7FBFC0346032B0AD115F02EFB1D
S31508022AE003460421184615F099FC594817F0EAFEE0
S31508022AF003E0584817F0E6FEA3E022E07B6803F5F8
S31508022B0080631A78544B1B78D31A002B15D17B682D
S31508022B1003F580631846FDF7D9FC0346012B0CD151
S31508022B204E4817F0CFFE4E4817F0CCFE4D4817F028
S31508022B30C9FE4D4817F0C6FE03E0464817F0C2FE26
S31508022B407FE07EE07B6803F5007309224749184651
S31508022B502EF014FD0346002B6FD17B6803F5007334
S31508022B601846FDF7B3FC0346092B66D17B6803F5C5
S31508022B7080631A783E4B1B78D31A002B08D17B68E0
S31508022B8003F580631846FDF7A1FC0346012B13D013
S31508022B907B6803F580630222364918462EF0EEFC5E
S31508022BA00346002B13D17B6803F580631846FDF7AD
S31508022BB08DFC0346022B0AD115F0C0FA03460821FA
S31508022BC0184615F00EFC2C4817F07CFE34E07B689C
S31508022BD003F580631A781C4B1B78D31A002B08D18D
S31508022BE07B6803F580631846FDF770FC0346012BE4
S31508022BF013D07B6803F580630322144918462EF026
S31508022C00BDFC0346002B13D17B6803F58063184687
S31508022C10FDF75CFC0346032B0AD115F08FFA03462F
S31508022C200821184615F0FAFB144817F04BFE03E084
S31508022C30084817F047FE04E003E0064817F042FE8C
S31508022C4000BF1037BD4680BDC44C0508444E050872
S31508022C50B0520508F4510508644B0508E052050808
S31508022C6004530508345305086453050894530508A4
S31508022C70FC4C050890510508A0530508CC530508D5
S31508022C8080B586B000AFF8600B467A60FB72002307
S31508022C907B61FB7A022B40F210817B6803F5007395
S31508022CA00322A94918462EF069FC0346002B34D1A3
S31508022CB07B6803F500731846FDF708FC0346032BE9
S31508022CC02BD17B6803F5806318462DF04DFB78619E
S31508022CD07B69002B1DDB7B69FF2B1ADC0DF0E6F9FD
S31508022CE00346022118460DF012FA0DF0DFF90246E4
S31508022CF07B69DBB2194610460DF018FA934817F0AD
S31508022D00E1FD7969924817F0DDFD924817F0DAFD80
S31508022D1016E1914817F0D6FD12E17B6803F50073B8
S31508022D2004228E4918462EF029FC0346002B34D17C
S31508022D307B6803F500731846FDF7C8FB0346042BA8
S31508022D402BD17B6803F5806318462DF00DFB78615D
S31508022D507B69002B1DDB7B69FF2B1ADC0DF0A6F9BC
S31508022D600346072118460DF0D2F90DF09FF90246DF
S31508022D707B69DBB2194610460DF0D8F9784817F088
S31508022D80A1FD7969724817F09DFD724817F09AFD00
S31508022D90D6E0714817F096FDD2E07B6803F500731A
S31508022DA00422704918462EF0E9FB0346002B34D15B
S31508022DB07B6803F500731846FDF788FB0346042B68
S31508022DC02BD17B6803F5806318462DF0CDFA78611E
S31508022DD07B69002B1DDB7B69FF2B1ADC0DF066F97C
S31508022DE00346082118460DF092F90DF05FF90246DE
S31508022DF07B69DBB2194610460DF098F95A4817F066
S31508022E0061FD7969524817F05DFD524817F05AFD7F
S31508022E1096E0514817F056FD92E07B6803F5007379
S31508022E200422524918462EF0A9FB0346002B40D12C
S31508022E307B6803F500731846FDF748FB0346042B27
S31508022E4037D17B6803F5806318462DF08DFA7861D1
S31508022E507B69012B0BD10DF029F903460921184686
S31508022E600DF055F90F21424817F02CFD68E07B69F1
S31508022E70022B0BD10DF01AF903460A2118460DF05A
S31508022E8046F919213B4817F01DFD59E07B69032BCA
S31508022E900BD10DF00BF903460B2118460DF037F945
S31508022EA02321354817F00EFD4AE02B4817F00AFD94
S31508022EB046E0294817F006FD42E0FB7A012B3BD98A
S31508022EC07B6803F5007302222C4918462EF056FB3E
S31508022ED00346002B10D17B6803F500731846FDF7ED
S31508022EE0F5FA0346022B07D10DF0E0F80346052151
S31508022EF018460DF00CF923E07B6803F500730422EB
S31508022F001F4918462EF03AFB0346002B10D17B6860
S31508022F1003F500731846FDF7D9FA0346042B07D1C1
S31508022F200DF0C4F80346062118460DF0F0F807E03E
S31508022F30094817F0C7FC03E0074817F0C3FC00BFAF
S31508022F401837BD4680BD00BFF8530508FC5305086F
S31508022F500C54050814540508F451050824540508A8
S31508022F602C540508405405084854050860540508B9
S31508022F706854050888540508A8540508C85405085D
S31508022F80CC54050880B586B000AFF8600B467A6067
S31508022F90FB7200233B6100237B617B6803F50073A8
S31508022FA00522B04918462EF0E9FA0346002B11D13C
S31508022FB07B6803F500731846FDF788FA0346052B66
S31508022FC008D1A94B01221A70A84817F07BFC08F011
S31508022FD0C1FE4BE37B6803F500730622A449184633
S31508022FE02EF0CCFA0346002B26D17B6803F5007334
S31508022FF01846FDF76BFA0346062B1DD19A4B01229A
S315080230001A709C4817F05EFC0FF096FA0346DAB27D
S31508023010994B1A70984B1B78012B04D1974817F0D5
S3150802302051FC00BF22E30A2024F03AFC944B1B7899
S31508023030184617F085FDE7E77B6803F50073052256
S31508023040904918462EF09AFA0346002B11D17B684E
S3150802305003F500731846FDF739FA0346052B08D11E
S31508023060814B01221A70884817F02CFC08F0BCFE26
S31508023070FCE27B6803F500730522844918462EF0A4
S315080230807DFA0346002B11D17B6803F500731846B7
S31508023090FDF71CFA0346052B08D1734B01221A7059
S315080230A07B4817F00FFC08F087FEDFE27B6803F522
S315080230B000730522774918462EF060FA0346002B5C
S315080230C011D17B6803F500731846FDF7FFF903462D
S315080230D0052B08D1644B01221A706F4817F0F2FBD0
S315080230E008F0B4FEC2E27B6803F5007308226B4956
S315080230F018462EF043FA0346002B10D17B6803F5D7
S3150802310000731846FDF7E2F90346082B07D108F0C3
S31508023110F9FD53EC102B624817F0D4FBA6E27B6844
S3150802312003F5007308225F4918462EF027FA03466C
S31508023130002B26D17B6803F500731846FDF7C6F9FE
S315080231400346082B1DD1484B01221A707B6803F5EA
S31508023150806318462DF008F938613B69002B0CDBB1
S315080231603B69642B09DC39694F4817F0ABFB3B69AD
S31508023170DBB2184608F046FD78E24C4817F0A2FB87
S3150802318074E27B6803F500730822494918462EF053
S31508023190F5F90346002B13D17B6803F5007318462D
S315080231A0FDF794F90346082B0AD1424817F08AFB21
S315080231B00CF0E2FF0346FE2118460DF0AAF855E286
S315080231C07B6803F500730B223B4918462EF0D6F9A5
S315080231D00346002B13D17B6803F500731846FDF7E7
S315080231E075F903460B2B0AD1344817F06BFB14F01A
S315080231F0A5FF03460121184615F060FC36E2FB7A64
S31508023200022B40F2FB807B6803F5007303222C49EC
S3150802321018462EF0B3F90346002B40F085807B68EA
S3150802322003F500731846FDF751F90346032B7BD1C4
S315080232300CF0A2FF0346052118460DF0BDF87B687F
S3150802324003F5806318462DF08FF83861FB7A032B55
S3150802325038D97B6803F5C06318462DF085F878617E
S3150802326032E000BF044F05080AA40020D45405081A
S31508023270E8540508F05405080BA40020045505086F
S31508023280E5A20020E84E050820550508345505082C
S315080232903C55050850550508585505086C55050846
S315080232A0785505088C55050898550508F4510508FA
S315080232B0B0550508BC550508DC550508E855050846
S315080232C0544E0508FF237B613B69002B27DB3B69CC
S315080232D0062B24DC3969B84817F0F4FA0CF04CFFCF
S315080232E002463B69DBB2194610460DF012F87B69B5
S315080232F0002B0CDB7B69062B09DC0CF03DFF024632
S315080233007B69DBB2194610460DF020F80BE00CF08B
S3150802331033FF0346FF2118460DF018F803E0A748C5
S3150802332017F0D0FAA2E1A1E17B6803F50073062241
S31508023330A34918462EF022F90346002B5AD17B6878
S3150802334003F500731846FDF7C1F80346062B51D15B
S315080233507B6803F5806318462DF006F83861FB7A18
S31508023360032B40F283817B6803F5C06318462CF071
S31508023370FBFF78613B69002B38DB3B69062B35DCA2
S315080233807B69002B32DB7B69062B2FDC39698D487A
S3150802339017F098FA79698C4817F094FA14F0CEFE69
S315080233A003460121184615F015FC0CF0E5FE034606
S315080233B0FF2118460CF0CAFF0CF0DEFE02463B69F6
S315080233C0DBB2194610460CF0A4FF0CF0D5FE0246F5
S315080233D07B69DBB2194610460CF0D3FF0CF0CCFE23
S315080233E00346012118460CF0E7FF3FE1774817F03C
S315080233F069FA3BE1714817F065FA37E1FB7A022B65
S3150802340040F030817B6803F500730822704918463C
S315080234102EF0B4F80346002B0FD17B6803F5007330
S315080234201846FDF753F80346082B06D101200FF07C
S3150802343031F8684817F046FA18E17B6803F5007315
S315080234400822654918462EF099F80346002B1BD127
S315080234507B6803F500731846FDF738F80346082B10
S3150802346012D114F06BFE03460121184615F0C3FA71
S3150802347026F0D6FA03460322584918462CF014F9C0
S31508023480574817F01FFAF1E07B6803F50073072225
S31508023490544918462EF072F80346002B18D17B6859
S315080234A003F500731846FDF711F80346072B0FD1EB
S315080234B014F044FE03460121184615F09CFA03222D
S315080234C049494A482CF0F0F8494817F0FBF9CDE08B
S315080234D07B6803F500730422464918462EF04EF817
S315080234E00346002B11D17B6803F500731846FCF7D7
S315080234F0EDFF0346042B08D103223F493B482CF033
S31508023500D3F83E4817F0DEF9B0E07B6803F500739E
S3150802351007223B4918462EF031F80346002B11D1F3
S315080235207B6803F500731846FCF7D0FF0346072BA2
S3150802353008D1032233492D482CF0B6F8324817F041
S31508023540C1F993E07B6803F5007308222F491846F0
S315080235502EF014F80346002B11D17B6803F500738D
S315080235601846FCF7B3FF0346082B08D1032228495D
S315080235701E482CF099F8274817F0A4F976E07B68DC
S3150802358003F500730722244918462DF0F7FF034670
S31508023590002B47D17B6803F500731846FCF796FFA4
S315080235A00346072B3ED103221C4910482CF07CF80F
S315080235B01B4817F087F959E000560508F451050823
S315080235C01C56050824560508485605086C5605086B
S315080235D0B84C050888560508A05605083016002076
S315080235E0AC560508D0560508381600200200040015
S315080235F0D8560508FC560508401600200457050843
S315080236001C57050848160020245705084057050880
S31508023610501600204C570508705705085816002002
S31508023620785705087B6803F500730722114918467F
S315080236302DF0A4FF0346002B10D17B6803F5007317
S315080236401846FCF743FF0346072B07D10DF0FCF992
S3150802365003461946084817F035F907E0074817F0F0
S3150802366031F903E0054817F02DF900BF1837BD46B2
S3150802367080BD00BF98570508A0570508F4510508EC
S3150802368080B584B000AFF8600B467A60FB7208F02A
S3150802369027F90346184608F059F90346012B03D1C0
S315080236A02A4817F00FF902E0294817F00BF908F033
S315080236B017F903460021184608F06FF90346012B4D
S315080236C003D1244817F0FEF802E0234817F0FAF867
S315080236D008F006F903460121184608F05EF9034682
S315080236E0012B03D11D4817F0EDF802E01C4817F02C
S315080236F0E9F808F0F5F803460221184608F04DF9EC
S315080237000346012B03D1174817F0DCF802E01648E6
S3150802371017F0D8F808F0E4F803460321184608F02B
S315080237203CF90346012B03D1104817F0CBF802E007
S315080237300F4817F0C7F80DF087F9034619460D48E2
S3150802374017F0C0F800BF1037BD4680BDBC57050844
S31508023750D4570508EC5705080858050824580508DB
S31508023760405805085C58050878580508945805080D
S31508023770B0580508CC58050880B586B000AFF86081
S315080237800B467A60FB7200237B61FB7A012B4BD9CD
S315080237907B6803F5007318462CF0E6FD78617B69B1
S315080237A0002B3DDD7B69052B3ADC7969224817F047
S315080237B089F87B69012B07D108F03AF803460121FB
S315080237C0184608F05AF833E07B69022B07D108F04D
S315080237D02FF803460221184608F04FF828E07B69BD
S315080237E0032B07D108F024F803460321184608F0EC
S315080237F044F81DE07B69042B07D108F019F8034643
S315080238000421184608F039F812E07B69052B0FD116
S3150802381008F00EF803460521184608F02EF807E0C8
S31508023820064817F04FF804E0044817F04BF800E092
S3150802383000BF1837BD4680BDEC580508F451050887
S3150802384080B584B000AFF8600B467A60FB7208F068
S3150802385047F803460021184608F0EDF80346012BFF
S3150802386003D1304817F02EF802E02F4817F02AF84D
S3150802387008F036F803460121184608F0DCF8034634
S31508023880012B03D1294817F01DF802E0284817F042
S3150802389019F808F025F803460221184608F0CBF86D
S315080238A00346012B03D1234817F00CF802E02248FD
S315080238B017F008F808F014F803460321184608F02A
S315080238C0BAF80346012B03D11C4816F0FBFF02E0A7
S315080238D01B4816F0F7FF08F003F8034604211846BA
S315080238E008F0A9F80346012B03D1164816F0EAFF99
S315080238F002E0154816F0E6FF07F0F2FF0346052137
S31508023900184608F098F80346012B03D10F4816F01B
S31508023910D9FF03E00E4816F0D5FF00BF1037BD46A3
S3150802392080BD00BFFC5805080C5905081C59050836
S315080239302C5905083C5905084C5905085C590508CF
S315080239406C5905087C5905088C5905089C590508BF
S31508023950AC59050880B586B000AFF8600B467A60A8
S31508023960FB7200237B6100233B61FB7A022B40F248
S3150802397091807B6803F5007318462CF0F5FC786194
S315080239807B6803F5806318462CF0EEFC38617B6988
S31508023990002B7BDD7B69052B78DC3B69012B3AD151
S315080239A07969404816F08EFF7B69012B07D107F02B
S315080239B03FFF03460621184607F05FFF6EE07B6964
S315080239C0022B07D107F034FF03460721184607F0F2
S315080239D054FF63E07B69032B07D107F029FF0346EF
S315080239E00821184607F049FF58E07B69042B07D1DE
S315080239F007F01EFF03460921184607F03EFF4DE071
S31508023A007B69052B4AD107F013FF03460A2118469C
S31508023A1007F033FF42E07969234816F053FF7B69C2
S31508023A20012B07D107F004FF03460B21184607F0BE
S31508023A3024FF33E07B69022B07D107F0F9FE034620
S31508023A400C21184607F019FF28E07B69032B07D1DA
S31508023A5007F0EEFE03460D21184607F00EFF1DE09D
S31508023A607B69042B07D107F0E3FE03460E211846AD
S31508023A7007F003FF12E07B69052B0FD107F0D8FE8A
S31508023A8003460F21184607F0F8FE07E0074816F026
S31508023A9019FF04E0054816F015FF00E000BF1837C5
S31508023AA0BD4680BDBC590508D8590508F451050814
S31508023AB080B586B000AFF8600B467A60FB720023C9
S31508023AC0FB75FB7A022B60D97B6803F50073042227
S31508023AD0334918462DF052FD0346002B55D17B6813
S31508023AE003F500731846FCF7F1FC0346042B4CD188
S31508023AF07B6803F580631A782A4B1B78D31A002B46
S31508023B0010D17B6803F580631846FCF7DFFC034691
S31508023B10012B07D1244B01221A7008F0F1F908F09B
S31508023B2013FA32E07B6803F580631A781F4B1B7819
S31508023B30D31A002B10D17B6803F580631846FCF76D
S31508023B40C5FC0346012B07D1174B01221A7008F050
S31508023B50D7F908F00DFA18E07B6803F580630422AA
S31508023B60134918462DF00AFD0346002B0DD17B6832
S31508023B7003F580631846FCF7A9FC0346042B04D117
S31508023B80094B00221A7008F0CDF9FB7D002B02D0F2
S31508023B90084816F097FE00BF1837BD4680BD00BF1D
S31508023BA0F0590508E84D0508008D0020244E050841
S31508023BB0F8590508F45105082DE9F0418EB002AF0F
S31508023BC0F8600B467A60FB7214F0B8FA0346184698
S31508023BD014F008FBF8620023BB6200237B62002311
S31508023BE03B620023FB610023BB6100237B617B6888
S31508023BF003F5007304226C4918462DF0BFFC0346F0
S31508023C00002B0FD17B6803F500731846FCF75EFCA0
S31508023C100346042B06D1654816F054FEF86AFDF7EA
S31508023C204BFBE0E17B6803F5007304226049184602
S31508023C302DF0A4FC0346002B4ED17B6803F50073D6
S31508023C401846FCF743FC0346042B45D1F86AFDF7F0
S31508023C5069FB03461946574816F034FEF86AFDF71B
S31508023C607BFB03461946544816F02CFE0021F86AD7
S31508023C70FDF78DFB03461D460121F86AFDF787FB12
S31508023C8003461E460221F86AFDF781FB034698465B
S31508023C900321F86AFDF77BFB03461C460421F86AF2
S31508023CA0FDF775FB034601930094434632462946BF
S31508023CB0424816F007FEF86AFDF79DFB03461946C9
S31508023CC03F4816F0FFFDF86AFDF7B0FB03461946B2
S31508023CD03C4816F0F7FD86E17B6803F5007311226E
S31508023CE0394918462DF04AFC0346002B20D17B6839
S31508023CF003F500731846FCF7E9FB0346112B17D1A7
S31508023D007B6803F5806318462CF02EFBB862B96A05
S31508023D102E4816F0D7FDBB6A002B05DDBB6A19468D
S31508023D20F86AFDF70BFB5EE1294816F0CBFD5AE16E
S31508023D307B6803F500730E22264918462DF01EFCF1
S31508023D400346002B4CD17B6803F500731846FCF733
S31508023D50BDFB03460E2B43D17B6803F580631846E9
S31508023D602CF002FBB862BB6A002B0AD1B96A1A4860
S31508023D7016F0A8FDBB6ADBB21946F86AFDF7F8FA2F
S31508023D8031E1BB6A012B0AD1B96A144816F09AFDC9
S31508023D90BB6ADBB21946F86AFDF7EAFA23E10C4870
S31508023DA016F090FD1FE100BF005A0508085A0508DB
S31508023DB01C5A0508245A0508505A05088C5A05083B
S31508023DC0BC5A0508EC5A0508345B0508485B050821
S31508023DD0F4510508785B0508885B0508C05B050889
S31508023DE07B6803F500730A22814918462DF0C6FB43
S31508023DF00346002B40F098807B6803F5007318464B
S31508023E00FCF764FB03460A2B40F08E807B6803F5B9
S31508023E10806318462CF0A8FA78627B6803F5C063BB
S31508023E2018462CF0A1FA38627B6803F50063184637
S31508023E302CF09AFAF8617B6803F5206318462CF091
S31508023E4093FAB8617B6803F5406318462CF08CFA3E
S31508023E5078617B6A002B02D07B6A012B60D13B6AB0
S31508023E60002B02D03B6A012B5AD1FB69002B02D0E8
S31508023E70FB69012B54D1BB69002B02D0BB69012B0C
S31508023E804ED17B69002B02D07B69012B48D17B6A14
S31508023E90DBB21A460021F86AFDF78EFA3B6ADBB2F4
S31508023EA01A460121F86AFDF787FAFB69DBB21A4658
S31508023EB00221F86AFDF780FABB69DBB21A460321CA
S31508023EC0F86AFDF779FA7B69DBB21A460421F86AC1
S31508023ED0FDF772FA0021F86AFDF759FA03461D46FC
S31508023EE00121F86AFDF753FA03461E460221F86ACB
S31508023EF0FDF74DFA034698460321F86AFDF747FA95
S31508023F0003461C460421F86AFDF741FA0346019363
S31508023F100094434632462946364816F0D3FC62E0F8
S31508023F20354816F0CFFC5EE07B6803F5007307227E
S31508023F30324918462DF022FB0346002B27D17B680F
S31508023F4003F500731846FCF7C1FA0346072B1ED180
S31508023F507B6803F5806318462CF006FAB862BB6ADA
S31508023F60002B02D0BB6A002B0DDDBB6A032B0ADCD1
S31508023F70B96A234816F0A6FCBB6ADBB21946F86A88
S31508023F80FDF760FA2FE01F4816F09CFC2BE07B68D1
S31508023F9003F500731A781C4B1B78D31A002B1ED113
S31508023FA07B6803F500731846FCF790FA0346012B63
S31508023FB015D1164816F086FC154816F083FC1548E6
S31508023FC016F080FC144816F07DFC144816F07AFCAC
S31508023FD0134816F077FC134816F074FC03E00648FB
S31508023FE016F070FC00BF3037BD46BDE8F08100BF51
S31508023FF0F85B0508045C0508F4510508305C0508F9
S31508024000385C0508044E0508644B05085C5C05081F
S31508024010785C0508945C0508B45C05080C5D05081F
S315080240206C5D0508C05D050890B585B000AF78607F
S315080240300023BB730023FB734FF4A05200212048D0
S315080240402DF094FA07F10E030A221D49786825F025
S31508024050B1F80346012B2ED10023FB7328E0FB7B24
S315080240604FF48E7202FB03F3164A13449C1C14483F
S31508024070FCF72CFA03461A46114920462DF07EFA19
S315080240800346002B11D1FB7B0E4A4FF48E7101FBBE
S3150802409003F3134418331B68B97B094A002098476F
S315080240A0094816F00FFC012306E0FB7B0133FB737C
S315080240B0FB7B132BD3D9002318461437BD4690BD74
S315080240C0048D002000000020544B050880B582B0FC
S315080240D000AF0346FB71FB790D2B24D14F4B00220F
S315080240E01A704F4816F0EEFB4E4B1B78002B16D073
S315080240F04D48FFF799FF0346012B08D1F02200210C
S315080241004A482DF033FA484948482DF0D0FA454B2B
S3150802411000221A70F022002143482DF027FA44485B
S3150802412016F0D0FB76E0FB790A2B03D13B4B002233
S315080241301A706FE0FB791B2B03D1384B01221A70D8
S3150802414068E0FB795B2B07D1344B1B78012B03D133
S31508024150324B02221A705DE0FB79412B1FD12F4B9D
S315080241601B78022B1BD12D4B00221A702D4B1B7864
S31508024170002B4FD12D492F4816F0A4FB2B48FCF7EC
S31508024180A5F90346DAB2274B1A70F022002126480F
S315080241902DF0ECF9254924482DF089FA3AE0FB7905
S315080241A0082B02D0FB797F2B16D11C4B00221A70E2
S315080241B01C4B1B78002B2DD01A4B1B78013BDAB20D
S315080241C0184B1A70174B1B781A46174B002199542D
S315080241D0194816F077FB1DE0124B1B785A1CD1B210
S315080241E0104A11701946104AFB7953540D4B1A7826
S315080241F0124BA3FB0213D9090B461B015B1A1B01BF
S31508024200D31ADAB2074B1A70FB7919460C4816F01C
S3150802421059FBFFE700BF0837BD4680BD0CA4002046
S31508024220544B0508E4A20020F4A1002004A10020B2
S31508024230145E05084C4B0508185E050889888888A7
S315080242401C5E050880B58EB008AF786000237B61D6
S315080242507B683B6107F10C0100234FF40072386951
S3150802426024F0B4F80346002B01D0022367E0FB686A
S31508024270B022069201220592002204920A22039291
S315080242800A2202924FF400720192009300232E4AE8
S315080242902E492F4824F0A4FA0346002B01D00E23F8
S315080242A04DE006220C212B4816F0A0FB786816F082
S315080242B03BF9786816F0AEF9786816F0D9F8786896
S315080242C014F0F8FD1C2301222349244824F092F90C
S315080242D01C2301222249234824F08CF91C2301229B
S315080242E02149224824F086F91C2301222049214823
S315080242F024F080F91C2301221F49204824F07AF968
S315080243001C2301221E491F4824F074F91C2301228A
S315080243101D491E4824F06EF91C2301221C491D481A
S3150802432024F068F91C2301221B491C4824F062F96F
S315080243301C2301221A491B4824F05CF97B6918469A
S315080243401837BD4680BD00BFA9430208285E050886
S3150802435010A40020385E0508485E0508C0A400209F
S315080243605C5E0508DCA40020805E0508F8A400202F
S31508024370985E050814A50020B05E050830A5002041
S31508024380C45E0508A0A50020DC5E050884A50020F9
S31508024390F85E05084CA50020085F050868A50020F8
S315080243A0185F0508BCA5002080B584B000AF786008
S315080243B07B68BB600023FB731C4816F083FA1C4912
S315080243C01C4816F07FFA1C491C4816F07BFA1C4852
S315080243D016F078FA1B4B1B780133DAB2194B1A70AE
S315080243E0184B1B78092B18D9164B00221A7016F08F
S315080243F0D5FB4FF48061144818F000FBFB7B032BB6
S3150802440005D10AF0C7FBFB7B0133FB7305E0FB7B97
S31508024410032B02D8FB7B0133FB73BB68DBB218465E
S3150802442016F08EFB642023F03BFAD3E7405F0508BB
S31508024430685F0508705F0508805F05088C5F0508D8
S31508024440A45F0508D8A500200018024280B500AF6F
S3150802445022F0C6FE00BF80BD80B400AF034B1B68C6
S315080244601846BD465DF8047B704700BFDCA50020F0
S3150802447080B500AF4FF400620E490F4824F004FFDE
S315080244804FF400620D490E4824F0FEFE4FF4007206
S315080244900C490D4824F0F8FE4FF400620B490C480B
S315080244A024F0F2FE4FF400620A490B4824F0ECFEAF
S315080244B000BF80BDF0A50020E0A5002000AE0020C8
S315080244C0F0AD002034B6002024B6002074B80020CF
S315080244D034B80020B4C0002074C0002084B0B0B440
S315080244E000AF07F10C0484E80F00074B1D4607F1DD
S315080244F00C040FCC0FC50FCC0FC523682B6000BF69
S31508024500BD46B0BC04B0704700B6002080B586B080
S3150802451000AF78600B467B800023FB7500233B6166
S315080245200023FB600023BB6000F0E6FC0346002B79
S315080245300BD0444BD3F844323B61424BD3F8843A0E
S31508024540FB607B681B68BB600AE03E4BD3F84432CB
S315080245503B613C4BD3F8843AFB607B681B68BB60C3
S315080245603A69BB689A4227D1364B93F86832002BD0
S315080245700AD1344BD3F850227B881344314AC2F805
S3150802458050320123FB7558E02E4BB3F86C321A46AB
S315080245907B881344B3F5006F0BDA2A4BB3F86C2207
S315080245A07B8813449AB2274BA3F86C220123FB7526
S315080245B043E00023FB7540E0FA68BB689A4227D1BC
S315080245C0204B93F8A83A002B0AD11E4BD3F8502257
S315080245D07B8813441B4AC2F850320223FB752CE02F
S315080245E0184BB3F8AC3A1A467B881344B3F5006FF6
S315080245F00BDA144BB3F8AC2A7B8813449AB2114BE4
S31508024600A3F8AC2A0223FB7517E00023FB7514E016
S315080246103B69002B07D1242279680B482DF05DF8F7
S315080246200123FB7509E0FB68002B06D12422796871
S3150802463006482DF052F80223FB75FB7D18461837FB
S31508024640BD4680BD00B6002044B8002084C00020C4
S3150802465080B584B000AF03463960FB711346BB8050
S315080246600023FB81FB79012B12D10023FB810AE08F
S31508024670FB893A68134401221946124824F0AAFE15
S31508024680FB890133FB81FA89BB889A42F0D314E08D
S31508024690FB79022B11D10023FB810AE0FB893A68D8
S315080246A0134401221946084824F094FEFB89013373
S315080246B0FB81FA89BB889A42F0D300BF1037BD4600
S315080246C080BD00BF34B8002074C0002080B582B017
S315080246D000AF0346FB71FB1D01221946074824F069
S315080246E079FE0346002B04D1FB791946044816F0D5
S315080246F0E9F800BF0837BD4680BD00BF24B60020D2
S31508024700CC5F0508F0B5ABB008AFF861B9617A615C
S315080247100023C7F88430F86916F07BFFC7F88000D3
S315080247200023C7F8843051E0D7F884305A1CC7F8FA
S315080247308420B3F5FA7F49D907F150031946F86977
S3150802474017F09AF83B6D3B617A6DFA60B86DB860FE
S31508024750FB6D3A6E796EB86EFC6E7C603D6F7E6F4D
S31508024760BC6F0794069605957C680494039002919B
S3150802477001920093BB68FA683969314816F0A2F8C3
S315080247807B6E002B07D0FB691B689A69FB691B685D
S3150802479022F001029A61F86916F03BFFC7F8800019
S315080247A0D7F88010F86916F040FF0023C7F884305E
S315080247B013F0C4FC03460121184613F0B6FD03465E
S315080247C0002B0BD01F4816F07DF807E00721F86981
S315080247D017F0A2F80346002BA6D100E000BF7A69BB
S315080247E0B969F86916F0D1FEF86900F0FFFA0346CE
S315080247F0FB67FB6F002B1ED007F120033022002136
S3150802480018462CF0B3FEF86900F0B6FA03460E4ACB
S315080248101360F86900F0CBFA03460B4A53600A4B59
S315080248201A68094B5B6807F1200008492CF00AFE52
S31508024830F86F00F02FFB00BF8C37BD46F0BD00BFF6
S31508024840F45F050838600508B4C800205C600508EE
S3150802485080B592B000AF3B464022002118462CF0A4
S3150802486085FE0023A7F8423000237B64974824F08C
S3150802487095FD034683F00103DBB2002B00F0E980C5
S31508024880934B93F86832002B62D1914BD3F850328E
S315080248909AB28F4BA3F86C228D4B0F22C3F8502283
S315080248A010233B703B785AB2894BB3F86C321B0A19
S315080248B09BB25BB203F00F035BB213435BB2DBB28C
S315080248C03B70834BB3F86C32DBB27B703B460233E8
S315080248D03E2219467D4824F0B8FD0346002B33D004
S315080248E04FF47A717B4823F01BFF0346002B0AD14B
S315080248F0FFF7B2FD3B461A467749FFF703FF7548AD
S3150802490023F050FF02E0754815F0DCFF704BB3F850
S315080249106C323E3B9AB26E4BA3F86C226C4BB3F8E0
S315080249206A3201339AB26A4BA3F86A22684B0122A9
S3150802493083F86822664BFF2283F86E22644B4FF493
S31508024940FA62C3F8702221E1654815F0BBFF1DE142
S315080249505F4B93F86E32002B05D05D4B93F86E329F
S31508024960012B40F013815A4BB3F86C323E2B02D915
S3150802497040237B6404E0564BB3F86C3201337B6404
S3150802498020233B703B785AB2514BB3F86A325BB27A
S3150802499003F00F035BB213435BB2DBB23B707B6C73
S315080249A05A1E3B4601331946484824F04EFD034633
S315080249B0002B4AD04FF47A71464823F0B1FE0346DB
S315080249C0002B13D17B6C9BB2184600F0C5FA03463E
S315080249D03F4AC2F85032FFF73FFD3B461A463E4968
S315080249E0FFF790FE3B4823F0DDFE02E03D4815F056
S315080249F069FF374BB3F86C227B6C9BB2D31A9BB216
S31508024A0001339AB2324BA3F86C22314BB3F86A32AD
S31508024A1001339AB22E4BA3F86A222D4BB3F86C32A5
S31508024A20002B40F0B380242200212B482CF09EFD57
S31508024A30274B002283F86822254B0022A3F86A2214
S31508024A40234BFF2283F86E22A0E0274815F03AFF8F
S31508024A509CE0264824F0A2FC034683F00103DBB25D
S31508024A60002B00F093803B46012219461F4824F08A
S31508024A70ECFC0346002B00F086803B781B09DBB270
S31508024A80032B37D13B46013302221946174824F035
S31508024A90DCFC0346002B79D00D4B0322DA604FF477
S31508024AA07A710C4823F03CFE0346002B0AD1FFF725
S31508024AB0D3FC3B461A460649FFF724FE054823F06F
S31508024AC071FE63E00A4815F0FDFE5FE034B8002087
S31508024AD000B6002030A5002044B8002084600508EE
S31508024AE0A4600508B8600508D860050824B6002041
S31508024AF0EC6005083B781B09DBB2002B46D13B4626
S31508024B00013301221946234824F09FFC0346002B51
S31508024B103BD03B781B029BB203F47063A7F8423082
S31508024B207B781A46B7F842301343A7F84230B7F8EB
S31508024B3042203B4602331946164824F086FC0346B1
S31508024B40002B23D0B7F8423002339BB2184600F046
S31508024B5003FA0346104AD3604FF47A710F4823F0DA
S31508024B60DFFD0346002B0AD1FFF776FC3B461A46C1
S31508024B700949FFF7C7FD094823F014FE06E008486D
S31508024B8015F0A0FE02E000BF00E000BF4837BD46B0
S31508024B9080BD00BF24B6002000B6002030A5002044
S31508024BA00C61050880B59AB000AF3B466822002121
S31508024BB018462CF0DBFC0E4824F0F0FB034683F083
S31508024BC00103DBB2002B0ED004E03B4668211846EF
S31508024BD000F010F83B4668221946054824F035FCD1
S31508024BE00346002BF1D100BF6837BD4680BD00BF22
S31508024BF0F0AD002080B582B000AF78600B467B80AE
S31508024C00786800F07FFC00BF0837BD4680BD00000B
S31508024C1080B500AF194B93F86832002B2BD0174B8F
S31508024C2093F86E32FF2B26D1144BD3F87032002B31
S31508024C3007D0124BD3F87032013B104AC2F87032D1
S31508024C4019E0242200210E482CF090FC4FF4006251
S31508024C500C490D4824F018FB084B002283F86822F9
S31508024C60064B0022A3F86A22044BFF2283F86E221F
S31508024C70064815F027FE00BF80BD00BF00B600201B
S31508024C8044B8002074B8002034B800202C61050806
S31508024C9080B582B000AF78600B467B80786800F0FA
S31508024CA057FB00BF0837BD4680BD000080B582B0FD
S31508024CB000AF78600B467B807B881A46796806487F
S31508024CC024F088FB0346002B02D1044815F0FAFDAE
S31508024CD000BF0837BD4680BDE0A500204061050833
S31508024CE080B59AB000AF3B466822002118462CF0E0
S31508024CF03DFC0E4824F052FB034683F00103DBB267
S31508024D00002B0ED004E03B4668211846FFF7C0FF89
S31508024D103B4668221946054824F097FB0346002BB2
S31508024D20F1D100BF6837BD4680BD00BFE0A50020AF
S31508024D3080B582B000AF78600B4A7B681360FFF7D4
S31508024D4097FB2422002109482CF010FC242200217A
S31508024D5007482CF00BFC2422002106482CF006FCFE
S31508024D6000BF0837BD4680BDDCA5002000B600207E
S31508024D7044B8002084C0002080B485B000AF7860B3
S31508024D807B681B681B6CBB600023FB60BB68DBB2DD
S31508024D90002B05D0BB68DBB2FB60FB68DBB2FB60AD
S31508024DA0FB6818461437BD465DF8047B704780B425
S31508024DB085B000AF78607B681B681B6CBB600023FC
S31508024DC0FB60BB6803F4FE43002B07D0BB6803F401
S31508024DD0FE43FB60FB681B0ADBB2FB60FB681846F6
S31508024DE01437BD465DF8047B7047000080B485B071
S31508024DF000AF78607B681B685B6CBB600023FB6056
S31508024E00BB6803F00703002B3BD0BB6803F007031C
S31508024E10013B052B2CD801A252F823F0354E020885
S31508024E203F4E0208494E0208534E02085D4E0208DA
S31508024E30674E0208FB6843F00103FB6019E0FB6852
S31508024E4043F00203FB6014E0FB6843F00303FB60D4
S31508024E500FE0FB6843F00403FB600AE0FB6843F0DB
S31508024E600503FB6005E0FB6843F00603FB6000E010
S31508024E7000BF7B681B685A6C7B681B6822F00702B6
S31508024E805A64FB68DBB218461437BD465DF8047BE4
S31508024E90704700BF80B483B000AF78607B68013B7F
S31508024EA0052B10D801A252F823F000BFC54E0208FE
S31508024EB0C54E0208C54E0208C54E0208C54E02086E
S31508024EC0C54E020800BF00BF0C37BD465DF8047B1D
S31508024ED0704700BF80B483B000AF0346FB71054A32
S31508024EE0FB791370012318460C37BD465DF8047B1F
S31508024EF0704700BFCCC8002080B400AF034B1B78B4
S31508024F001846BD465DF8047B704700BFCCC8002032
S31508024F1080B500AFFFF7F0FF0346002B02D04FF42F
S31508024F20807301E04FF48073184680BD80B400AFE9
S31508024F304FF400231846BD465DF8047B704780B5DA
S31508024F4000AFFFF7D9FF0346002B02D040F20B133E
S31508024F5000E00023184680BD80B483B000AF034644
S31508024F60FB80FB88002B01D1002346E0FB88012B3E
S31508024F7001D1012341E0FB88022B01D102233CE047
S31508024F80FB88032B01D1032337E0FB88042B01D1CD
S31508024F90042332E0FB88052B01D105232DE0FB888B
S31508024FA0062B01D1062328E0FB88072B01D107230C
S31508024FB023E0FB88082B01D108231EE0FB880C2B73
S31508024FC001D8092319E0FB88102B01D80A2314E01B
S31508024FD0FB88142B01D80B230FE0FB88182B01D86A
S31508024FE00C230AE0FB88202B01D80D2305E0FB8859
S31508024FF0302B01D80E2300E00F2318460C37BD4686
S315080250005DF8047B704780B483B000AF78607B6834
S31508025010002B01D1002346E07B68012B01D1012335
S3150802502041E07B68022B01D102233CE07B68032B1B
S3150802503001D1032337E07B68042B01D1042332E034
S315080250407B68052B01D105232DE07B68062B01D150
S31508025050062328E07B68072B01D1072323E07B6818
S31508025060082B01D108231EE07B68092B01D80C23E3
S3150802507019E07B680A2B01D8102314E07B680B2BF6
S3150802508001D814230FE07B680C2B01D818230AE0F9
S315080250907B680D2B01D8202305E07B680E2B01D8EF
S315080250A0302300E0402318460C37BD465DF8047BE2
S315080250B07047B0B5A4B006AFF860B9601346FB8076
S315080250C00023A7F87630FB683B65FFF715FF034612
S315080250D0002B03D04FF080437B6501E000237B65FC
S315080250E00023BB65FB8802339BB21846FFF734FFE1
S315080250F00346FB6500233B664FF480137B664FF439
S315080251000013BB660023FB6600233B6700233B7440
S315080251103B7C5AB2FB881B0A9BB25BB203F00F03B5
S315080251205BB213435BB2DBB23B74FB88DBB27B74C4
S315080251300223A7F8763010E0B7F87630023BBA6851
S315080251401A44B7F87630127878333B4403F8682C59
S31508025150B7F876300133A7F87630B7F87620FB88A9
S3150802516001339A42E8DD0023A7F876300DE0B7F856
S31508025170763078333B4413F8683C1846FFF7A6FAAC
S31508025180B7F876300133A7F87630B7F87620FB8879
S3150802519001339A42EBDD6D4607F160040FCC0FC569
S315080251A023682B6007F150030FCBFFF797F900BF6F
S315080251B07837BD46B0BD80B58EB000AFF860B9602D
S315080251C01346FB80002387F83730FB683B61FFF7FD
S315080251D093FE0346002B03D04FF080437B6101E028
S315080251E000237B610023BB61FB88FB6100233B62D2
S315080251F04FF480137B624FF40013BB620023FB62F9
S3150802520000233B63FA8807F1100311461846FFF795
S315080252107DF9034687F8373097F83730002B06D0E2
S31508025220FA8897F83730B9681846FFF711FA00BFB7
S315080252303837BD4680BDB0B5A2B006AF786008461D
S3150802524011461A460346FB700B46BB7013467B7023
S31508025250002387F86F307B68BB64FFF74DFE034671
S31508025260002B03D04FF08043FB6401E00023FB646C
S3150802527000233B6503237B650023BB654FF480133C
S31508025280FB654FF400133B6600237B660023BB666F
S3150802529030233B723B7A5AB297F9033003F00F0375
S315080252A05BB213435BB2DBB23B72BB787B727B7831
S315080252B0BB72002387F86F300DE097F86F307033B2
S315080252C03B4413F8683C1846FFF700FA97F86F3024
S315080252D0013387F86F3097F86F30022BEDD96D4698
S315080252E007F158040FCC0FC523682B6007F1480352
S315080252F00FCBFFF7F3F800BF7037BD46B0BD80B5D8
S3150802530082B000AF78600023002200217868FFF798
S3150802531092FF00BF0837BD4680BD80B584B000AF96
S31508025320F860B9601346FB80FB883E2B06D8FB88DB
S315080253301A46B968F868FFF7BCFE05E0FB881A4604
S31508025340B968F868FFF737FF00BF1037BD4680BD5A
S3150802535080B588B000AF7860FF23FB7600237B61B7
S315080253600023FB6100237B827B68FB60FB6893F862
S3150802537028301B09FB76FB681B687B61FFF7D6FDA5
S3150802538002467B69934202D1FFF7D9FDF861FB7E9B
S31508025390032B00F2A78001A252F823F0AD530208AC
S315080253A0EF5302083954020887540208FB6893F837
S315080253B0283003F00F039AB24C4B1A804B4B1B88CA
S315080253C01B029AB2494B1A80FB6893F829301A468F
S315080253D0464B1B8813439AB2444B1A80FB682A33FE
S315080253E0424A12881146184608F07EFE7AE0FB68A1
S315080253F093F8283003F00F039AB23C4B1A803B4BC2
S315080254001B881B029AB2394B1A80FB6893F829301B
S315080254101A46364B1B8813439AB2344B1A80344BBE
S3150802542001221A70FB682A333E21184608F05CFEF0
S31508025430F869FFF764FF55E02D4B1B781A46FB689F
S3150802544093F8283003F00F039A4248D1FB68DB68C9
S315080254501846FFF7D8FD0346013B7B82FB682933D2
S315080254607A8A1146184608F03FFE214B1B7801330B
S31508025470DAB21F4B1A701E4B1B780F2B2FD91C4BF7
S3150802548000221A702BE01B4BD3F84432FA699A426F
S315080254900FD1FB6893F8283003F00F03DAB2154BE5
S315080254A083F86E22FB6893F82920124B83F86F2241
S315080254B017E0104BD3F8843AFA699A4211D1FB687D
S315080254C093F8283003F00F03DAB20A4B83F8AE2AB0
S315080254D0FB6893F82920074B83F8AF2A01E000BF3F
S315080254E000E000BF00BF2037BD4680BDCEC8002001
S315080254F0D0C8002000B6002080B500AF2AF020F8F8
S3150802550000BF80BD80B584B000AF78607B68FB6061
S31508025510FFF7F2FC0346002B0AD0FB681B68B3F5BB
S31508025520806F10D1FB6893F82830002B0BD10AE064
S31508025530FB681B68B3F5806F05D1FB6893F82830C2
S31508025540002B00D100BF00BF1037BD4680BD00004A
S3150802555080B500AF80220349034823F095FE00BFB9
S3150802556080BD00BF9CCB00208CCB002080B500AF4D
S31508025570054823F013FF0346002B01D0012300E060
S315080255800023184680BD00BF8CCB002080B582B0B0
S3150802559000AF78600B46FB704FF0FF31074823F0E7
S315080255A0BFF8FB781A467968054824F082F803485A
S315080255B023F0F8F800BF0837BD4680BD4CA5002089
S315080255C08CCB002080B584B000AF78600023FB73D3
S315080255D04FF0FF31084823F0A3F87968074824F00A
S315080255E079F80346FB73044823F0DCF8FB7B18467C
S315080255F01037BD4680BD00BF4CA500208CCB0020CD
S3150802560090B5A5B000AF0346FB71002387F88E302C
S31508025610002387F88F3012F091FD0346184613F0DF
S315080256206BF80346002B40F0E48212F087FD03462E
S31508025630184613F053FA0346012B40F04781B14B43
S315080256401B885A1C91B2AF4A1180092B40F23E813F
S3150802565012F074FD03460021184613F04CFAA94BC2
S3150802566000221A8012F06AFD0346184612F03AFF23
S3150802567003461946A44825F05EFB12F05FFD034671
S31508025680184613F059F9034619469F4825F06EFB4A
S3150802569002219D4825F085FB9B4825F040FB0346E1
S315080256A019469A4815F00EF99949974826F0F2F8DC
S315080256B0984815F007F9002387F88F300DE097F818
S315080256C08F30934A13445B781946934815F0FAF8D3
S315080256D097F88F30013387F88F308D4B1B7897F800
S315080256E08F209A42EBD38D4815F0ECF812F026FD7E
S315080256F00346184612F0DAFE854B1B781A46884985
S3150802570029F0F0FE12F01AFD03460021184613F09E
S315080257108FF9844815F0D6F88349844823F085F929
S31508025720814823F04FF904467F4823F057F9034688
S315080257301946204608F0C4FC12F000FD0346184636
S3150802574012F0B4FE03461946794815F0BBF812F072
S31508025750F5FC03460221184613F028F812F0EEFC6F
S315080257600346184612F0A2FE03461A4671497248C3
S315080257702BF068FE6C49714823F057F96A4823F002
S3150802578021F90446684823F029F9034619462046B2
S3150802579008F096FC12F0D2FC03460021184612F0D5
S315080257A09BFF674825F042FB0346052B1BD165483C
S315080257B015F088F824F00AF9554B1B781A46584909
S315080257C029F090FE5849604823F02FF9564823F0ED
S315080257D0F9F80446544823F001F9034619462046C7
S315080257E008F06EFC6BE0564825F020FB0346032BB7
S315080257F00BD0534825F01AFB0346042B05D0504814
S3150802580025F014FB0346022B1BD1504815F05AF813
S3150802581024F03AF93E4B1B781A46414929F062FEB2
S3150802582041494B4823F001F93F4823F0CBF8044697
S315080258303D4823F0D3F803461946204608F040FCB3
S315080258403DE03F4825F0F2FA0346062B1BD14148B4
S3150802585015F038F824F0DAF82D4B1B781A46304939
S3150802586029F040FE30493C4823F0DFF82E4823F061
S31508025870A9F804462C4823F0B1F8034619462046EF
S3150802588008F01EFC1BE0354815F01CF82C4825F0DC
S31508025890CDFA03461A46324927482BF0D3FD224948
S315080258A0254823F0C2F8204823F08CF804461E48FF
S315080258B023F094F803461946204608F001FC12F034
S315080258C03DFC03460021184612F0FCFDFFF74EFE8A
S315080258D00346002B40F08D8107F10C03802200213C
S315080258E018462BF043FE07F10C031846FFF76AFE2B
S315080258F0034687F88E301B4814F0E4FF002387F826
S315080259008F3040E01CCC00206CCC00208461050856
S3150802591028CC002098610508A8610508B061050829
S3150802592029CC0020B4610508D4C80020D061050836
S31508025930F461050814620508D8CA00204062050801
S3150802594020CC00204C6205086062050888620508BA
S315080259509C620508C0620508D4620508FC6205084F
S31508025960206305085063050897F88F3090333B4447
S3150802597013F8843C1946A14814F0A4FF97F88F300F
S31508025980013387F88F3097F88F2097F88E309A422E
S31508025990EAD39B4814F096FF07F10C0302339949A0
S315080259A0184625F0A6FF974825F040FA0346002B2D
S315080259B010D1944825F055FA0346002B0AD112F065
S315080259C0BDFB03460021184612F0F0FE8E4814F07D
S315080259D079FF0EE18B4825F0F3F9034619468B4801
S315080259E014F070FF874825F006FA034619468848D8
S315080259F014F068FF834825F019FA03461C468148C5
S31508025A0025F02FFA03461A462146824814F05AFF11
S31508025A107C4825F00BFA0346002B00F0E68079480D
S31508025A2025F01FFA0346002B00F0DF80754825F0A3
S31508025A30FDF90346072B06D10021724825F002FA22
S31508025A40754814F03FFF6F4825F00BFA0346072BFB
S31508025A5006D100216B4825F010FA704814F032FF7F
S31508025A60684825F0E3F9034619466D4814F02AFFFB
S31508025A70644825F0F6F9034619466A4814F022FFE7
S31508025A8012F05CFB04465F4825F0D0F90346194636
S31508025A90204612F024FF12F051FB0446594825F01D
S31508025AA0E0F903461946204612F036FF12F046FB85
S31508025AB00446544825F084F903461946204612F04E
S31508025AC001FD12F03BFB04464E4825F094F90346C5
S31508025AD01946204612F013FD4A4825F071F9034685
S31508025AE01A46514951482BF0ADFC51494F4822F00C
S31508025AF09CFF4F4822F066FF04464D4822F06EFF8F
S31508025B0003461946204608F0DBFA3E4825F073F9A3
S31508025B1003461A46474945482BF094FC44494348EC
S31508025B2022F083FF424822F04DFF0446404822F005
S31508025B3055FF03461946204608F0C2FA314825F0B1
S31508025B4075F903461A463C4938482BF07BFC384916
S31508025B50364822F06AFF364822F034FF04463448B3
S31508025B6022F03CFF03461946204608F0A9FA2548C2
S31508025B7025F077F903461A4630492C482BF062FC81
S31508025B802B492A4822F051FF294822F01BFF0446D6
S31508025B90274822F023FF03461946204608F090FAC2
S31508025BA00AF0EAFA0446174825F040F90346194668
S31508025BB020460AF0AEFB0AF0DFFA0446114825F041
S31508025BC050F90346194620460AF0DBFB0AF0D4FAD6
S31508025BD00346012118460AF0EFFB12F0AFFA034614
S31508025BE00121184612F078FD03E0154814F06AFE02
S31508025BF0FFE700BF9437BD4690BD00BF5C6305084A
S31508025C00B061050820CC0020646305088463050892
S31508025C10A0630508B8630508E0630508006405087B
S31508025C20206405084464050868640508D8CA002083
S31508025C30D4C800208C640508AC640508D864050835
S31508025C400465050880B500AF40220349034823F0DE
S31508025C501BFB0123184680BD4CCB00203CCB002001
S31508025C6080B500AF054823F099FB0346002B01D007
S31508025C70012300E00023184680BD00BF3CCB00206C
S31508025C8080B582B000AF78600B46FB704FF0FF31EB
S31508025C90084822F045FDFB781A467968064823F03B
S31508025CA008FD044822F07EFD012318460837BD4642
S31508025CB080BD00BF14A500203CCB002080B584B06F
S31508025CC000AF78600023FB734FF0FF31084822F0DB
S31508025CD027FD7968074823F0FDFC0346FB73044851
S31508025CE022F060FDFB7B18461037BD4680BD00BF1B
S31508025CF014A500203CCB0020F0B595B002AF0023D6
S31508025D0087F8473012F01AFA0346184612F0AEFA26
S31508025D100346002B15D028F017FD0346FF21184627
S31508025D2028F005FEC34B00221A70C34B00221A70D4
S31508025D30C24B00221A70C24B00221A70C14B0022B3
S31508025D401A70FFF78DFF0346002B42F02981BE48E1
S31508025D5014F0B8FD3B1D4022002118462BF006FC24
S31508025D603B1D1846FFF7AAFF034687F847303B79DB
S31508025D70012B42F0108197F84730002B02F00B8175
S31508025D807B79202B4ADC002B42F3F880013B1F2B40
S31508025D9002F2F48001A252F823F000BF275E02083D
S31508025DA0275E02087D7F02087D7F02087D7F020842
S31508025DB0F9770208FD7A0208617E02087D7F0208E9
S31508025DC07D7F02087D7F02087D7F02087D7F0208AB
S31508025DD07D7F02087D7F02087D7F02087D7F02089B
S31508025DE07D7F02087D7F02087D7F02087D7F02088B
S31508025DF07D7F02087D7F02087D7F02087D7F02087B
S31508025E007D7F02087D7F02087D7F02087D7F02086A
S31508025E107D7F02087D7F0208617F0208FF2B02F060
S31508025E208A8002F0ABB8834B1B78002B42F0AF8016
S31508025E307B79022B15D197F84730023BD9B23B1D25
S31508025E400233824A184625F050FB0AF095F90446B1
S31508025E507E4824F0F9FD0346194620460AF091FACF
S31508025E6016E00AF089F90346052118460AF0A4FA4B
S31508025E7097F84730023BD9B23B1D0233734A18469C
S31508025E8025F063FB12F05AF90346184612F0E8FAAF
S31508025E906E4824F0A3FD0346072B03D100216B4865
S31508025EA024F0A8FD12F04AF90446684824F096FD43
S31508025EB003461946204612F059FC12F03FF90446E9
S31508025EC0624824F0C1FD03461946204612F05EFCDC
S31508025ED05E4824F083FD0346002B01F0EB835B4802
S31508025EE024F07CFD0346072B01F2E483574824F08D
S31508025EF05AFD0346002B01F0DD83544824F053FD76
S31508025F000346042B01F2D683504824F04CFD03467F
S31508025F101A464F4B1A704D4824F060FD03461A463E
S31508025F204C4B1A704A4B1B7819464A4B1B781A4631
S31508025F30494814F0C7FC474B1B78012B40F0988060
S31508025F40434B1B78012B19D10AF016F90446072090
S31508025F500AF080FE0346194620460AF0DAF90720B7
S31508025F600AF078FE03461A463C4B1A703B4B1B78DE
S31508025F7019463B4814F0A6FC00F0F6BF344B1B78D2
S31508025F80022B19D10AF0F8F8044607200AF0ECFEAB
S31508025F900346194620460AF0BCF907200AF0E4FE31
S31508025FA003461A462D4B1A702C4B1B7819462D4858
S31508025FB014F088FC00F0D8BF254B1B78032B19D1A7
S31508025FC00AF0DAF8044607200AF02CFF03461946B7
S31508025FD020460AF09EF907200AF024FF03461A46CD
S31508025FE01E4B1A701D4B1B7819461F4814F06AFC83
S31508025FF000F0BABF164B1B78042B40F0B5870AF09F
S31508026000BBF8044607200AF06BFF034619462046EA
S315080260100AF07FF907200AF063FF03461A460F4B78
S315080260201A700E4B1B781946104814F04BFC00F0F8
S315080260309BBF00BFC5CC0020D3CC0020D1CC00200A
S31508026040D0CC0020D2CC002034650508B4CC002080
S31508026050CCCC0020CECC002060650508CDCC002033
S31508026060B8650508D8650508F865050818660508B7
S31508026070BB4B1B78022B78D1BA4B1B78012B19D153
S315080260800AF07AF8044602200AF0E4FD03461946A5
S3150802609020460AF03EF902200AF0DCFD03461A46BB
S315080260A0B14B1A70B04B1B781946B04814F00AFC6B
S315080260B000F05ABFAB4B1B78022B19D10AF05CF8D9
S315080260C0044602200AF050FE0346194620460AF004
S315080260D020F902200AF048FE03461A46A24B1A7015
S315080260E0A14B1B781946A24814F0ECFB00F03CBF02
S315080260F09C4B1B78032B19D10AF03EF80446022062
S315080261000AF090FE0346194620460AF002F90220D2
S315080261100AF088FE03461A46934B1A70924B1B786E
S315080261201946944814F0CEFB00F01EBF8D4B1B781F
S31508026130042B40F019870AF01FF8044602200AF0D9
S31508026140CFFE0346194620460AF0E3F802200AF073
S31508026150C7FE03461A46844B1A70834B1B781946A8
S31508026160854814F0AFFB00F0FFBE7D4B1B78032B6E
S3150802617078D17C4B1B78012B19D109F0FDFF044617
S3150802618003200AF067FD0346194620460AF0C1F8BD
S3150802619003200AF05FFD03461A46734B1A70724BC8
S315080261A01B781946714814F08DFB00F0DDBE6D4B65
S315080261B01B78022B19D109F0DFFF044603200AF0E7
S315080261C0D3FD0346194620460AF0A3F803200AF02F
S315080261D0CBFD03461A46644B1A70634B1B78194665
S315080261E0634814F06FFB00F0BFBE5E4B1B78032BAF
S315080261F019D109F0C1FF044603200AF013FE03462B
S31508026200194620460AF085F803200AF00BFE0346D3
S315080262101A46554B1A70544B1B781946554814F0B2
S3150802622051FB00F0A1BE4F4B1B78042B40F09C8615
S3150802623009F0A2FF044603200AF052FE0346194655
S3150802624020460AF066F803200AF04AFE03461A4672
S31508026250454B1A70444B1B781946474814F032FBD3
S3150802626000F082BE3E4B1B78042B40F087803D4BE4
S315080262701B78012B19D109F07FFF044609200AF081
S31508026280E9FC0346194620460AF043F809200AF0B3
S31508026290E1FC03461A46344B1A70334B1B781946EF
S315080262A0324814F00FFB00F05FBE2E4B1B78022B10
S315080262B019D109F061FF044609200AF055FD034683
S315080262C0194620460AF025F809200AF04DFD03462C
S315080262D01A46254B1A70244B1B781946244814F083
S315080262E0F1FA00F041BE1F4B1B78032B19D109F0B6
S315080262F043FF044609200AF095FD0346194620463F
S315080263000AF007F809200AF08DFD03461A46164BCD
S315080263101A70154B1B781946164814F0D3FA00F072
S3150802632023BE104B1B78042B40F01E8609F024FF6F
S31508026330044609200AF0D4FD03461946204609F008
S31508026340E8FF09200AF0CCFD03461A46064B1A70E6
S31508026350054B1B781946084814F0B4FA00F004BE37
S31508026360CECC0020CCCC0020CDCC0020B8650508C8
S31508026370D8650508F865050818660508BB4B1B7835
S31508026380052B78D1BA4B1B78012B19D109F0F4FEEB
S31508026390044608200AF05EFC03461946204609F020
S315080263A0B8FF08200AF056FC03461A46B14B1A7083
S315080263B0B04B1B781946B04814F084FA00F0D4BDE5
S315080263C0AB4B1B78022B19D109F0D6FE04460820DE
S315080263D00AF0CAFC03461946204609F09AFF082025
S315080263E00AF0C2FC03461A46A24B1A70A14B1B7846
S315080263F01946A24814F066FA00F0B6BD9C4B1B7803
S31508026400032B19D109F0B8FE044608200AF00AFD42
S3150802641003461946204609F07CFF08200AF002FDC9
S3150802642003461A46934B1A70924B1B7819469448A0
S3150802643014F048FA00F098BD8D4B1B78042B40F0F7
S31508026440938509F099FE044608200AF049FD034699
S315080264501946204609F05DFF08200AF041FD034669
S315080264601A46844B1A70834B1B781946854814F0D2
S3150802647029FA00F079BD7D4B1B78062B78D17C4B27
S315080264801B78012B19D109F077FE044604200AF07D
S31508026490E1FB03461946204609F03BFF04200AF0B1
S315080264A0D9FB03461A46734B1A70724B1B78194668
S315080264B0714814F007FA00F057BD6D4B1B78022B92
S315080264C019D109F059FE044604200AF04DFC034688
S315080264D01946204609F01DFF04200AF045FC03462A
S315080264E01A46644B1A70634B1B781946634814F0B4
S315080264F0E9F900F039BD5E4B1B78032B19D109F077
S315080265003BFE044604200AF08DFC03461946204643
S3150802651009F0FFFE04200AF085FC03461A46554B8D
S315080265201A70544B1B781946554814F0CBF900F0EB
S315080265301BBD4F4B1B78042B40F0168509F01CFE39
S31508026540044604200AF0CCFC03461946204609F004
S31508026550E0FE04200AF0C4FC03461A46454B1A70AC
S31508026560444B1B781946474814F0ACF900F0FCBCBA
S315080265703E4B1B78072B40F087803D4B1B78012B3F
S3150802658019D109F0F9FD044605200AF063FB034612
S315080265901946204609F0BDFE05200AF05BFB0346B4
S315080265A01A46344B1A70334B1B781946324814F084
S315080265B089F900F0D9BC2E4B1B78022B19D109F0A8
S315080265C0DBFD044605200AF0CFFB034619462046A2
S315080265D009F09FFE05200AF0C7FB03461A46254B1B
S315080265E01A70244B1B781946244814F06BF900F0EC
S315080265F0BBBC1F4B1B78032B19D109F0BDFD044602
S3150802660005200AF00FFC03461946204609F081FECA
S3150802661005200AF007FC03461A46164B1A70154B54
S315080266201B781946164814F04DF900F09DBC104B1C
S315080266301B78042B40F0988409F09EFD0446052039
S315080266400AF04EFC03461946204609F062FE05206A
S315080266500AF046FC03461A46064B1A70054B1B7887
S315080266601946084814F02EF900F07EBCCECC00205C
S31508026670CCCC0020CDCC0020B8650508D865050825
S31508026680F865050818660508B74B1B78082B77D1F5
S31508026690B64B1B78012B19D109F06EFD044606206C
S315080266A00AF0D8FA03461946204609F032FE0620B1
S315080266B00AF0D0FA03461A46AD4B1A70AC4B1B7851
S315080266C01946AC4814F0FEF800F04EBCA74B1B78EE
S315080266D0022B19D109F050FD044606200AF044FBA4
S315080266E003461946204609F014FE06200AF03CFB2A
S315080266F003461A469E4B1A709D4B1B7819469E48AE
S3150802670014F0E0F800F030BC984B1B78032B19D133
S3150802671009F032FD044606200AF084FB03461946B0
S31508026720204609F0F6FD06200AF07CFB03461A46C7
S315080267308F4B1A708E4B1B781946904814F0C2F884
S3150802674000F012BC894B1B78042B40F00D8409F02B
S3150802675013FD044606200AF0C3FB034619462046E3
S3150802676009F0D7FD06200AF0BBFB03461A46804B02
S315080267701A707F4B1B781946814814F0A3F8F3E385
S31508026780794B1B78092B74D1784B1B78012B18D1BE
S3150802679009F0F2FC04460A200AF05CFA0346194696
S315080267A0204609F0B6FD0A200AF054FA03461A46AC
S315080267B06F4B1A706E4B1B7819466E4814F082F8A6
S315080267C0D2E36A4B1B78022B18D109F0D5FC044692
S315080267D00A200AF0C9FA03461946204609F099FD25
S315080267E00A200AF0C1FA03461A46614B1A70604B30
S315080267F01B781946604814F065F8B5E35B4B1B78BD
S31508026800032B18D109F0B8FC04460A200AF00AFB41
S3150802681003461946204609F07CFD0A200AF002FBC7
S3150802682003461A46524B1A70514B1B78194653485F
S3150802683014F048F898E34D4B1B78042B40F09483E8
S3150802684009F09AFC04460A200AF04AFB034619464E
S31508026850204609F05EFD0A200AF042FB03461A4664
S31508026860434B1A70424B1B781946454814F02AF8CE
S315080268707AE33D4B1B780A2B40F084803B4B1B780E
S31508026880012B18D109F078FC04460B200AF0E2F92C
S3150802689003461946204609F03CFD0B200AF0DAF9B0
S315080268A003461A46324B1A70314B1B781946314841
S315080268B014F008F858E32D4B1B78022B18D109F06F
S315080268C05BFC04460B200AF04FFA0346194620469B
S315080268D009F01FFD0B200AF047FA03461A46244B15
S315080268E01A70234B1B781946234813F0EBFF3BE338
S315080268F01E4B1B78032B18D109F03EFC04460B20CD
S315080269000AF090FA03461946204609F002FD0B20C2
S315080269100AF088FA03461A46154B1A70144B1B7866
S315080269201946164813F0CEFF1EE3104B1B78042BAC
S3150802693040F01A8309F020FC04460B200AF0D0FA2C
S3150802694003461946204609F0E4FC0B200AF0C8FA69
S3150802695003461A46064B1A70054B1B781946084811
S3150802696013F0B0FF00E300BFCECC0020CCCC002051
S31508026970CDCC0020B8650508D8650508F865050870
S3150802698018660508B54B1B780B2B74D1B44B1B78CC
S31508026990012B18D109F0F0FB04460C200AF05AF92B
S315080269A003461946204609F0B4FC0C200AF052F9AF
S315080269B003461A46AB4B1A70AA4B1B781946AA48C5
S315080269C013F080FFD0E2A64B1B78022B18D109F0F0
S315080269D0D3FB04460C200AF0C7F90346194620469B
S315080269E009F097FC0C200AF0BFF903461A469D4B9C
S315080269F01A709C4B1B7819469C4813F063FFB3E246
S31508026A00974B1B78032B18D109F0B6FB04460C20CA
S31508026A100AF008FA03461946204609F07AFC0C20C1
S31508026A200AF000FA03461A468E4B1A708D4B1B78EB
S31508026A3019468F4813F046FF96E2894B1B78042BBA
S31508026A4040F0928209F098FB04460C200AF048FAB4
S31508026A5003461946204609F05CFC0C200AF040FA67
S31508026A6003461A467F4B1A707E4B1B781946814895
S31508026A7013F028FF78E2794B1B780C2B74D1784BEC
S31508026A801B78012B18D109F077FB04460D200AF072
S31508026A90E1F803461946204609F03BFC0D200AF0A8
S31508026AA0D9F803461A466F4B1A706E4B1B7819466D
S31508026AB06D4813F007FF57E2694B1B78022B18D172
S31508026AC009F05AFB04460D200AF04EF90346194608
S31508026AD0204609F01EFC0D200AF046F903461A461E
S31508026AE0604B1A705F4B1B781946604813F0EAFE32
S31508026AF03AE25B4B1B78032B18D109F03DFB04469F
S31508026B000D200AF08FF903461946204609F001FCC2
S31508026B100D200AF087F903461A46524B1A70514B52
S31508026B201B781946524813F0CDFE1DE24C4B1B78D2
S31508026B30042B40F0198209F01FFB04460D200AF0C7
S31508026B40CFF903461946204609F0E3FB0D200AF061
S31508026B50C7F903461A46434B1A70424B1B78194625
S31508026B60444813F0AFFEFFE13C4B1B780D2B40F077
S31508026B7083803B4B1B78012B18D109F0FDFA04469A
S31508026B800E200AF067F803461946204609F0C1FBAB
S31508026B900E200AF05FF803461A46324B1A70314B3A
S31508026BA01B781946304813F08DFEDDE12C4B1B7815
S31508026BB0022B18D109F0E0FA04460E200AF0D4F89E
S31508026BC003461946204609F0A4FB0E200AF0CCF823
S31508026BD003461A46234B1A70224B1B78194623483A
S31508026BE013F070FEC0E11E4B1B78032B18D109F077
S31508026BF0C3FA04460E200AF015F90346194620463A
S31508026C0009F087FB0E200AF00DF903461A46154BC2
S31508026C101A70144B1B781946154813F053FEA3E154
S31508026C200F4B1B78042B40F09F8109F0A5FA044606
S31508026C300E200AF055F903461946204609F069FB63
S31508026C400E200AF04DF903461A46064B1A70054BF2
S31508026C501B781946074813F035FE85E1CECC00208D
S31508026C60CCCC0020CDCC0020B8650508D86505082F
S31508026C70F865050818660508A64B1B780E2B74D10D
S31508026C80A54B1B78012B18D109F076FA04460F207A
S31508026C9009F0E0FF03461946204609F03AFB0F20A1
S31508026CA009F0D8FF03461A469C4B1A709B4B1B7871
S31508026CB019469B4813F006FE56E1974B1B78022BA2
S31508026CC018D109F059FA04460F200AF04DF803467E
S31508026CD01946204609F01DFB0F200AF045F803461F
S31508026CE01A468E4B1A708D4B1B7819468D4813F02F
S31508026CF0E9FD39E1884B1B78032B18D109F03CFAD8
S31508026D0004460F200AF08EF803461946204609F073
S31508026D1000FB0F200AF086F803461A467F4B1A70C4
S31508026D207E4B1B781946804813F0CCFD1CE17A4B42
S31508026D301B78042B40F0188109F01EFA04460F202E
S31508026D400AF0CEF803461946204609F0E2FA0F2061
S31508026D500AF0C6F803461A46704B1A706F4B1B7830
S31508026D601946724813F0AEFDFEE06A4B1B780F2BEC
S31508026D7074D1694B1B78012B18D109F0FDF9044629
S31508026D80102009F067FF03461946204609F0C1FAA2
S31508026D90102009F05FFF03461A46604B1A705F4BD4
S31508026DA01B7819465E4813F08DFDDDE05A4B1B78B9
S31508026DB0022B18D109F0E0F90446102009F0D4FF95
S31508026DC003461946204609F0A4FA102009F0CCFF1A
S31508026DD003461A46514B1A70504B1B7819465148AE
S31508026DE013F070FDC0E04C4B1B78032B18D109F049
S31508026DF0C3F9044610200AF015F803461946204638
S31508026E0009F087FA10200AF00DF803461A46434B92
S31508026E101A70424B1B781946434813F053FDA3E0F8
S31508026E203D4B1B78042B40F09F8009F0A5F90446D8
S31508026E3010200AF055F803461946204609F069FA61
S31508026E4010200AF04DF803461A46344B1A70334B93
S31508026E501B781946354813F035FD85E02D4B1B780E
S31508026E60102B40F081802C4B1B78012B18D109F08E
S31508026E7083F90446112009F0EDFE03461946204619
S31508026E8009F047FA112009F0E5FE03461A46234B94
S31508026E901A70224B1B781946214813F013FD63E03A
S31508026EA01D4B1B78022B18D109F066F904461120EE
S31508026EB009F05AFF03461946204609F02AFA112014
S31508026EC009F052FF03461A46144B1A70134B1B78E5
S31508026ED01946144813F0F6FC46E00F4B1B78032BB1
S31508026EE026D109F049F90446112009F09BFF034609
S31508026EF01946204609F00DFA112009F093FF0346B8
S31508026F001A46064B1A70054B1B781946064813F0A3
S31508026F10D9FC29E0CECC0020CCCC0020CDCC002058
S31508026F20B8650508D8650508F865050818660508E8
S31508026F30AC4B1B78042B17D109F01EF90446112015
S31508026F4009F0CEFF03461946204609F0E2F9112058
S31508026F5009F0C6FF03461A46A34B1A70A24B1B78C2
S31508026F601946A24813F0AEFCA14823F052FD034687
S31508026F70002B00F08D839E4823F04BFD0346102B11
S31508026F8000F286839A4823F044FD0346013B0F2B01
S31508026F9000F2728301A252F823F000BFDD6F0208E5
S31508026FA045700208AD700208157102087D71020863
S31508026FB0F971020861720208C9720208317302087D
S31508026FC0997302080174020869740208D9740208DE
S31508026FD041750208A975020811760208814B1B78C9
S31508026FE0012B07D1072009F035FE03461A46814BC5
S31508026FF01A7045E37B4B1B78022B07D1072009F051
S31508027000B3FE03461A467B4B1A7039E3754B1B7857
S31508027010032B07D1072009F005FF03461A46754BCD
S315080270201A702DE36F4B1B78042B07D1072009F042
S3150802703057FF03461A466F4B1A7021E36D4BFF2220
S315080270401A701DE3674B1B78012B07D1022009F042
S3150802705001FE03461A46674B1A7011E3614B1B7809
S31508027060022B07D1022009F07FFE03461A46614B1E
S315080270701A7005E35B4B1B78032B07D1022009F034
S31508027080D1FE03461A465B4B1A70F9E2554B1B783A
S31508027090042B07D1022009F023FF03461A46554B53
S315080270A01A70EDE2534BFF221A70E9E24D4B1B7838
S315080270B0012B07D1032009F0CDFD03461A464D4B95
S315080270C01A70DDE2474B1B78022B07D1032009F021
S315080270D04BFE03461A46474B1A70D1E2414B1B78C0
S315080270E0032B07D1032009F09DFE03461A46414B9E
S315080270F01A70C5E23B4B1B78042B07D1032009F013
S31508027100EFFE03461A463B4B1A70B9E2394BFF2289
S315080271101A70B5E2334B1B78012B07D1092009F007
S3150802712099FD03461A46334B1A70A9E22D4B1B7872
S31508027130022B07D1092009F017FE03461A462D4BE2
S315080271401A709DE2274B1B78032B07D1092009F0F9
S3150802715069FE03461A46274B1A7091E2214B1B78A1
S31508027160042B07D1092009F0BBFE03461A46214B18
S315080271701A7085E21F4BFF221A7081E2194B1B789F
S31508027180012B07D1082009F065FD03461A46194B5B
S315080271901A7075E2134B1B78022B07D1082009F0E7
S315080271A0E3FD03461A46134B1A7069E20D4B1B7828
S315080271B0032B07D1082009F035FE03461A460D4B64
S315080271C01A705DE2074B1B78042B07D1082009F0D9
S315080271D087FE03461A46074B1A7051E2054BFF22F1
S315080271E01A704DE2CCCC0020CDCC002018660508DA
S315080271F0B4CC0020CFCC0020A74B1B78012B07D19B
S31508027200042009F027FD03461A46A44B1A7037E2F2
S31508027210A14B1B78022B07D1042009F0A5FD0346D2
S315080272201A469E4B1A702BE29B4B1B78032B07D1EF
S31508027230042009F0F7FD03461A46984B1A701FE216
S31508027240954B1B78042B07D1042009F049FE034607
S315080272501A46924B1A7013E2904BFF221A700FE2EB
S315080272608D4B1B78012B07D1052009F0F3FC034649
S315080272701A468A4B1A7003E2874B1B78022B07D1F0
S31508027280052009F071FD03461A46844B1A70F7E188
S31508027290814B1B78032B07D1052009F0C3FD034652
S315080272A01A467E4B1A70EBE17B4B1B78042B07D1EF
S315080272B0052009F015FE03461A46784B1A70DFE1D7
S315080272C0764BFF221A70DBE1734B1B78012B07D131
S315080272D0062009F0BFFC03461A46704B1A70CFE126
S315080272E06D4B1B78022B07D1062009F03DFD03469C
S315080272F01A466A4B1A70C3E1674B1B78032B07D1F0
S31508027300062009F08FFD03461A46644B1A70B7E148
S31508027310614B1B78042B07D1062009F0E1FD0346D1
S315080273201A465E4B1A70ABE15C4BFF221A70A7E154
S31508027330594B1B78012B07D10A2009F08BFC03460F
S315080273401A46564B1A709BE1534B1B78022B07D1F0
S315080273500A2009F009FD03461A46504B1A708FE1B6
S315080273604D4B1B78032B07D10A2009F05BFD034618
S315080273701A464A4B1A7083E1474B1B78042B07D1EE
S315080273800A2009F0ADFD03461A46444B1A7077E106
S31508027390424BFF221A7073E13F4B1B78012B07D130
S315080273A00B2009F057FC03461A463C4B1A7067E154
S315080273B0394B1B78022B07D10B2009F0D5FC034663
S315080273C01A46364B1A705BE1334B1B78032B07D1EF
S315080273D00B2009F027FD03461A46304B1A704FE177
S315080273E02D4B1B78042B07D10B2009F079FD034698
S315080273F01A462A4B1A7043E1284BFF221A703FE1BC
S31508027400254B1B78012B07D10C2009F023FC0346D8
S315080274101A46224B1A7033E11F4B1B78022B07D1EF
S315080274200C2009F0A1FC03461A461C4B1A7027E1E8
S31508027430194B1B78032B07D10C2009F0F3FC0346E2
S315080274401A46164B1A701BE1134B1B78042B07D1ED
S315080274500C2009F045FD03461A46104B1A700FE137
S315080274600E4BFF221A700BE10B4B1B78012B07D12F
S315080274700D2009F0EFFB03461A46084B1A70FFE087
S31508027480054B1B78022B0BD10D2009F06DFC034628
S315080274901A46024B1A70F3E0CCCC0020CFCC00205F
S315080274A0AD4B1B78032B07D10D2009F0BBFC034615
S315080274B01A46AA4B1A70E3E0A74B1B78042B07D18E
S315080274C00D2009F00DFD03461A46A44B1A70D7E0A3
S315080274D0A24BFF221A70D3E09F4B1B78012B07D1D0
S315080274E00E2009F0B7FB03461A469C4B1A70C7E0F2
S315080274F0994B1B78022B07D10E2009F035FC03465F
S315080275001A46964B1A70BBE0934B1B78032B07D18E
S315080275100E2009F087FC03461A46904B1A70AFE014
S315080275208D4B1B78042B07D10E2009F0D9FC034694
S315080275301A468A4B1A70A3E0884BFF221A709FE0FC
S31508027540854B1B78012B07D10F2009F083FB0346D5
S315080275501A46824B1A7093E07F4B1B78022B07D18F
S315080275600F2009F001FC03461A467C4B1A7087E085
S31508027570794B1B78032B07D10F2009F053FC0346DE
S315080275801A46764B1A707BE0734B1B78042B07D18D
S315080275900F2009F0A5FC03461A46704B1A706FE0D5
S315080275A06E4BFF221A706BE06B4B1B78012B07D1CF
S315080275B0102009F04FFB03461A46684B1A705FE023
S315080275C0654B1B78022B07D1102009F0CDFB034629
S315080275D01A46624B1A7053E05F4B1B78032B07D18E
S315080275E0102009F01FFC03461A465C4B1A7047E046
S315080275F0594B1B78042B07D1102009F071FC03465E
S315080276001A46564B1A703BE0544BFF221A7037E063
S31508027610514B1B78012B07D1112009F01BFB03469E
S315080276201A464E4B1A702BE04B4B1B78022B07D18E
S31508027630112009F099FB03461A46484B1A701FE0B7
S31508027640454B1B78032B07D1112009F0EBFB0346A8
S315080276501A46424B1A7013E03F4B1B78042B07D18C
S31508027660112009F03DFC03461A463C4B1A7007E006
S315080276703A4BFF221A7003E0384BFF221A7000BFFA
S3150802768008F07AFD0346FF21184608F05FFE06E079
S3150802769008F072FD0346FF21184608F057FE3048E7
S315080276A013F010F92F4B00221A602F4B01221A7081
S315080276B000F06DBC2D4823F091F90346FE2B40F0ED
S315080276C08C802A4823F06FF903461A46224B1A7011
S315080276D0264823F083F903461A46254B1A701E4B91
S315080276E01B781946224B1B781A46224813F0EAF8E9
S315080276F008F042FD0346FE21184608F00AFE08F085
S315080277003BFD0346FF21184608F020FE124B1B7864
S31508027710012B0ED108F030FD0346184608F0D2FDBB
S315080277200346184609F042FA03461A46124B1A70DD
S3150802773049E0094B1B78022B20D108F01DFD0346B0
S31508027740184608F0BFFD0346184609F0D7FA03465D
S315080277501A46094B1A7036E0CCCC0020CFCC002052
S3150802776038660508C8CC0020C5CC0020B4CC002059
S31508027770CECC002060650508CDCC0020D44B1B7802
S31508027780032B0ED108F0F8FC0346184608F09AFDBA
S315080277900346184609F010FB03461A46CD4B1A70E3
S315080277A011E0CB4B1B78042B0DD108F0E5FC034600
S315080277B0184608F087FD0346184609F05BFB0346A0
S315080277C01A46C44B1A70C34B1B78042BC24B0022B1
S315080277D01A60C24B01221A70D9E3C14823F0FEF897
S315080277E003461C46BE4823F0DEF803461A462146DF
S315080277F0BC4813F067F8CAE310F0A0FC0346184623
S3150802780010F02EFE3B1D0233B749184623F017FF28
S31508027810B54823F069FA0346002B09D1B34813F099
S3150802782051F810F08BFC0346184610F0F3FCB1E34E
S31508027830AD4823F059FA0346022B58D1AC4813F047
S3150802784041F826F081FF0346184626F0BFFF034695
S315080278500021184623F018F826F076FF0346184644
S3150802786026F0B4FF03460021184623F028F826F02E
S315080278706BFF03460A21184627F0ABF826F064FF89
S3150802788003460B21184627F0A4F826F05DFF0346A7
S315080278900C21184627F09DF826F056FF03460D21BF
S315080278A0184627F096F826F04FFF03460E2118468B
S315080278B027F08FF826F048FF03460F21184627F0CF
S315080278C088F826F041FF03461021184627F081F86A
S315080278D026F03AFF03461121184627F07AF808F0EF
S315080278E04BFC03460021184609F051F952E37E483B
S315080278F023F0FAF90346032B40F0E0807D4812F0A4
S31508027900E1FF26F021FF0346184626F05FFF0346ED
S315080279100021184622F0E2FF26F016FF0346184613
S3150802792026F054FF03460021184622F0F2FF26F0FD
S315080279300BFF03464721184627F04BF826F004FFAB
S3150802794003464821184627F044F826F0FDFE03466A
S315080279504921184627F03DF826F0F6FE03464B2144
S31508027960184627F036F826F0EFFE03464C2118464D
S3150802797027F02FF826F0E8FE03464D21184627F091
S3150802798028F826F0E1FE03465021184627F021F88A
S3150802799026F0DAFE03465121184627F01AF826F091
S315080279A0D3FE03465221184627F013F826F0CCFEDA
S315080279B003465321184627F00CF826F0C5FE03465F
S315080279C05621184627F005F826F0BEFE034657212B
S315080279D0184626F0FEFF26F0B7FE0346582118463B
S315080279E026F0F7FF26F0B0FE03465B21184626F07E
S315080279F0F0FF26F0A9FE03465C21184626F0E9FFA9
S31508027A0026F0A2FE03465D21184626F0E2FF26F07E
S31508027A109BFE03465E21184626F0DBFF26F094FEFF
S31508027A2003466121184626F0D4FF26F08DFE03464A
S31508027A306221184626F0CDFF26F086FE034663210C
S31508027A40184626F0C6FF26F07FFE0346662118462C
S31508027A5026F0BFFF26F078FE03466721184626F071
S31508027A60B8FF26F071FE03466821184626F0B1FFD4
S31508027A7026F06AFE03466921184626F0AAFF26F072
S31508027A8063FE03466F21184626F0A3FF26F05CFE26
S31508027A9003467121184626F09CFF26F055FE03463A
S31508027AA07221184626F095FF26F04EFE03467321EC
S31508027AB0184626F08EFF13F00BF96BE20A4823F0FC
S31508027AC013F9034619460C4812F0FCFE62E200BF9F
S31508027AD0CCCC0020CDCC0020C8CC0020C5CC0020C0
S31508027AE0B4CC002074660508C4CC0020DC66050800
S31508027AF00C6705082C670508506705083B1D023305
S31508027B00D349184623F002FED14823F066F8034605
S31508027B101946D04812F0D6FECF4B00221A7010F042
S31508027B200DFB0346184610F05DFB03460021184676
S31508027B30F9F72DFC0346012B06D1C74B1B7843F0F8
S31508027B400103DAB2C44B1A7010F0F8FA0346184663
S31508027B5010F048FB034601211846F9F718FC0346BC
S31508027B60012B06D1BC4B1B7843F00203DAB2BA4B9F
S31508027B701A7010F0E3FA0346184610F033FB034670
S31508027B8002211846F9F703FC0346012B06D1B24B2C
S31508027B901B7843F00403DAB2AF4B1A7010F0CEFA30
S31508027BA00346184610F01EFB034603211846F9F74A
S31508027BB0EEFB0346012B06D1A74B1B7843F00803BD
S31508027BC0DAB2A54B1A7010F0B9FA0346184610F045
S31508027BD009FB034604211846F9F7D9FB0346012B8C
S31508027BE006D19D4B1B7843F01003DAB29A4B1A70F2
S31508027BF010F0A4FA0346184610F0F4FA034618469B
S31508027C00F9F790FB0446924822F0E7FF03469C42A6
S31508027C102DD18F4822F0FCFF03461A468E4B1B785D
S31508027C209A4224D110F08AFA0346184610F0DAFA74
S31508027C3003461846F9F7DFFB03461C46844823F039
S31508027C4002F803469C4212D110F078FA0346184607
S31508027C5010F0C8FA03461846F9F7E8FB03461C462D
S31508027C607B4823F00BF803469C4200F0DC8010F0B8
S31508027C7065FA0346184610F0B5FA0446744822F027
S31508027C80ACFF034619462046F9F758FB704822F01E
S31508027C90BFFF034603F00103002B0CD010F04EFA87
S31508027CA00346184610F09EFA03460122002118469A
S31508027CB0F9F782FB0BE010F041FA0346184610F07A
S31508027CC091FA0346002200211846F9F775FB604827
S31508027CD022F09EFF034603F00203002B0CD010F09D
S31508027CE02DFA0346184610F07DFA034601220121B1
S31508027CF01846F9F761FB0BE010F020FA034618461E
S31508027D0010F070FA0346002201211846F9F754FBCF
S31508027D104F4822F07DFF034603F00403002B0CD0E4
S31508027D2010F00CFA0346184610F05CFA03460122D4
S31508027D3002211846F9F740FB0BE010F0FFF903465B
S31508027D40184610F04FFA0346002202211846F9F7A0
S31508027D5033FB3F4822F05CFF034603F00803002B7F
S31508027D600CD010F0EBF90346184610F03BFA03461E
S31508027D70012203211846F9F71FFB0BE010F0DEF982
S31508027D800346184610F02EFA034600220321184627
S31508027D90F9F712FB2E4822F03BFF034603F01003C5
S31508027DA0002B0CD010F0CAF90346184610F01AFA3E
S31508027DB00346012204211846F9F7FEFA0BE010F0F1
S31508027DC0BDF90346184610F00DFA034600220421AF
S31508027DD01846F9F7F1FA10F0B1F90346184610F009
S31508027DE001FA04461A4822F02EFF0346194620468F
S31508027DF0F9F70DFB10F0A2F90346184610F0F2F94E
S31508027E000446134822F03AFF034619462046F9F774
S31508027E1019FB10F093F90346184610F0E3F90346E6
S31508027E201846F9F749FA01210C4823F0CEFC21F04D
S31508027E3046FE0446094823F0EDFA0546074823F0AC
S31508027E40F5FA03461A462946204627F02DFCA1E0F4
S31508027E50B8CC002078670508D4CC002070CC002066
S31508027E603B1D0233C249184623F0CCFCC04822F017
S31508027E7020FF03461946BF4812F024FDBC4822F0EB
S31508027E8018FF0346002B45D126F05EFC0346002167
S31508027E90184626F0F3FDB84812F014FD26F054FCF5
S31508027EA003460221184626F0B8FCB44812F00AFD29
S31508027EB008F0FCF80346184608F01DF90346012B9C
S31508027EC001D008F047F908F057F90346184608F0B2
S31508027ED052FE0346012B09D0A94812F0F3FC08F01A
S31508027EE04BF903460021184608F051FE12F0BEFE71
S31508027EF00346184612F0D0FE0346022B04D0A148C8
S31508027F0012F0E0FC12F0E4FE9F4812F0DBFC03F0EC
S31508027F10CBFC3EE0964822F0CCFE0346012B38D134
S31508027F2026F012FC03463721184626F052FD9748DA
S31508027F3012F0C8FC2DE0964823F0D2FB21F0BFFDD3
S31508027F40934B1B781A46934927F0CCFA924812F0BB
S31508027F50B9FC10F0F3F80346184610F05BF919E07D
S31508027F60BB7919468D4812F0ADFC08F005F90246B0
S31508027F70BB791946104608F021F90BE07B791946B8
S31508027F8097F847301A46864812F09CFC02E000BF72
S31508027F9006E000BF04E03B791946824812F092FCDB
S31508027FA008F0EAF80346184608F0FCF80346012BDF
S31508027FB045D110F0C3F80346184610F00FFD0346E4
S31508027FC0012B11D110F0BAF803460021184610F019
S31508027FD012FD754812F076FC08F0CEF80346002129
S31508027FE0184608F0E9F922E008F0C6F8044608F04F
S31508027FF0C3F80346184608F0B8F903461946204658
S3150802800008F087F908F0B8F803460221184608F07E
S31508028010D3F9664812F056FC08F0AEF8034618463D
S3150802802008F0A3F903461946614812F04BFC08F01A
S31508028030A3F803460021184608F0C0F819E008F02C
S315080280409BF80346184608F0ADF80346032B10D1F1
S3150802805008F092F803460021184608F0ADF955488B
S3150802806012F030FC08F088F803460021184608F09A
S31508028070A5F8514B1B78002B02D0012B04D0CAE27B
S315080280804E4B00221A60C6E208F076F803461846F6
S3150802809008F071FD03461946494812F013FC08F028
S315080280A06BF80346184608F00DF903461946454883
S315080280B012F008FC444B1B781946444812F002FC9D
S315080280C008F05AF80346184608F055FD0346012BF0
S315080280D00BD108F051F80346184608F0F3F80346A0
S315080280E01A463B4B1B789A420ED008F045F80346CF
S315080280F0184608F040FD0346012B40F00682324B33
S315080281001B78FE2B40F001822F4B1B78012B15D1D1
S31508028110304B1B78012B0AD126F016FB03460B219E
S31508028120184626F07AFB2C4812F0CCFBE3E1294BE1
S315080281301B781946294812F0C5FBDCE1224B1B784D
S31508028140022B4FD1234B1B78012B0AD126F0FCFABE
S3150802815003460C21184626F060FB214812F0B2FBB2
S31508028160C9E11C4B1B7819461C4812F0ABFBC2E14D
S31508028170C0CC0020B0670508F46705080C68050836
S315080281802068050830680508446805085C6805081B
S3150802819028CC002029CC00207868050894680508B0
S315080281A0AC680508DC680508106905083069050821
S315080281B04C6905085C690508C5CC0020C8CC0020B6
S315080281C07869050888690508CECC0020A4690508DF
S315080281D0CDCC0020CCCC0020C4690508006A05086D
S315080281E0146A05089B4B1B78032B15D19A4B1B78EF
S315080281F0012B0AD126F0A8FA03460D21184626F0C5
S315080282000CFB964812F05EFB75E1934B1B781946F8
S31508028210934812F057FB6EE18E4B1B78042B15D14F
S315080282208D4B1B78012B0AD126F08EFA03460E21B6
S31508028230184626F0F2FA8B4812F044FB5BE1864BAD
S315080282401B781946864812F03DFB54E1814B1B7890
S31508028250052B15D1804B1B78012B0AD126F074FA0F
S3150802826003460F21184626F0D8FA7F4812F02AFB51
S3150802827041E1794B1B781946794812F023FB3AE11A
S31508028280744B1B78062B15D1734B1B78012B0AD11D
S3150802829026F05AFA03461021184626F0BEFA734803
S315080282A012F010FB27E16C4B1B7819466C4812F04A
S315080282B009FB20E1674B1B78072B15D1664B1B7808
S315080282C0012B0AD126F040FA03461121184626F058
S315080282D0A4FA674812F0F6FA0DE15F4B1B781946C5
S315080282E05F4812F0EFFA06E15A4B1B78082B15D1B4
S315080282F0594B1B78012B0AD126F026FA034612217E
S31508028300184626F08AFA5B4812F0DCFAF3E0524B7A
S315080283101B781946524812F0D5FAECE04D4B1B78F9
S31508028320092B15D14C4B1B78012B0AD126F00CFAD6
S3150802833003461321184626F070FA4F4812F0C2FA7D
S31508028340D9E0454B1B781946454812F0BBFAD2E0EC
S31508028350404B1B780A2B15D13F4B1B78012B0AD1B0
S3150802836026F0F2F903461421184626F056FA43482F
S3150802837012F0A8FABFE0384B1B781946384812F0B3
S31508028380A1FAB8E0334B1B780B2B15D1324B1B786D
S31508028390012B0AD126F0D8F903461521184626F0EC
S315080283A03CFA374812F08EFAA5E02B4B1B78194691
S315080283B02B4812F087FA9EE0264B1B780C2B15D118
S315080283C0254B1B78012B0AD126F0BEF90346162146
S315080283D0184626F022FA2B4812F074FA8BE01E4B46
S315080283E01B7819461E4812F06DFA84E0194B1B7861
S315080283F00D2B15D1184B1B78012B0AD126F0A4F99F
S3150802840003461721184626F008FA1F4812F05AFAA8
S3150802841071E0114B1B781946114812F053FA6AE0BB
S315080284200C4B1B780E2B33D10B4B1B78012B0AD125
S3150802843026F08AF903461821184626F0EEF913485B
S3150802844012F040FA57E0044B1B781946044812F01A
S3150802845039FA50E0CECC0020CCCC0020506A050870
S31508028460006A05088C6A0508C86A0508046B0508C7
S31508028470406B05087C6B0508B86B0508F46B0508A4
S31508028480306C05086C6C0508A86C0508E46C0508D0
S31508028490634B1B780F2B15D1624B1B78012B0AD124
S315080284A026F052F903461921184626F0B6F95E480F
S315080284B012F008FA1FE05B4B1B7819465B4812F06C
S315080284C001FA18E0564B1B78102B14D1554B1B7822
S315080284D0012B0AD126F038F903461A21184626F046
S315080284E09CF9534812F0EEF905E04E4B1B781946F3
S315080284F04E4812F0E7F90FF021FE034618460FF030
S3150802850006FF4C4B00221A703FE007F035FE034681
S31508028510184608F030FB0346012B0CD107F02CFE57
S315080285200346184607F0E9FE0346FF2B03D100204F
S3150802853009F0B0FF29E007F01FFE0346184608F0C7
S315080285401AFB0346012B20D107F016FE03461846EE
S3150802855007F0B8FE03461C4607F00EFE0346184609
S3150802856007F0CBFE03469C420FD107F005FE0346F1
S31508028570FF21184607F0EAFE07F0FEFD02462E4BDB
S315080285801B781946104607F0C4FE2C4B1B680133AC
S315080285902A4A1360294B1B684AF6C772934239D98D
S315080285A0264B1C681E4B1B781D4607F0E5FD034645
S315080285B0184607F087FE03461E4607F0DDFD03460A
S315080285C0184607F09AFE0346009333462A46214682
S315080285D01B4812F077F907F0CFFD0346184608F054
S315080285E0CAFA0346032B12D009F0F2FC0346002B03
S315080285F00DD126F0A9F803460A21184626F097F95E
S315080286000FF09CFD03460A21184610F02EF9094B75
S3150802861000221A7000BF00BF4C37BD46F0BD00BF2E
S31508028620CECC0020CCCC0020206D0508006A0508B7
S315080286305C6D0508C5CC0020CDCC0020C8CC002036
S31508028640986D050880B500AF4FF4007203490448D7
S3150802865020F01AFE0123184680BD00BFD8CC0020A0
S31508028660D8CE002080B582B000AF0023FB71074840
S3150802867020F094FE0346FB71FB79002B01D00123FF
S3150802868000E0002318460837BD4680BDD8CE002034
S3150802869080B584B000AF78600B46FB700023FB60A0
S315080286A04FF47A710F4820F03BF80346002B0AD1A3
S315080286B0FB781A4679680C4820F0FBFFF8600948EF
S315080286C020F070F802E0094812F0FCF8FB68002B6B
S315080286D002D1074812F0F6F8012318461037BD46AC
S315080286E080BD00BFBCA50020D8CE0020C86D0508F5
S315080286F0046E050880B584B000AF78600023FB736A
S315080287004FF47A710B4820F00BF80346002B09D177
S315080287107968094820F0DEFF0346FB73054820F016
S3150802872041F802E0054812F0CDF8FB7B18461037EF
S31508028730BD4680BDBCA50020D8CE0020306E0508F7
S3150802874080B584B000AF78600B46FB700023FB60EF
S315080287500023FB6009E0FB78184612F0F1F90120C4
S315080287601FF09EF8FB680133FB60FA687B689A4241
S31508028770F1D300BF00BF1037BD4680BD80B584B0B7
S3150802878000AF0346FB710023FB73FFF76BFF03463B
S31508028790002B40F08D82CF4B00221A7080220021D6
S315080287A0CD4828F0E3FECC48FFF7A4FF03461A4655
S315080287B0C84B1A70C84B1B78722B00F37182602B58
S315080287C004DA212B30D0222B39D069E2603B122BF6
S315080287D000F2668201A252F823F000BF4F8802080F
S315080287E01189020883890208A18C0208A18C020851
S315080287F0A18C0208A18C0208A18C0208A18C02088D
S31508028800A18C0208A18C0208A18C0208A18C02087C
S31508028810A18C0208A18C0208A18C0208858A02088A
S315080288206F8B02080B8C0208AC480FF02BFCAC4984
S31508028830AC4820F03DFAAA4820F0A7F938E2AA483F
S315080288400FF020FCA949A74820F08DFA30E2A84883
S315080288500FF018FCA749A34805F0ABF8A54804F0A1
S3150802886022FF0346062B49D801A252F823F000BF7D
S315080288708D8802089D880208AD880208BD8802080C
S31508028880CD880208DD880208ED88020807F074FC24
S3150802889003460021184607F03CFD38E007F06CFC59
S315080288A003460421184607F034FD30E007F064FC5D
S315080288B003460321184607F02CFD28E007F05CFC66
S315080288C003460221184607F024FD20E007F054FC6F
S315080288D003460121184607F01CFD18E007F04CFC78
S315080288E003460521184607F014FD10E007F044FC7C
S315080288F003460621184607F00CFD08E07D4804F0F9
S31508028900D2FE034619467C480FF0BCFB00BFCFE1F6
S315080289107A480FF0B7FB7A49724805F0ADF87848FD
S3150802892004F0F7FE0346012B0CD10FF007FC0346B1
S315080289300121184610F05FF803227249724826F0A0
S31508028940B3FEB5E16E4804F0E4FE0346022B0FD1EE
S315080289500FF0F4FB03460121184610F04CF821F0FB
S315080289605FF8034603226949184626F09DFE9FE1F1
S31508028970634804F0CEFE0346194665480FF082FBAB
S3150802898096E164480FF07EFB6349564805F0D7F82E
S31508028990614804F0F4FE0346013B052B68D801A2A0
S315080289A052F823F0BD890208DB890208F989020810
S315080289B0178A0208358A0208538A02080FF0BEFB94
S315080289C00346012118460FF016FE00F0EDF903469C
S315080289D00121184600F04FFA53E00FF0AFFB0346A9
S315080289E0012118460FF007FE00F0DEF903460221C0
S315080289F0184600F040FA44E00FF0A0FB03460121B6
S31508028A0018460FF0F8FD00F0CFF903460321184681
S31508028A1000F031FA35E00FF091FB034601211846C2
S31508028A200FF0E9FD00F0C0F903460421184600F0EC
S31508028A3022FA26E00FF082FB0346012118460FF0C0
S31508028A40DAFD00F0B1F903460521184600F013FADB
S31508028A5017E00FF073FB0346012118460FF0CBFD12
S31508028A6000F0A2F903460621184600F004FA08E0C7
S31508028A70294804F084FE0346194628480FF002FBEB
S31508028A8000BF15E126480FF0FDFA2649154805F0FC
S31508028A90C1F8244804F0C4FE0346FB73FB7B642B2F
S31508028AA003D9642003F0AEF803E0FB7B184603F013
S31508028AB0A9F81C4804F099FE0346002B02D0FB7B5A
S31508028AC0002B33D103F078F903F0C0F9164B0022D4
S31508028AD01A70EDE068CF0020E8CE0020AC6E0508DB
S31508028AE06CCF0020E9CE0020C86E050870CF0020A2
S31508028AF0E86E050874CF0020086F05083C6F050864
S31508028B0078CF0020601600200200040068160020B4
S31508028B105C6F05088C6F05087CCF0020B06F0508CE
S31508028B20E86F050880CF00200AA40020624804F0F6
S31508028B305CFE0346012B09D1604B01221A7003F031
S31508028B4053F9FB7B184603F05DF8B0E05A4804F087
S31508028B504CFE0346022B40F0AA80584B01221A709B
S31508028B6003F0F8F8FB7B184603F04CF89FE05448EC
S31508028B700FF088FA5349544805F0BAF8514804F0F8
S31508028B8085FE0346042B36D801A252F823F000BF0D
S31508028B90A58B0208C78B0208D38B0208DF8B020853
S31508028BA0EB8B020803224949494826F07DFDFB79E9
S31508028BB019464FF47A70FFF7C3FD03224549444824
S31508028BC026F072FD20E003224249414826F06CFD58
S31508028BD01AE0032240493E4826F066FD14E00322C5
S31508028BE03A493B4826F060FD0EE003223B493848E5
S31508028BF026F05AFD08E0334804F048FE03461946B3
S31508028C0037480FF03FFA00BF52E036480FF03AFAFB
S31508028C1035492D4805F0CFF8334804F06DFE034672
S31508028C20022B24D0022B31DC002B02D0012B0FD0D1
S31508028C302CE000F0B9F803460321184600F0CAF8FA
S31508028C4000F0B2F803460321184600F0F9F826E0C8
S31508028C5000F0AAF803460321184600F0BBF800F014
S31508028C60A3F803460121184600F0EAF817E000F0D7
S31508028C709BF803460321184600F0ACF800F094F876
S31508028C8003460221184600F0DBF808E0164804F00D
S31508028C9033FE0346194615480FF0F4F900BF07E0FC
S31508028CA0134B1B78194613480FF0ECF900E000BF86
S31508028CB000BF1037BD4680BD80CF00200AA4002021
S31508028CC00870050884CF0020E9CE0020701600201F
S31508028CD0020004007816002080160020881600205C
S31508028CE0287005085C70050888CF00208070050882
S31508028CF0E8CE0020B870050880B500AF8022034987
S31508028D00034820F0C1FA00BF80BD00BF08D2002088
S31508028D10F8D1002080B500AF054820F03FFB034696
S31508028D20002B01D0012300E00023184680BD00BFB6
S31508028D30F8D1002080B582B000AF78600B46FB7090
S31508028D404FF0FF3107481FF0EBFCFB781A467968AB
S31508028D50054820F0AEFC03481FF024FD00BF083783
S31508028D60BD4680BD68A50020F8D1002080B584B034
S31508028D7000AF78600023FB734FF0FF3108481FF0FD
S31508028D80CFFC7968074820F0A5FC0346FB73044824
S31508028D901FF008FDFB7B18461037BD4680BD00BF95
S31508028DA068A50020F8D1002080B500AF074B1B78D4
S31508028DB0DBB2002B07D1054B01221A7005220021CE
S31508028DC0034828F0D3FB024B184680BD56D3002031
S31508028DD058D3002080B483B000AF78600B46FB708E
S31508028DE07B68FA785A7000BF0C37BD465DF8047B7B
S31508028DF0704780B483B000AF78607B685B781846AA
S31508028E000C37BD465DF8047B704780B483B000AF6B
S31508028E1078600B46FB707B68FA781A7100BF0C37CC
S31508028E20BD465DF8047B704780B483B000AF7860B6
S31508028E307B681B7918460C37BD465DF8047B70477C
S31508028E4080B483B000AF78600B46FB707B68FA7813
S31508028E509A7000BF0C37BD465DF8047B704780B434
S31508028E6083B000AF78607B689B7818460C37BD469E
S31508028E705DF8047B704780B483B000AF78600B4618
S31508028E80FB707B68FA78DA7000BF0C37BD465DF86E
S31508028E90047B704780B483B000AF78607B68DB7868
S31508028EA018460C37BD465DF8047B70472DE9F0413C
S31508028EB084B002AF0023FB710023BB7100237B71D0
S31508028EC000233B710421334813F068FD0346012B46
S31508028ED001D10123FB7108212E4813F05FFD0346D9
S31508028EE0012B01D10223BB7110212A4813F056FD2A
S31508028EF00346012B01D104237B71FA79BB7913430B
S31508028F00DAB27B7913433B714021224813F046FDBE
S31508028F100346012B35D110211E4813F03FFD0346A7
S31508028F20012B0CBF01230023DBB21D460821194879
S31508028F3013F034FD0346012B0CBF01230023DBB2D9
S31508028F401E460421134813F029FD0346012B0CBFC4
S31508028F5001230023DBB298463C7940210D4813F0E1
S31508028F601DFD0346012B0CBF01230023DBB201932F
S31508028F700094434632462946074811F0A3FC3B793A
S31508028F8003E0064811F09EFC002318460837BD4642
S31508028F90BDE8F08100100242D87005080071050884
S31508028FA080B500AF5B4B1B78022B00F09880022B32
S31508028FB000F3AC80002B02D0012B4ED0A6E0564B14
S31508028FC01B780133DAB2544B1A70534B1B78022BB7
S31508028FD02AD8514B1B781946504811F073FCFFF7F3
S31508028FE0E3FE034600211846FFF7F4FEFFF7DCFE10
S31508028FF0034600211846FFF723FF494811F062FC91
S31508029000484B1B686422DA63464B1B6800221A64C3
S315080290100C2144481AF08CF80821424819F028FF16
S315080290203C4B01221A7071E03F4811F04BFCFFF7E6
S31508029030BBFE034600211846FFF7CCFEFFF7B4FE37
S31508029040034600211846FFF7FBFE334B00221A702F
S31508029050364B00221A70FF2359E002F041FC034600
S315080290600321184603F0AAFD0346022B15D1304800
S3150802907011F028FC2B4B1B686322DA63294B1B6809
S3150802908063221A640C21274819F0F2FE08212548A2
S3150802909019F0EEFE1F4B02221A7002F021FC03465B
S315080290A00121184603F08AFD0346022B2DD12148D9
S315080290B011F008FC1B4B1B686322DA63194B1B6809
S315080290C063221A640C21174819F0D2FE08211548A2
S315080290D019F0CEFE0F4B00221A70FF2317E016482E
S315080290E011F0F0FBFFF760FE034603211846FFF76F
S315080290F071FEFFF759FE034602211846FFF7A0FE46
S31508029100044B00221A70012301E000BF002318460F
S3150802911080BD00BFDDD20020E0D20020187105080C
S3150802912040710508F8E700206C710508DAD20020BC
S3150802913098710508C4710508F47105082DE9F0430C
S3150802914085B004AFFFF730FE03461846FFF751FE17
S315080291500346082B40F098809C4B1B78032B61D062
S31508029160032B00F3A383012B02DC002B03DA9DE316
S31508029170022B45D09AE302F0B3FB0346184602F0E7
S31508029180CFFC0346012B16D10EF0D8FF034618462C
S315080291900FF095FA03461A468D4B1B68DA638C4B19
S315080291A01B6800221A640821894819F061FE0C21FD
S315080291B0874819F0BDFF02F093FB0346184602F0F2
S315080291C0AFFC0346022B40F066830EF0B7FF034658
S315080291D018460FF074FA03461A467D4B1B68DA6383
S315080291E07B4B1B6800221A640821794819F040FE55
S315080291F00C21774819F09CFF744B02221A704AE335
S31508029200744B1B8801339AB2724B1A80714B1B88B6
S31508029210952B40F24283704811F054FB6B4B0322A4
S315080292201A703AE302F05CFB0346184602F078FC31
S315080292300346012B40F03383684B1B780133DAB2BD
S31508029240664B1A70624B1B686422DA63604B1B68B2
S3150802925064221A6408215E4819F00AFE0C215C4849
S3150802926019F006FEFFF722FE034619465C4811F07E
S3150802927029FBFFF799FD034600211846FFF7AAFDC9
S31508029280524B00221A700AE3FFF78EFD0346184670
S31508029290FFF7AFFD0346012B40F0A4804B4B1B782A
S315080292A0032B61D0032B00F30183012B02DC002B75
S315080292B003DAFBE2022B45D0F8E202F011FB034681
S315080292C0184602F02DFC0346012B16D1404B1B68AB
S315080292D00022DA630EF032FF034618460FF0EFF962
S315080292E003461A463A4B1B681A640C21384819F089
S315080292F0BFFD0821364819F01BFF02F0F1FA0346B2
S31508029300184602F00DFC0346022B40F0CA82304B87
S315080293101B680022DA630EF011FF034618460FF0A7
S31508029320CEF903461A462A4B1B681A640C212848AA
S3150802933019F09EFD0821264819F0FAFE234B02224F
S315080293401A70AEE2234B1B8801339AB2214B1A805C
S31508029350204B1B88632B40F2A6821F4811F0B2FAF3
S315080293601A4B03221A709EE202F0BAFA034618460C
S3150802937002F0D6FB0346012B40F09782174B1B7867
S315080293800133DAB2154B1A70114B1B686422DA6381
S315080293900F4B1B6864221A6408210D4819F068FDF0
S315080293A00C210B4819F064FDFFF780FD03461946A8
S315080293B00B4811F087FAFFF7F7FC03460021184617
S315080293C0FFF708FD014B00221A706EE2F4D1002065
S315080293D060E70020D8D200201C720508DBD20020E4
S315080293E02C720508FFF7E0FC03461846FFF701FD55
S315080293F00346022B3ED102F073FA034601211846B0
S3150802940003F0DCFB03461E4602F06AFA0346022113
S31508029410184603F0D3FB0346984602F061FA034660
S315080294200321184603F0CAFB034699461021C7488A
S3150802943013F0B4FA0346012B14BF01230023DBB24F
S315080294401C4602F04DFA0346184603F0ABFF0346E4
S315080294501D4602F045FA0346184603F0CCFF0346BA
S315080294600293019500944B4642463146B84811F09C
S3150802947029FA1BE2FFF798FC03461846FFF7B9FCE0
S315080294800346032B40F01282FFF78EFC03460021A7
S315080294901846FFF79FFCFFF787FC03461846FFF7B7
S315080294A0DEFC03461946AB4811F00CFAFFF77CFCC2
S315080294B003461846FFF7D3FC0346022B58D102F09F
S315080294C00FFA03460221184603F078FB0346022BDD
S315080294D02AD1A14811F0F6F9FFF766FC03460021E6
S315080294E01846FFF7ADFC01219C4821F032FD9C4944
S315080294F09A4822F0BEFA20F07FFA994B1B781A4650
S31508029500984925F0EFFF984998481FF08EFA964831
S315080295101FF058FA044694481FF060FA03461946A3
S31508029520204604F0CDFDC1E1FFF73EFC03460021CB
S315080295301846FFF785FC8E4811F0C4F98A498D480A
S315080295401FF073FA88481FF03DFA044686481FF052
S3150802955045FA03461946204604F0B2FD864B012217
S315080295601A70864B02221A70854B00221A809DE1D8
S31508029570FFF71AFC03461846FFF771FC0346012B50
S315080295806AD102F0ADF903460121184603F016FB2B
S315080295900346022B2AD1FFF707FC03460021184689
S315080295A0FFF74EFC774811F08DF901216B4821F03F
S315080295B0D0FC6B49694822F05CFA20F01DFA684B28
S315080295C01B781A46674925F08DFF67496E481FF0D2
S315080295D02CFA65481FF0F6F9044663481FF0FEF9AF
S315080295E003461946204604F06BFD5FE102F078F95E
S315080295F003460321184603F0E1FA0346022B0AD072
S3150802960002F06EF903460121184603F0D7FA03461B
S31508029610022B40F04B81FFF7C7FB03460021184691
S31508029620FFF70EFC594811F04DF94F4958481FF0FB
S31508029630FCF94D481FF0C6F904464B481FF0CEF90F
S3150802964003461946204604F03BFD4B4B02221A708C
S315080296504A4B01221A7029E1FFF7A6FB0346184670
S31508029660FFF7FDFB0346032B40F0208102F038F991
S3150802967003460321184603F0A1FA0346022B2AD110
S31508029680FFF792FB034600211846FFF7D9FB41482C
S3150802969011F018F90121314821F05BFC30492F48B5
S315080296A022F0E7F920F0A8F92D4B1B781A462D4926
S315080296B025F018FF2C4938481FF0B7F92A481FF039
S315080296C081F9044628481FF089F9034619462046B7
S315080296D004F0F6FCEAE002F003F903460121184613
S315080296E003F06CFA0346022B60D1FFF75DFB0346D3
S315080296F000211846FFF7A4FB284811F0E3F81A4997
S3150802970027481FF092F918481FF05CF904461648D4
S315080297101FF064F903461946204604F0D1FC214B92
S315080297201B680022DA631F4B1B6864221A640C2129
S315080297301C4819F09DFB08211A4819F0F9FC1A4B26
S3150802974001221A700D4B03221A70AFE0001402426E
S3150802975038720508707205088472050888D20020D6
S315080297608CD200208DD200208CCF0020947205085E
S31508029770AC720508C4720508DCD20020DAD20020D1
S31508029780DED20020E4720508F47205080C73050897
S315080297902473050844730508547305086C73050891
S315080297A084730508F8E70020E1D2002002F098F851
S315080297B003460221184603F001FA0346022B30D16A
S315080297C0FFF7F2FA034600211846FFF739FB3A4833
S315080297D011F078F839493A481FF027F937481FF047
S315080297E0F1F8044635481FF0F9F8034619462046AB
S315080297F004F066FC334B1B6800221A64314B1B6863
S315080298006422DA6308212F4819F032FB0C212D480D
S3150802981019F08EFC2C4B02221A702C4B03221A705A
S3150802982044E0FFF7C1FA034603211846FFF7D2FAC6
S31508029830FFF7BAFA034603211846FFF701FB224B44
S315080298401B78022B13D1224811F03CF81D4B1B68DA
S315080298506422DA631B4B1B6800221A640821194822
S3150802986019F006FB0C21174819F062FC1EE019488C
S3150802987011F028F8134B1B680022DA63114B1B6898
S3150802988064221A640C210F4819F0F2FA08210D48CD
S3150802989019F04EFC0AE000BF08E000BF06E000BF70
S315080298A004E000BF02E000BF00E000BF00BF0437CB
S315080298B0BD46BDE8F08300BFA47305088CCF00201F
S315080298C0BC730508F8E70020E1D20020DAD20020AE
S315080298D0DC730508F473050890B583B000AF7860A9
S315080298E003F0F6FA03F0C8F903F05CFA03F086FB14
S315080298F0B74B1B78012B05D1B64B01221A7001F022
S3150802990099FD08E0B24B1B78022B04D1B14B022217
S315080299101A7001F01BFDB04B1B780F2B0FD1FFF706
S315080299203FFB03461A46AD4B1A70AC4B1B78012B0C
S3150802993005D1AB4810F0C6FFA74B00221A70A64BFA
S315080299401B78012B40F08580A64B1B8801339AB2FF
S31508029950A44B1A80A34B1B8842F20F7293424AD930
S31508029960FFF722FA03461846FFF75EFA0346012B6B
S315080299701CD103F0FBFBFFF717FA03460021184632
S31508029980FFF743FA984810F09DFF984998481FF048
S315080299904CF896481FF016F8044694481FF01EF82D
S315080299A003461946204604F08BFB1BE0914810F04B
S315080299B089FF03F0DBFB8D498F481FF036F88B4889
S315080299C01FF000F8044689481FF008F803461946AE
S315080299D0204604F075FB22F035FE01232422662177
S315080299E00FF042F97F4B00221A807B4B00221A7035
S315080299F0774B00221A7001F073FF034601211846BD
S31508029A0003F0DCF80346022B40F0F18264201DF0D5
S31508029A1047FF03F0ABFB704B00221A706C4B002217
S31508029A201A70764B00221A70754810F04BFF6F4970
S31508029A3074481EF0FAFF6D481EF0C4FF04466B48D0
S31508029A401EF0CCFF03461946204604F039FB0123D3
S31508029A50CEE2614B1B78022B40F0E680614B1B88F5
S31508029A6001339AB25F4B1A805E4B1B8842F20F7221
S31508029A70934251D9FFF798F903461846FFF7D4F9E6
S31508029A800346012B1CD103F071FBFFF78DF9034640
S31508029A9000211846FFF7B9F95B4810F013FF53493E
S31508029AA05A481EF0C2FF51481EF08CFF04464F4822
S31508029AB01EF094FF03461946204604F001FB22E0F5
S31508029AC0534810F0FFFE494952481EF0AEFF474878
S31508029AD01EF078FF044645481EF080FF03461946E5
S31508029AE0204604F0EDFA03F041FBFFF75DF9034661
S31508029AF003211846FFF76EF9FFF756F903460121C7
S31508029B001846FFF79DF9374B00221A80324B00227E
S31508029B101A702F4B00221A7001F0E2FE0346022148
S31508029B20184603F04BF80346022B40F06082284B96
S31508029B301B781A464FF4C871374810F0C3FE374BE4
S31508029B4000221A80354B1B8801339AB2334B1A808E
S31508029B50324B1B88B3F5C87F15D21D4B1B78012BD8
S31508029B6002D103F0F5FA05E0194B1B78022B01D155
S31508029B7003F0E0FA7B68DBB2184610F0E1FF012039
S31508029B801DF08EFEDEE700BF164B00221A8003F098
S31508029B90EDFA114B00221A70184B00221A700C4B60
S31508029BA000221A701E4810F08DFE10491D481EF03C
S31508029BB03CFF0E481EF006FF04460C481EF00EFF38
S31508029BC003461946204604F07BFA012310E200BF39
S31508029BD0DCD20020E1D20020DAD20020E3D2002033
S31508029BE00C740508DED20020407405088CCF0020CC
S31508029BF06474050890740508B4740508D4D2002064
S31508029C00DC740508F8740508187505083C75050816
S31508029C106875050894750508CC750508E4D2002010
S31508029C20F07505080C760508C14B1B78032B08D07E
S31508029C30BF4B1B78072B04D0BD4B1B78042B40F077
S31508029C400581BB4B1B78072B07D10EF077FA034623
S31508029C500122022118460EF06FFFB64B1B8801330C
S31508029C609AB2B44B1A80B34B1B8842F20F729342D4
S31508029C704AD9FFF799F803461846FFF7D5F8034677
S31508029C80012B1CD103F072FAFFF78EF80346002166
S31508029C901846FFF7BAF8A84810F014FEA749A848CC
S31508029CA01EF0C3FEA5481EF08DFE0446A3481EF00C
S31508029CB095FE03461946204604F002FA1BE003F015
S31508029CC055FAA04810F0FEFD9C499F481EF0ADFECD
S31508029CD09A481EF077FE044698481EF07FFE034611
S31508029CE01946204604F0ECF922F0ACFC01232522A1
S31508029CF066210EF0B9FF8F4B00221A808C4B002288
S31508029D001A70924B00221A7001F0EAFD03460321EB
S31508029D10184602F053FF0346022B36D18C4B00221B
S31508029D201A708C4B1B78012B07D164218A4810F0D4
S31508029D30C9FD64201DF0B4FD0AE0864B1B78022B90
S31508029D4006D16421844810F0BDFD64201DF0A8FDEB
S31508029D5003F00CFA764B00221A70804B01221A7015
S31508029D607F4810F0AFFD75497E481EF05EFE7348C7
S31508029D701EF028FE044671481EF030FE03461946B8
S31508029D80204604F09DF9022332E1694B1B78042B25
S31508029D9028D101F0A5FD03460221184602F00EFF5E
S31508029DA00346022B1ED165496F481EF03EFE6348E4
S31508029DB01EF008FE044661481EF010FE03461946C8
S31508029DC0204604F07DF903F0D1F9594B00221A70A6
S31508029DD022F038FC0123282266210EF045FF4FF0B7
S31508029DE0FF3305E101F07CFD03460121184602F026
S31508029DF0E5FE0346022B40F0FA8050495B481EF006
S31508029E0014FE4E481EF0DEFD04464C481EF0E6FDE2
S31508029E1003461946204604F053F903F0A7F9544BB2
S31508029E201B680022DA63524B1B6864221A640821F3
S31508029E304F4819F07DF90C214D4819F019F8454B90
S31508029E4001221A703A4B04221A70D0E0384B1B785A
S31508029E50092B40F0CC8001F043FD03460321184646
S31508029E6002F0ACFE0346022B14D001F039FD03467C
S31508029E700121184602F0A2FE0346022B0AD001F07F
S31508029E802FFD03460221184602F098FE0346022BCE
S31508029E9040F0988001F024FD03460321184602F09B
S31508029EA08DFE0346022B03D14FF4FA701DF0F8FC1F
S31508029EB003F05CF901F014FD03460321184602F08B
S31508029EC07DFE0346022B0ED12A4810F0FBFC184BE6
S31508029ED000221A700EF032F90346012202211846B0
S31508029EE00EF02AFE82E001F0FBFC03460121184629
S31508029EF002F064FE0346022B40D11F4810F0E2FC32
S31508029F001B4B1B680022DA63194B1B6864221A640E
S31508029F100821174819F00CF90C21154818F0A8FF62
S31508029F200C4B01221A70024B07221A705EE000BF20
S31508029F30DAD20020DED200202C7605088CCF00204B
S31508029F40507605087C76050898760508DCD2002046
S31508029F50D5D20020E1D20020BC760508E2D2002044
S31508029F60CC760508E87605080877050840770508D7
S31508029F70F8E70020787705089077050801F0B0FC25
S31508029F8003460221184602F019FE0346022B2DD17A
S31508029F90194810F097FC194B1B686422DA63174BB1
S31508029FA01B6800221A640C21144819F0C1F808210A
S31508029FB0124818F05DFF124B02221A70114B072243
S31508029FC01A7013E00D4B1B680022DA630B4B1B68F1
S31508029FD064221A640821094819F0AAF80C210748CC
S31508029FE018F046FF064B01221A7000E000BF002354
S31508029FF018460C37BD4690BDA8770508F8E7002035
S3150802A000E1D20020DAD2002090B5A3B000AF002337
S3150802A01087F88630002387F887300EF08FF80346D4
S3150802A02018460EF0F8FA0346002B09D00EF086F809
S3150802A030034618460EF0EFFA0346022B40F0DE807E
S3150802A040FEF768FE0346002B40F0D8803B1D8022AF
S3150802A0500021184627F08AFA3B1D1846FEF786FEA7
S3150802A060034687F886303A463B1D023311461846A0
S3150802A07021F0A6FC0EF062F80346012118460EF0FE
S3150802A08054F90346002B1ED05E4810F01BFC002331
S3150802A09087F887300EE097F8873088333B4413F801
S3150802A0A0843C1946584810F00DFC97F8873001335E
S3150802A0B087F8873097F8872097F886309A42EAD346
S3150802A0C0524810F0FFFB3B46184620F01BFF03469A
S3150802A0D0002B21D14E4810F0F5FB4E494E481EF092
S3150802A0E0A4FC4C481EF06EFC04464A481EF076FC58
S3150802A0F003461946204603F0E3FF0EF01FF803460F
S3150802A100002118460EF077FA0EF018F803460021D9
S3150802A11018460EF053FA71E03B46184620F0F2FE56
S3150802A1200346002B50D03B46184620F0EBFE03466A
S3150802A130062B49D8374939481EF077FC35481EF0B0
S3150802A14041FC044633481EF049FC0346194620469C
S3150802A15003F0B6FF3B46184620F0D4FE03461C46DB
S3150802A160FEF7A4FE03461A4621462D4810F0AAFB1E
S3150802A1700DF0E4FF04463B46184620F0A8FE0346C7
S3150802A180194620460EF0FDF9FEF70EFE04463B463A
S3150802A190184620F0B7FE034619462046FEF76BFE20
S3150802A1A00DF0CCFF04463B46184620F075FE0346E2
S3150802A1B0194620460EF002FA0DF0C0FF03460121A9
S3150802A1C018460EF018FA19E03B46184620F09AFE91
S3150802A1D003461A461349144827F034F90D4912481A
S3150802A1E01EF023FC0B481EF0EDFB044609481EF040
S3150802A1F0F5FB03461946204603F062FF00BF8C377B
S3150802A200BD4690BDC0770508CC770508D477050802
S3150802A210D87705088CCF0020F87705081478050842
S3150802A220307805085C78050890D1002080B500AF23
S3150802A2302A4B1B7819462A4810F044FB274B1B78F1
S3150802A240023B062B46D801A252F823F08DA2020839
S3150802A250D5A20208B1A20208D5A202088DA2020856
S3150802A260D5A2020869A202081E4810F02BFBFEF7C7
S3150802A2709BFD034603211846FEF7ACFDFEF794FD47
S3150802A280034602211846FEF7DBFD24E0164810F0C5
S3150802A29019FBFEF789FD034603211846FEF79AFDC8
S3150802A2A0FEF782FD034603211846FEF7C9FD12E0B2
S3150802A2B00E4810F007FBFEF777FD03460321184602
S3150802A2C0FEF788FDFEF770FD034601211846FEF7E4
S3150802A2D0B7FD00E000BF00BF80BD00BF30D300203D
S3150802A2E084780508A0780508C4780508E87805087A
S3150802A2F090B583B000AF7860AA4B1B78002B4ED17D
S3150802A30001F00CF90346A84A1360A74B1B68012BF8
S3150802A31023D1A64810F0D6FAA24B01221A7000F0F1
S3150802A3202BFEA34B01221A70A249A3481EF07DFBFD
S3150802A330A0481EF047FB04469E481EF04FFB034604
S3150802A3401946204603F0BCFE0DF0F8FE034601222C
S3150802A350012118460EF0F0FB21E0934B1B68B3F17E
S3150802A360FF3F1CD10DF0EAFE0346322118460EF0D5
S3150802A3705FF9924810F0A6FA8E4991481EF055FBED
S3150802A3808C481EF01FFB04468A481EF027FB03462C
S3150802A3901946204603F094FE824B01221A70844B1A
S3150802A3A01B78012B12D1012000F028FE0346012B4F
S3150802A3B00CD17F4B00221A700DF0C0FE0446FEF740
S3150802A3C075FD0346194620460EF06CFAFEF7B6FEF0
S3150802A3D07868FFF781FA0346DAB27A4B1A70794B34
S3150802A3E01B78002B15D0784810F06CFA01217748B3
S3150802A3F020F0AFFD7649754821F03BFB1FF0FCFAC9
S3150802A400734B1B781A46734925F06CF8724B002277
S3150802A4101A80FEF7C9FC03461846FEF705FD0346F1
S3150802A420012B06D1674B1B78012B02D16B4B0122FC
S3150802A4301A70FEF7B9FC03461846FEF7F5FC034602
S3150802A440002B08D1654B00221A70634B00221A8032
S3150802A450634B00221A70614B1B78012B1FD1604B8C
S3150802A4601B78082B02D95E4B00221A705A4B1B889E
S3150802A47001339AB2584B1A80574B1B88B3F57A6F39
S3150802A4800DD3584810F01EFA554B1B780233DAB230
S3150802A490534B1A70504B00221A80FFF7C7FEFFF77C
S3150802A4A0B3FD0DF04BFE034618460EF0B4F803460C
S3150802A4B0012B40F0CE80786800F000FA03461A466F
S3150802A4C0494B1A70484B1B78002B00F0C2800DF0DE
S3150802A4D035FE034618460EF0F5F903461C460DF0FE
S3150802A4E02DFE034618460EF096F8034622463F49C5
S3150802A4F03F4826F0A7FF2F493D481EF096FA2D48F9
S3150802A5001EF060FA04462B481EF068FA03461946FE
S3150802A510204603F0D5FDFEF7C9FC03461946354821
S3150802A52010F0D0F9FEF740FC0346FF211846FEF765
S3150802A530A2FC0DF003FE0346022118460EF05BF854
S3150802A5400DF0FCFD0346002118460EF037F80DF013
S3150802A550F5FD034618460EF096F803469BB21946D1
S3150802A560254820F011FD254B1B780133DAB2234B1F
S3150802A5701A70224B1B7819461F4820F020FD02212B
S3150802A5801D4820F037FD1E491B4821F0D0FA1D4B05
S3150802A59001221A701C4810F095F91C4B00221A70F9
S3150802A5A046E000BFCED20020D0D200200C790508A2
S3150802A5B02FD300208CCF002024790508407905087E
S3150802A5C05C790508CDD200208C79050888D200204E
S3150802A5D08CD200208DD2002032D3002034D3002022
S3150802A5E030D30020B079050836D30020C079050893
S3150802A5F090D10020EC790508E8D200202DD300205E
S3150802A600ECD2002035D30020047A05082ED3002088
S3150802A610274B1B781A46274B13445B78194626485C
S3150802A62010F050F9224B1B780133DAB2204B1A701C
S3150802A630204B1A781E4B1B789A42E9D81F4810F00D
S3150802A64041F91FF021FA1B4B1B781A461C4925F0C3
S3150802A6502BF81C4B1B78012B26D1FEF7A5FB0346CC
S3150802A6601846FEF717FC0346012B1AD1FEF71EFC05
S3150802A67003461C46FEF798FB03461846FEF70AFCF5
S3150802A68003469C4206D0104810F01CF9012000F03F
S3150802A690B5FC09E00D4810F015F90A4B00221A70AC
S3150802A6A002E0084B00221A7000BF0C37BD4690BD67
S3150802A6B02ED30020ECD20020187A0508D477050894
S3150802A6C0EDD2002035D30020207A0508407A050805
S3150802A6D090B583B000AF0346FB71FB79012B40F0BE
S3150802A6E094806B496B481EF0A0F969481EF06AF916
S3150802A6F0044667481EF072F903461946204603F0D7
S3150802A700DFFCFEF7D3FB0346062B3AD0062B5ADCB0
S3150802A710012B05D0002B56DD023B032B53D80EE046
S3150802A720FEF742FB034603211846FEF753FBFEF7E4
S3150802A7303BFB034602211846FEF782FBA4E0564B72
S3150802A74000221A80FEF730FB034603211846FEF75D
S3150802A75041FBFEF729FB034602211846FEF770FB6A
S3150802A7604B494E481EF061F949481EF02BF904463A
S3150802A77047481EF033F903461946204603F0A0FC63
S3150802A78082E0454B00221A80FEF70EFB03460321A0
S3150802A7901846FEF71FFBFEF707FB0346012118467C
S3150802A7A0FEF74EFB3A493E481EF03FF938481EF07E
S3150802A7B009F9044636481EF011F903461946204699
S3150802A7C003F07EFC60E0344B00221A80FEF7ECFAB6
S3150802A7D0034603211846FEF7FDFAFEF7E5FA034695
S3150802A7E002211846FEF72CFB29492E481EF01DF9B0
S3150802A7F027481EF0E7F8044625481EF0EFF80346F8
S3150802A8001946204603F05CFC3EE0FB79022B21D177
S3150802A810254810F057F81E4924481EF006F91C4828
S3150802A8201EF0D0F804461A481EF0D8F80346194610
S3150802A830204603F045FCFEF7B7FA034603211846FD
S3150802A840FEF7C8FAFEF7B0FA034603211846FEF7E2
S3150802A850F7FA19E0164810F035F8FB791A46154941
S3150802A860154826F0EFFD0A4913481EF0DEF8084897
S3150802A8701EF0A8F8044606481EF0B0F80346194624
S3150802A880204603F01DFCFFE700BF0C37BD4690BD0E
S3150802A8908CCF00208C7A0508DED20020A47A05081F
S3150802A8A0D07A0508FC7A05082C7B05084C7B050836
S3150802A8B0747B0508987B050890D10020B0B584B052
S3150802A8C002AF7860BB4B1B78062B00F2488301A2C5
S3150802A8D052F823F0F1A80208A5AB020801AC020857
S3150802A8E05DAD02082DAF02082DAF02082DAF020892
S3150802A8F0FEF7DCFA0346002B00F01A81FEF7D6FAB9
S3150802A90003461C46FEF750FA03461846FEF7C2FAF5
S3150802A91003469C4200F0D680FEF746FA03461846DE
S3150802A920FEF7B8FA03461C46FEF7C0FA03469C42EF
S3150802A9305ED9FEF739FA03461846FEF7ABFA03461E
S3150802A9401C46FEF7B3FA0346E31ADAB29A4B1A70B2
S3150802A950994B1B78194699480FF0B4FFFEF7A6FAE9
S3150802A96003461C46944B1B781D46FEF71DFA034602
S3150802A9701846FEF78FFA034600932B46224690495D
S3150802A980904826F05FFD90498E481EF04EF88E4894
S3150802A9901EF018F804468C481EF020F8034619469D
S3150802A9A0204603F08DFB894B1B680022DA63874B2E
S3150802A9B01B683C221A640821844818F0B9FB0C214A
S3150802A9C0824818F055FA7B4B01221A70804B0222F4
S3150802A9D01A7010217F4811F0E1FF0346012B03D0BC
S3150802A9E032201CF05DFFBAE264201CF059FFB6E281
S3150802A9F0FEF75CFA03461C46FEF7D6F903461846E6
S3150802AA00FEF748FA0346E31ADAB26B4B1A706A4B38
S3150802AA101B78194669480FF055FFFEF747FA0346B1
S3150802AA201C46654B1B781D46FEF7BEF903461846BB
S3150802AA30FEF730FA034600932B46224666496148DA
S3150802AA4026F000FD60495F481DF0EFFF5E481DF0E5
S3150802AA50B9FF04465C481DF0C1FF03461946204665
S3150802AA6003F02EFB594B1B683C22DA63574B1B68D3
S3150802AA7000221A640821554818F0FAF90C2153489D
S3150802AA8018F056FB4B4B01221A70514B01221A70D1
S3150802AA90494B1B78012B11D1FEF708FA0346062B00
S3150802AAA00CD1FEF781F903461846FEF7F3F9034679
S3150802AAB0052B03D1C8201CF0F3FE72E0C8201CF057
S3150802AAC0EFFE4CE23B4B00221A700DF037FB0446B0
S3150802AAD0FEF7ECF90346194620460DF0E3FEFEF7AB
S3150802AAE063F903461846FEF7D5F9034619463B4865
S3150802AAF00FF0E8FEFEF758F903461846FEF7CAF9BC
S3150802AB0003461A4636492F4826F09CFC2E492D48FC
S3150802AB101DF08BFF2C481DF055FF04462A481DF0F0
S3150802AB205DFF03461946204603F0CAFA012317E2D7
S3150802AB302C4B00221A802C480FF0C4FE2B4B002205
S3150802AB401A70786800F022FB0346DAB2284B1A70AC
S3150802AB50274B1B78012B07D1FEF7A8F9034619469E
S3150802AB6024480FF0AFFE1CE01E4B1B8801339AB235
S3150802AB701C4B1A801B4B1B8844F61F62934207D94B
S3150802AB80184B00221A801C480FF09CFEFF23E7E1AF
S3150802AB9001201CF085FE7B68DBB218460FF0D0FF59
S3150802ABA0CFE7DCE1154B00221A80024B02221A700B
S3150802ABB0D5E100BF40D3002041D30020C87B050859
S3150802ABC0DC7B050890D100208CCF002060E70020AE
S3150802ABD042D30020001402420C7C05083C7C05087E
S3150802ABE0587C050848D30020787C0508D7D200206F
S3150802ABF046D30020907C0508B87C050844D300207B
S3150802AC00B44B1B8801339AB2B24B1A80B14B1B88DC
S3150802AC1042F20F72934223D9642001F0E3FCAE4B51
S3150802AC201B78002B1CD1AD480FF04CFEA94B002215
S3150802AC301A80AB49AB481DF0F8FEA9481DF0C2FEC2
S3150802AC400446A7481DF0CAFE03461946204603F0E5
S3150802AC5037FA21F0F7FC0123272266210EF004F8C1
S3150802AC604021A14811F09AFE0346012B0ED19A4BB8
S3150802AC701B780133DAB2984B1A70974B1B78194630
S3150802AC809A480FF01FFE64201CF00AFE984B1B78A8
S3150802AC90012B25D1904B1A78964B1B789A4208D1EC
S3150802ACA08D4B1B78194694480FF00CFE3C2001F098
S3150802ACB099FC894B1A78914B1B789A4240F04E813F
S3150802ACC0854B1B7819468E480FF0FCFD642001F06F
S3150802ACD089FC8C4B03221A70854B00221A703DE1BF
S3150802ACE07D4B1A78884B1B789A4240F037817A4B0B
S3150802ACF01B78194682480FF0E5FD774B1B781A46F2
S3150802AD008249834826F09EFB754981481DF08DFECF
S3150802AD1073481DF057FE044671481DF05FFE034650
S3150802AD201946204603F0CCF97A4B1B686422DA638B
S3150802AD30784B1B6864221A640821764818F098F83A
S3150802AD400C21744818F094F86E4B03221A70684B5B
S3150802AD5000221A70604B00221A70FFE040216248F6
S3150802AD6011F01CFE0346012B40F08780642001F097
S3150802AD7039FCFEF79BF803461C46FEF715F8034610
S3150802AD801846FEF787F803469C4234D10DF0D6F9E9
S3150802AD900446FEF78BF80346194620460DF082FD57
S3150802ADA0FEF702F803461846FEF774F803461946F4
S3150802ADB059480FF087FDFDF7F7FF03461846FEF7D9
S3150802ADC069F803461A465549514826F03BFB444959
S3150802ADD04F481DF02AFE42481DF0F4FD044640483D
S3150802ADE01DF0FCFD03461946204603F069F9454B5A
S3150802ADF004221A706AE0FEF759F803461C46FDF764
S3150802AE00D3FF03461846FEF745F803461A46214677
S3150802AE1043480FF057FDFEF749F803461C46FDF76F
S3150802AE20C3FF03461846FEF735F8034622463D4950
S3150802AE30374826F007FB2A4935481DF0F6FD28480B
S3150802AE401DF0C0FD044626481DF0C8FD03461946F6
S3150802AE50204603F035F9FDF7A7FF0446FDF7A4FFE0
S3150802AE6003461846FEF716F8034619462046FEF725
S3150802AE7002F8244B00221A7071E02B4B1B78022B26
S3150802AE8010D1244B1B681422DA63224B1B6800225A
S3150802AE901A6408211F4817F0EBFF0C211D4818F009
S3150802AEA047F913E0204B1B78012B0FD1194B1B686E
S3150802AEB00022DA63174B1B6814221A640821154804
S3150802AEC018F036F90C21134817F0D2FF024B00226C
S3150802AED01A7044E044D300203CD30020E07C0508E5
S3150802AEE08CCF0020147D050800100242507D05080B
S3150802AEF03ED300203FD30020687D05083DD30020BD
S3150802AF00807D050840D3002041D30020987D05089E
S3150802AF1090D1002060E70020CC7D0508E07D050879
S3150802AF20047E05083C7E050842D300200E480FF031
S3150802AF30C9FC0E490E481DF078FD0C481DF042FD6D
S3150802AF4004460A481DF04AFD03461946204603F000
S3150802AF50B7F8084B00221A70012301E000BF00234C
S3150802AF6018460837BD46B0BD6C7E05088CCF002052
S3150802AF70847E050840D3002080B500AF00F0B0FCFF
S3150802AF8003460321184601F019FE0346012B13D086
S3150802AF9000F0A6FC03460121184601F00FFE0346FF
S3150802AFA0012B09D000F09CFC03460221184601F049
S3150802AFB005FE0346012B17D10D480FF083FC0D4BF6
S3150802AFC01B680022DA630B4B1B680A221A640821E3
S3150802AFD0084818F0ADF80C21064817F049FF064B49
S3150802AFE009221A70012300E00023184680BD00BF1B
S3150802AFF0AC7E0508F8E70020DAD2002090B583B0C7
S3150802B00000AF0346FB71554B1B78002B02D0012B70
S3150802B01041D09EE0FB79002B13D051480FF052FC29
S3150802B020504B1B680022DA634E4B1B6808221A64CF
S3150802B03008214C4818F07CF80C214A4817F018FFEA
S3150802B04012E049480FF03EFC464B1B680F22DA63B2
S3150802B050444B1B6800221A640821424818F068F813
S3150802B0600C21404817F004FF3C4B01221A703F4B53
S3150802B07000221A803E493F481DF0D7FC3C481DF085
S3150802B080A1FC04463A481DF0A9FC03461946204687
S3150802B09003F016F85DE04021374811F07FFC0346BD
S3150802B0A0012B26D1642001F09DFAFDF7FFFE034627
S3150802B0B0194632480FF006FCFDF7F8FE03461A4613
S3150802B0C02E492F4826F0BEF929492D481DF0ADFC18
S3150802B0D027481DF077FC044625481DF07FFC0346E9
S3150802B0E01946204602F0ECFF1C4B00221A70012377
S3150802B0F030E01E4B1B8801339AB21C4B1A801B4B3D
S3150802B1001B8842F20F72934222D9144B00221A70FC
S3150802B110642001F067FA154B00221A8019480FF0CD
S3150802B120D1FB1949164826F08DF9114914481DF024
S3150802B1307CFC0F481DF046FC04460D481DF04EFCEB
S3150802B14003461946204602F0BBFF4FF0FF3301E0E3
S3150802B15000BF002318460C37BD4690BDD6D2002044
S3150802B160CC7E050860E70020F87E05084AD3002051
S3150802B1708CCF0020247F0508001002424C7F050868
S3150802B18090D10020707F0508907F050890B583B09E
S3150802B19000AF78605E4B1B78002B02D0012B2DD0B6
S3150802B1A0B1E05C480FF08EFB5B495C481DF03DFC44
S3150802B1B059481DF007FC044657481DF00FFC034684
S3150802B1C01946204602F07CFF554B00221A80554B41
S3150802B1D01B681422DA63534B1B6800221A640C217B
S3150802B1E0504817F0A5FF08214E4817F041FE4E4B6E
S3150802B1F000221A70464B01221A7084E040214B48FD
S3150802B20011F0CCFB0346012B26D1642001F0EAF9A2
S3150802B210FDF74CFE0346194645480FF053FBFDF76A
S3150802B22045FE03461A464249424826F00BF93A4970
S3150802B23040481DF0FAFB38481DF0C4FB0446364860
S3150802B2401DF0CCFB03461946204602F039FF304B67
S3150802B25000221A70012357E0334B1B78002B0FD1BB
S3150802B2601021354811F09AFB0346012B08D06420B9
S3150802B27001F0B8F92C4B01221A7030480FF022FB64
S3150802B280294B1B78012B15D10020FFF7B7FE034681
S3150802B290DAB22B4B1A702A4B1B78012B0AD1294892
S3150802B2A00FF010FB1A4B00221A701F4B00221A705D
S3150802B2B0012329E01A4B1B8801339AB2184B1A80CC
S3150802B2C0174B1B8842F6DF6293421BD9642001F0B2
S3150802B2D089F90F4B00221A70114B00221A800E4967
S3150802B2E019481DF0A2FB0C481DF06CFB04460A48DF
S3150802B2F01DF074FB03461946204602F0E1FE4FF0A4
S3150802B300FF3301E000BF002318460C37BD4690BD47
S3150802B310D7D20020AC7F05088CCF0020E07F050835
S3150802B3204CD3002060E700204ED3002000100242D2
S3150802B3301080050890D10020001402423C800508BE
S3150802B3404FD30020608005088C80050880B500AFC1
S3150802B350344B1B78002B02D0012B2FD05FE0324BE7
S3150802B3601B8801339AB2304B1A802F4B1B88952BB8
S3150802B37052D92E4B1B780133DAB22C4B1A702B4B4F
S3150802B3801B78042B03D9274B01221A7044E0284B59
S3150802B3901B686322DA63264B1B6863221A640C2134
S3150802B3A0234817F065FD0821214817F061FD1E4B59
S3150802B3B000221A801B4B01221A702DE01A4B1B8899
S3150802B3C001339AB2184B1A80174B1B88B3F57A7F4A
S3150802B3D024D3154B00221A80124B00221A70144BE2
S3150802B3E01B6800221A64114B1B78042B07D90F4BD2
S3150802B3F000221A700E4B1B680A22DA6303E00C4B12
S3150802B4001B686422DA630821094817F031FD0C210A
S3150802B410074817F08DFE01E000BF00E000BF00BF3D
S3150802B42080BD00BFD4D2002050D30020D5D2002040
S3150802B430F8E7002080B500AF344B1B78002B02D00A
S3150802B440012B2FD05FE0324B1B8801339AB2304B67
S3150802B4501A802F4B1B88952B52D92E4B1B780133FA
S3150802B460DAB22C4B1A702B4B1B78042B03D9274BB9
S3150802B47001221A7012E0284B1B686322DA63264BF4
S3150802B4801B6863221A640C21234817F0F1FC082171
S3150802B490214817F0EDFC1D4B01221A701C4B0022A5
S3150802B4A01A802DE01A4B1B8801339AB2184B1A8060
S3150802B4B0174B1B88B3F57A7F24D3154B00221A80C3
S3150802B4C0124B00221A70144B1B680022DA63114BC6
S3150802B4D01B78042B07D90F4B00221A700E4B1B68D8
S3150802B4E008221A6403E00C4B1B6864221A640C21B6
S3150802B4F0094817F0BDFC0821074817F019FE01E0B4
S3150802B50000BF00E000BF00BF80BD00BFD4D200204C
S3150802B51050D30020D5D20020F8E7002098B500AF16
S3150802B5207E4B1B78002B02D0012B2AD0F2E07C48F6
S3150802B5300FF0C8F97B497C481DF077FA79481DF067
S3150802B54041FA044677481DF049FA03461946204649
S3150802B55002F0B6FD754B1B681E22DA63734B1B6835
S3150802B56000221A640821714817F082FC0C216F48E0
S3150802B57017F0DEFD6E4B01221A70684B01221A7013
S3150802B580C8E010216B4811F009FA0346012B00F0B6
S3150802B5908A80642001F026F8674B1B780133DAB2F9
S3150802B5A0654B1A70644B1B78632B7CD9624B00225D
S3150802B5B01A70002001F016F8584B00221A705F4BD9
S3150802B5C01B885F4AA2FB03239B099BB219465D4867
S3150802B5D00FF078F9594B1B88594AA2FB03239B099A
S3150802B5E09BB21A465749584825F02CFF4D495648EA
S3150802B5F01DF01BFA4B481DF0E5F9044649481DF0B3
S3150802B600EDF903461946204602F05AFD484B022236
S3150802B6101A704A4B00221A8000F062F90346032187
S3150802B620184601F0CBFA0346012B3AD100F058F935
S3150802B63003460121184601F0C1FA0346022B13D12B
S3150802B640424B1B680022DA63404B1B6864221A6469
S3150802B65008213E4817F06CFD0C213C4817F008FCFF
S3150802B6603B4B03221A701CE000F03AF9034602210A
S3150802B670184601F0A3FA0346022B12D1334B1B6874
S3150802B6806422DA63314B1B6800221A6408212F48A8
S3150802B69017F0EEFB0C212D4817F04AFD2C4B03221E
S3150802B6A01A70012337E0224B1B78012B31D1234B29
S3150802B6B01B8801339AB2214B1A80204B1B8842F20F
S3150802B6C00F72934225D923480FF0FCF8002000F0A8
S3150802B6D089FF144920481DF0A8F912481DF072F98D
S3150802B6E0044610481DF07AF903461946204602F028
S3150802B6F0E7FC20F0A7FF0123262266210DF0B4FA03
S3150802B7000E4B00221A80054B00221A704FF0FF33A7
S3150802B71001E000BF0023184698BD00BF37D30020BA
S3150802B720BC8005088CCF0020D480050860E700207D
S3150802B73039D300200014024238D300203AD300201D
S3150802B740D34D6210F480050890D10020F8E7002056
S3150802B750DAD20020108105083481050880B582B046
S3150802B76000AF0346FB71304B1B78632B4DD0632B1E
S3150802B77051DC002B02D0012B11D04CE02B4B0022BE
S3150802B7801A80FB79012B03D1642001F0B3FD02E094
S3150802B790642001F093FD244B01221A703EE0FB79E6
S3150802B7A0012B0FD100F09CF80346184601F023FE40
S3150802B7B00346022B16D101F0B9FD1B4B00221A7063
S3150802B7C001232CE000F08CF80346184601F0EAFD46
S3150802B7D00346022B06D101F0A9FD134B00221A706B
S3150802B7E001231CE0114B1B8801339AB20F4B1A80B6
S3150802B7F00E4B1B88632B10D901F0AEFD0B4B0022B2
S3150802B8001A80094B63221A7007E0074B00221A7046
S3150802B8104FF0FF3303E000BF00E000BF00231846E5
S3150802B8200837BD4680BD00BF52D3002054D300203E
S3150802B83080B500AF074B1B78DBB2002B07D1054B4F
S3150802B84001221A7002220021034825F08FFE024BBC
S3150802B850184680BD68D300206CD3002080B483B01C
S3150802B86000AF78600B46FB707B68FA781A7000BFE7
S3150802B8700C37BD465DF8047B704780B582B000AFD1
S3150802B88078600B46FB707B68FA785A70FB78002B57
S3150802B89006D0FB78052B03D800217868FFF7DEFF70
S3150802B8A000BF0837BD4680BD80B400AF084B0022F2
S3150802B8B01A70084B00221A70074B00221A80074B8F
S3150802B8C000221A6000BFBD465DF8047B704700BFC0
S3150802B8D05DD300205ED3002060D3002064D300200D
S3150802B8E080B500AF174B1B78DBB2002B27D1154B5F
S3150802B8F001221A7034220221134825F037FE124B10
S3150802B9000122DA77012200210F4800F0B1F801225C
S3150802B91001210D4800F0ACF8012202210A4800F084
S3150802B920A7F801220321084800F0A2F801220421FF
S3150802B930054800F09DF80121034800F0ADF8024BD6
S3150802B940184680BD89D300208CD3002080B483B0EA
S3150802B95000AF78607B68DB79012B01D1012306E011
S3150802B9607B68DB79022B01D1022300E0002318460B
S3150802B9700C37BD465DF8047B704780B483B000AFD0
S3150802B98078600B46FB707B68FA78DA7101231846F1
S3150802B9900C37BD465DF8047B704780B483B000AFB0
S3150802B9A078600B46FB70FB787A6813441B7A012B86
S3150802B9B001D1012308E0FB787A6813441B7A022B2B
S3150802B9C001D1022300E0002318460C37BD465DF874
S3150802B9D0047B704780B483B000AF78600B46FB7077
S3150802B9E01346BB70FB787A681344BA781A72012335
S3150802B9F018460C37BD465DF8047B704780B483B0A1
S3150802BA0000AF78600B46FB70FB787A6813441B7BA1
S3150802BA10012B01D1012308E0FB787A6813441B7BCA
S3150802BA20022B01D1022300E0002318460C37BD463B
S3150802BA305DF8047B704780B483B000AF78600B462C
S3150802BA40FB70FB787A6813445B7D012B01D10123D5
S3150802BA5008E0FB787A6813445B7D022B01D1022346
S3150802BA6000E0002318460C37BD465DF8047B704794
S3150802BA7080B483B000AF78600B46FB701346BB7088
S3150802BA80FB787A681344BA785A75012318460C3734
S3150802BA90BD465DF8047B704780B483B000AF78601A
S3150802BAA00B46FB707B68FA781A77012318460C371F
S3150802BAB0BD465DF8047B704780B483B000AF7860FA
S3150802BAC00B46FB70FB787A68134493F82630012BF1
S3150802BAD001D1012309E0FB787A68134493F82630EA
S3150802BAE0022B01D1022300E0002318460C37BD467B
S3150802BAF05DF8047B704780B483B000AF78600B466C
S3150802BB00FB701346BB70FB787A681344BA7883F8DD
S3150802BB102620012318460C37BD465DF8047B70477C
S3150802BB2080B483B000AF78607B6893F82A30012B23
S3150802BB3001D1012307E07B6893F82A30022B01D151
S3150802BB40022300E0002318460C37BD465DF8047B45
S3150802BB50704780B483B000AF78600B46FB707B6891
S3150802BB60FA7883F82A20012318460C37BD465DF871
S3150802BB70047B704780B483B000AF78607B6893F823
S3150802BB80253018460C37BD465DF8047B704780B4ED
S3150802BB9083B000AF78600B46FB707B68FA7883F84F
S3150802BBA02520012318460C37BD465DF8047B7047ED
S3150802BBB080B483B000AF78607B6893F82B30184660
S3150802BBC00C37BD465DF8047B704780B483B000AF7E
S3150802BBD078607B6893F82C3018460C37BD465DF8BA
S3150802BBE0047B704780B483B000AF78600B46FB7065
S3150802BBF07B68FA7883F82C2000BF0C37BD465DF8BF
S3150802BC00047B704780B582B000AF0346FB71FB79AF
S3150802BC101846F4F7A5FD02460B463649C1E9002344
S3150802BC20FB79002B3AD0FFF75BFE03460321184641
S3150802BC3000F0BFF9FFF754FE03461846FFF79AFFCE
S3150802BC400346012B10D12C4B1B68FA79DA632B4B6E
S3150802BC501B78002B49D00821274817F009F9042137
S3150802BC60254817F065FA40E0FFF73AFE03461846FC
S3150802BC70FFF780FF0346022B37D11F4B1B68FA7961
S3150802BC809A631E4B1B78002B2FD008211A4817F0EF
S3150802BC904FFA0421184817F0EBF826E0FB79002B37
S3150802BCA023D1FFF71DFE0346184600F075F9034631
S3150802BCB0012B06D0FFF714FE03460421184600F0AE
S3150802BCC078F90F4B1B78002B0FD10B4B1B6863229D
S3150802BCD0DA63094B1B6863229A630821064817F040
S3150802BCE0C7F80421044817F0C3F800BF0837BD4651
S3150802BCF080BD00BF70D30020ACE7002078D30020B7
S3150802BD00F8F2002080B400AF064BD3E9002343ECD7
S3150802BD10172BB0EE470AF0EE670ABD465DF8047BBC
S3150802BD20704700BF70D3002080B500AFFFF7D8FD7B
S3150802BD30034601211846FFF72AFF00BF80BD80B5DA
S3150802BD4000AFFFF7CDFD034602211846FFF71FFF96
S3150802BD5000BF80BD80B500AFFFF7C2FD03460321D1
S3150802BD60184600F026F9FFF7DFFFFFF7CBFF51EC85
S3150802BD70100B4FF000024FF00003F4F7D3FF03460F
S3150802BD80002B08D008210A4817F0D2F904210848DE
S3150802BD9017F0CEF907E00821054817F069F80421DB
S3150802BDA0034817F0C5F9034B01221A7000BF80BD7C
S3150802BDB0ACE7002078D3002080B500AFFFF790FDEE
S3150802BDC003460421184600F0F4F8054B00221A70BF
S3150802BDD0044B00221A700020FFF714FF00BF80BD33
S3150802BDE078D3002079D3002080B500AFFFF778FD1D
S3150802BDF003460321184600F0DCF8FFF7A0FFFFF719
S3150802BE0081FF51EC100B4FF000024FF00003F4F7DC
S3150802BE1089FF0346002B08D008210A4817F088F93B
S3150802BE200421084817F084F907E00821054817F0A5
S3150802BE307FF90421034817F01BF8034B01221A70F5
S3150802BE4000BF80BDACE7002078D3002080B500AFE4
S3150802BE50FFF746FD03460421184600F0AAF8064BEA
S3150802BE6000221A70054B00221A700020FFF7CAFE3C
S3150802BE70FFF75AFF00BF80BD78D3002079D3002090
S3150802BE8080B500AFFFF72CFD03460221184600F0E5
S3150802BE9090F80821074817F04BF90421054817F0CE
S3150802BEA047F9054B00221A70044B00221A7000BF8C
S3150802BEB080BD00BFACE7002078D3002079D30020EC
S3150802BEC080B500AFFFF70CFD03460121184600F0C6
S3150802BED070F80821074817F02BF90421054817F0CE
S3150802BEE027F9054B00221A70044B00221A7000BF6C
S3150802BEF080BD00BFACE7002078D3002079D30020AC
S3150802BF0080B500AF00228021054810F05FFDFFF7DB
S3150802BF10E7FC03460121184600F05BF800BF80BD26
S3150802BF200010024280B500AF01228021054810F0B8
S3150802BF304DFDFFF7D5FC03460221184600F049F8E5
S3150802BF4000BF80BD0010024280B500AF00224FF448
S3150802BF508071064810F03AFDFFF7C2FC034601213C
S3150802BF60184600F047F800BF80BD00BF0010024225
S3150802BF7080B500AF01224FF48071064810F026FD05
S3150802BF80FFF7AEFC03460221184600F033F800BF5D
S3150802BF9080BD00BF0010024280B483B000AF786053
S3150802BFA07B6893F8223018460C37BD465DF8047B49
S3150802BFB0704780B483B000AF78600B46FB707B682D
S3150802BFC0FA7883F8222000BF0C37BD465DF8047B59
S3150802BFD0704780B483B000AF78600B46FB707B680D
S3150802BFE0FA7883F82320012318460C37BD465DF8F4
S3150802BFF0047B704780B483B000AF78600B46FB7051
S3150802C0007B68FA7883F82420012318460C37BD4644
S3150802C0105DF8047B7047000080B582B000AF4FF42C
S3150802C0208071404810F0BAFC0346012B0CBF01236D
S3150802C0300023DBB2BB710023FB713B4B1B78BA7939
S3150802C0409A421BD1394B1B78012B02D9BB79FB715A
S3150802C05028E0364B1B780133DAB2344B1A70FFF7F5
S3150802C0603FFC03461846FFF771FC0346012B02D133
S3150802C0700123FB7116E00023FB7113E02A4ABB7900
S3150802C08013702A4B00221A70FFF72AFC0346184639
S3150802C090FFF75CFC0346012B02D10123FB7101E089
S3150802C0A00023FB71FB79002B1CD0FFF719FC034612
S3150802C0B001211846FFF761FC1D4B1B78FA799A4253
S3150802C0C02CD00CF03BF80346042118460CF02DF947
S3150802C0D00346002B02D017480EF0F4FB144AFB79EC
S3150802C0E013701BE0FFF7FCFB034602211846FFF715
S3150802C0F044FC0F4B1B78FA799A420FD00CF01EF8C3
S3150802C1000346042118460CF010F90346002B02D008
S3150802C11009480EF0D7FB064AFB79137000BF0837A9
S3150802C120BD4680BD000C0242C0D30020C1D3002008
S3150802C130C2D30020008505083885050880B582B077
S3150802C14000AF4021404810F029FC0346012B0CBFE2
S3150802C15001230023DBB2BB710023FB713B4B1B7827
S3150802C160BA799A421BD13A4B1B78012B02D9BB7971
S3150802C170FB7128E0364B1B780133DAB2344B1A705E
S3150802C180FFF7AEFB03461846FFF7CAFC0346012B28
S3150802C19002D10123FB7116E00023FB7113E02B4A3F
S3150802C1A0BB7913702A4B00221A70FFF799FB0346D4
S3150802C1B01846FFF7B5FC0346012B02D10123FB7192
S3150802C1C001E00023FB71FB79002B1CD0FFF788FBEB
S3150802C1D0034601211846FFF7BCFC1E4B1B78FA7969
S3150802C1E09A422CD00BF0AAFF0346042118460CF0FB
S3150802C1F09CF80346002B02D017480EF063FB154A3B
S3150802C200FB7913701BE0FFF76BFB03460221184606
S3150802C210FFF79FFC0F4B1B78FA799A420FD00BF067
S3150802C2208DFF0346042118460CF07FF80346002BBF
S3150802C23002D00A480EF046FB064AFB79137000BF85
S3150802C2400837BD4680BD00BF00100242C3D3002096
S3150802C250C4D30020C5D3002070850508AC8505081F
S3150802C26080B582B000AF0421424810F097FB03461E
S3150802C270012B0CBF01230023DBB2BB710023FB7128
S3150802C2803D4B1B78BA799A421CD13C4B1B78032B3F
S3150802C29002D9BB79FB712AE0384B1B780133DAB233
S3150802C2A0364B1A70FFF71CFB034600211846FFF7A8
S3150802C2B003FC0346012B02D10123FB7117E000237D
S3150802C2C0FB7114E02C4ABB7913702C4B00221A70AE
S3150802C2D0FFF706FB034600211846FFF7EDFB034668
S3150802C2E0012B02D10123FB7101E00023FB71FB79CB
S3150802C2F0002B1DD0FFF7F4FA034601220021184647
S3150802C300FFF7F9FB1E4B1B78FA799A422DD00BF0F0
S3150802C31015FF0346042118460CF007F80346002BBE
S3150802C32002D018480EF0CEFA154AFB7913701CE0B3
S3150802C330FFF7D6FA0346022200211846FFF7DBFB6F
S3150802C3400F4B1B78FA799A420FD00BF0F7FE034689
S3150802C350042118460BF0E9FF0346002B02D00A48CF
S3150802C3600EF0B0FA064AFB79137000BF0837BD46CD
S3150802C37080BD00BF00100242C6D30020C7D30020EA
S3150802C380C8D30020E88505082086050880B582B04E
S3150802C39000AF1021424810F001FB0346012B0CBFE7
S3150802C3A001230023DBB2BB710023FB713D4B1B78D3
S3150802C3B0BA799A421CD13C4B1B78032B02D9BB791A
S3150802C3C0FB712AE0384B1B780133DAB2364B1A7006
S3150802C3D0FFF786FA034601211846FFF76DFB034667
S3150802C3E0012B02D10123FB7117E00023FB7114E034
S3150802C3F02C4ABB7913702C4B00221A70FFF770FA7D
S3150802C400034601211846FFF757FB0346012B02D1C3
S3150802C4100123FB7101E00023FB71FB79002B1DD080
S3150802C420FFF75EFA0346012201211846FFF763FB6E
S3150802C4301E4B1B78FA799A422DD00BF07FFE0346E3
S3150802C440042118460BF071FF0346002B02D0184848
S3150802C4500EF038FA154AFB7913701CE0FFF740FA1A
S3150802C4600346022201211846FFF745FB0F4B1B78AC
S3150802C470FA799A420FD00BF061FE03460421184658
S3150802C4800BF053FF0346002B02D00A480EF01AFAA5
S3150802C490064AFB79137000BF0837BD4680BD00BF48
S3150802C4A000100242C9D30020CAD30020CBD30020F1
S3150802C4B05C8605089486050880B582B000AF082117
S3150802C4C0424810F06BFA0346012B0CBF01230023E6
S3150802C4D0DBB2BB710023FB713D4B1B78BA799A42DA
S3150802C4E01CD13C4B1B78032B02D9BB79FB712AE082
S3150802C4F0384B1B780133DAB2364B1A70FFF7F0F96C
S3150802C500034602211846FFF7D7FA0346012B02D142
S3150802C5100123FB7117E00023FB7114E02C4ABB7957
S3150802C52013702C4B00221A70FFF7DAF90346022120
S3150802C5301846FFF7C1FA0346012B02D10123FB7104
S3150802C54001E00023FB71FB79002B1DD0FFF7C8F928
S3150802C5500346012202211846FFF7CDFA1E4B1B7825
S3150802C560FA799A422DD00BF0E9FD034604211846C2
S3150802C5700BF0DBFE0346002B02D018480EF0A2F998
S3150802C580154AFB7913701CE0FFF7AAF90346022243
S3150802C59002211846FFF7AFFA0F4B1B78FA799A422F
S3150802C5A00FD00BF0CBFD0346042118460BF0BDFE57
S3150802C5B00346002B02D00A480EF084F9064AFB7994
S3150802C5C0137000BF0837BD4680BD00BF0010024287
S3150802C5D0CCD30020CDD30020CED30020D0860508A8
S3150802C5E00887050880B582B000AF0346FB71FB7960
S3150802C5F01846F4F7B5F802460B464149C1E9002345
S3150802C600FB79642B10D13F4B1B686422DA633D4BDE
S3150802C6101B6864221A6408213A4816F029FC0C2180
S3150802C620384816F025FC66E0FB79002B3ED0FB79EC
S3150802C630632B3BD8FFF754F903461846FFF7B8FAB7
S3150802C6400346012B14D12F4B1B68FA79DA632D4B5B
S3150802C6501B6800221A642C4B1B78002B4AD008212F
S3150802C660284816F005FC0C21264816F061FD41E023
S3150802C670FFF736F903461846FFF79AFA0346022BDE
S3150802C68038D1204B1B68FA791A641E4B1B680022A4
S3150802C690DA631D4B1B78002B2CD00C21194816F097
S3150802C6A0E7FB0821174816F043FD23E0FB79002B28
S3150802C6B021D1FFF715F903461846FFF786FA03460E
S3150802C6C0012B06D0FFF70CF9034604211846FFF79B
S3150802C6D089FA0C4B1B680022DA630A4B1B68002294
S3150802C6E01A640C21074816F023FD0821054816F09E
S3150802C6F01FFD00E000BF00BF0837BD4680BD00BF72
S3150802C70080D3002060E7002088D3002080B582B05D
S3150802C71000AF4FF40071424810F040F90346012B6E
S3150802C7200CBF01230023DBB2BB710023FB713D4B17
S3150802C7301B78BA799A421CD13B4B1B78032B02D938
S3150802C740BB79FB712AE0384B1B780133DAB2364BD8
S3150802C7501A70FFF7C5F8034600211846FFF71DF9B8
S3150802C7600346012B02D10123FB7117E00023FB715B
S3150802C77014E02C4ABB7913702B4B00221A70FFF770
S3150802C780AFF8034600211846FFF707F90346012BBF
S3150802C79002D10123FB7101E00023FB71FB79002B17
S3150802C7A01DD0FFF79DF80346012200211846FFF720
S3150802C7B011F91E4B1B78FA799A422DD00BF0BEFC62
S3150802C7C00346042118460BF0B0FD0346002B02D09F
S3150802C7D017480EF077F8154AFB7913701CE0FFF735
S3150802C7E07FF80346022200211846FFF7F3F80F4B9B
S3150802C7F01B78FA799A420FD00BF0A0FC0346042163
S3150802C80018460BF092FD0346002B02D009480EF09B
S3150802C81059F8064AFB79137000BF0837BD4680BD32
S3150802C820000C0242CFD30020D0D30020D1D300205F
S3150802C830448705088087050880B582B000AF4FF4A3
S3150802C8408061424810F0AAF80346012B0CBF012367
S3150802C8500023DBB2BB710023FB713D4B1B78BA790F
S3150802C8609A421CD13B4B1B78032B02D9BB79FB712D
S3150802C8702AE0384B1B780133DAB2364B1A70FFF7C7
S3150802C8802FF8034601211846FFF787F80346012BBE
S3150802C89002D10123FB7117E00023FB7114E02C4A35
S3150802C8A0BB7913702B4B00221A70FFF719F803464F
S3150802C8B001211846FFF771F80346012B02D101231D
S3150802C8C0FB7101E00023FB71FB79002B1DD0FFF7FA
S3150802C8D007F80346012201211846FFF77BF81E4B8B
S3150802C8E01B78FA799A422DD00BF028FC03460421CC
S3150802C8F018460BF01AFD0346002B02D017480DF016
S3150802C900E1FF154AFB7913701CE0FEF7E9FF0346BF
S3150802C910022201211846FFF75DF80F4B1B78FA79B8
S3150802C9209A420FD00BF00AFC0346042118460BF074
S3150802C930FCFC0346002B02D009480DF0C3FF064A49
S3150802C940FB79137000BF0837BD4680BD000C024252
S3150802C950D2D30020D3D30020D4D30020C087050821
S3150802C960FC87050880B582B000AF4FF400614248E3
S3150802C97010F014F80346012B0CBF01230023DBB287
S3150802C980BB710023FB713D4B1B78BA799A421CD1C5
S3150802C9903B4B1B78032B02D9BB79FB712AE0384B38
S3150802C9A01B780133DAB2364B1A70FEF799FF034643
S3150802C9B002211846FEF7F1FF0346012B02D1012395
S3150802C9C0FB7117E00023FB7114E02C4ABB79137044
S3150802C9D02B4B00221A70FEF783FF034602211846E4
S3150802C9E0FEF7DBFF0346012B02D10123FB7101E0AF
S3150802C9F00023FB71FB79002B1DD0FEF771FF03465E
S3150802CA00012202211846FEF7E5FF1E4B1B78FA792A
S3150802CA109A422DD00BF092FB0346042118460BF0DE
S3150802CA2084FC0346002B02D017480DF04BFF154A2B
S3150802CA30FB7913701CE0FEF753FF0346022202211C
S3150802CA401846FEF7C7FF0F4B1B78FA799A420FD0A2
S3150802CA500BF074FB0346042118460BF066FC0346EA
S3150802CA60002B02D009480DF02DFF064AFB791370F8
S3150802CA7000BF0837BD4680BD000C0242D5D3002050
S3150802CA80D6D30020D7D300203C8805087888050825
S3150802CA9080B582B000AF4FF4805142480FF07EFF56
S3150802CAA00346012B0CBF01230023DBB2BB71002313
S3150802CAB0FB713D4B1B78BA799A421CD13B4B1B78CA
S3150802CAC0032B02D9BB79FB712AE0384B1B78013359
S3150802CAD0DAB2364B1A70FEF703FF034603211846ED
S3150802CAE0FEF75BFF0346012B02D10123FB7117E018
S3150802CAF00023FB7114E02C4ABB7913702B4B0022DE
S3150802CB001A70FEF7EDFE034603211846FEF745FFA7
S3150802CB100346012B02D10123FB7101E00023FB71BD
S3150802CB20FB79002B1DD0FEF7DBFE0346012203210B
S3150802CB301846FEF74FFF1E4B1B78FA799A422DD0FC
S3150802CB400BF0FCFA0346042118460BF0EEFB0346EB
S3150802CB50002B02D017480DF0B5FE154AFB79137063
S3150802CB601CE0FEF7BDFE0346022203211846FEF725
S3150802CB7031FF0F4B1B78FA799A420FD00BF0DEFA87
S3150802CB800346042118460BF0D0FB0346002B02D0BD
S3150802CB9009480DF097FE064AFB79137000BF08375D
S3150802CBA0BD4680BD000C0242D8D30020D9D300204E
S3150802CBB0DAD30020B8880508F488050880B483B05B
S3150802CBC000AF78600B46FB70FB787A68134493F8DB
S3150802CBD02D30012B01D1012309E0FB787A68134431
S3150802CBE093F82D30022B01D1022300E000231846C8
S3150802CBF00C37BD465DF8047B704780B483B000AF3E
S3150802CC0078600B46FB707B68FA7883F8312000BFA0
S3150802CC100C37BD465DF8047B704780B483B000AF1D
S3150802CC2078607B6893F83130012B01D1012307E044
S3150802CC307B6893F83130022B01D1022300E00023EE
S3150802CC4018460C37BD465DF8047B704780B483B03E
S3150802CC5000AF78600B46FB701346BB70FB787A68A8
S3150802CC601344BA7883F82D20012318460C37BD469B
S3150802CC705DF8047B7047000080B582B000AF0821DA
S3150802CC8042480FF08BFE0346012B0CBF01230023FB
S3150802CC90DBB2BB710023FB713D4B1B78BA799A4212
S3150802CCA01CD13C4B1B78312B02D9BB79FB712AE08C
S3150802CCB0384B1B780133DAB2364B1A70FEF710FE80
S3150802CCC0034601211846FFF779FF0346012B02D1D5
S3150802CCD00123FB7117E00023FB7114E02C4ABB7990
S3150802CCE013702C4B00221A70FEF7FAFD0346012137
S3150802CCF01846FFF763FF0346012B02D10123FB7196
S3150802CD0001E00023FB71FB79002B1DD0FEF7E8FD3D
S3150802CD100346012201211846FFF798FF1E4B1B788E
S3150802CD20FA799A422DD00BF009FA034604211846DD
S3150802CD300BF0FBFA0346002B02D018480DF0C2FD91
S3150802CD40154AFB7913701CE0FEF7CAFD0346022258
S3150802CD5001211846FFF77AFF0F4B1B78FA799A4298
S3150802CD600FD00BF0EBF90346042118460BF0DDFA57
S3150802CD700346002B02D00A480DF0A4FD064AFB79A9
S3150802CD80137000BF0837BD4680BD00BF00140242BB
S3150802CD90DBD30020DCD30020DDD3002080910508F8
S3150802CDA0BC91050880B582B000AF022142480FF057
S3150802CDB0F5FD0346012B0CBF01230023DBB2BB7131
S3150802CDC00023FB713D4B1B78BA799A421CD13C4B26
S3150802CDD01B78132B02D9BB79FB712AE0384B1B78D7
S3150802CDE00133DAB2364B1A70FEF77AFD0346022190
S3150802CDF01846FFF7E3FE0346012B02D10123FB7116
S3150802CE0017E00023FB7114E02C4ABB7913702C4BF4
S3150802CE1000221A70FEF764FD034602211846FFF740
S3150802CE20CDFE0346012B02D10123FB7101E000234B
S3150802CE30FB71FB79002B1DD0FEF752FD034601223A
S3150802CE4002211846FFF702FF1E4B1B78FA799A420F
S3150802CE502DD00BF073F90346042118460BF065FA38
S3150802CE600346002B02D018480DF02CFD154AFB7913
S3150802CE7013701CE0FEF734FD03460222022118460F
S3150802CE80FFF7E4FE0F4B1B78FA799A420FD00BF0A4
S3150802CE9055F90346042118460BF047FA0346002BB8
S3150802CEA002D00A480DF00EFD064AFB79137000BF40
S3150802CEB00837BD4680BD00BF00140242DED30020FB
S3150802CEC0DFD30020E0D30020FC910508389205083C
S3150802CED080B582B000AF042142480FF05FFD0346D9
S3150802CEE0012B0CBF01230023DBB2BB710023FB71AC
S3150802CEF03D4B1B78BA799A421CD13C4B1B78132BB3
S3150802CF0002D9BB79FB712AE0384B1B780133DAB2B6
S3150802CF10364B1A70FEF7E4FC034603211846FFF760
S3150802CF204DFE0346012B02D10123FB7117E00023B4
S3150802CF30FB7114E02C4ABB7913702C4B00221A7031
S3150802CF40FEF7CEFC034603211846FFF737FE0346D3
S3150802CF50012B02D10123FB7101E00023FB71FB794E
S3150802CF60002B1DD0FEF7BCFC0346012203211846FE
S3150802CF70FFF76CFE1E4B1B78FA799A422DD00BF0FE
S3150802CF80DDF80346042118460BF0CFF90346002BB9
S3150802CF9002D018480DF096FC154AFB7913701CE06E
S3150802CFA0FEF79EFC0346022203211846FFF74EFEB1
S3150802CFB00F4B1B78FA799A420FD00BF0BFF803464B
S3150802CFC0042118460BF0B1F90346002B02D00A4891
S3150802CFD00DF078FC064AFB79137000BF0837BD4688
S3150802CFE080BD00BF00140242E1D30020E2D3002034
S3150802CFF0E3D3002078920508B492050880B582B07A
S3150802D00000AF402144480FF0C9FC0346012B0CBF70
S3150802D01001230023DBB2FB71404B1B78FA799A4253
S3150802D0201ED13F4B1B78632B03D93E4AFB791370FB
S3150802D0302CE03B4B1B780133DAB2394B1A70FEF7F8
S3150802D0404FFC03461846FFF7E8FD0346012B03D1BA
S3150802D050344B01221A7019E0324B00221A7015E07D
S3150802D0602E4AFB7913702E4B00221A70FEF738FCF3
S3150802D07003461846FFF7D1FD0346012B03D1294B78
S3150802D08001221A7002E0274B00221A70254B1B78E0
S3150802D090002B1ED0FEF724FC034601211846FFF793
S3150802D0A0ACFD214B1A781F4B1B789A422FD00BF0F6
S3150802D0B045F80346042118460BF037F90346002BB8
S3150802D0C002D01A480DF0FEFB164B1A78164B1A7048
S3150802D0D01DE0FEF705FC034602211846FFF78DFD03
S3150802D0E0114B1A780F4B1B789A4210D00BF026F880
S3150802D0F00346042118460BF018F90346002B02D002
S3150802D1000B480DF0DFFB074B1A78074B1A7000BF66
S3150802D1100837BD4680BD00BF00100242E4D3002096
S3150802D120E5D30020E6D30020E7D30020789205084D
S3150802D130B492050880B500AF0821044815F098FE98
S3150802D1400C21024815F0F4FF00BF80BDF8E7002065
S3150802D15080B500AF0C21044815F08AFE0821024862
S3150802D16015F0E6FF00BF80BDF8E7002080B500AFE6
S3150802D170084B1B6863221A64064B1B686322DA6330
S3150802D1800C21044815F074FE0821024815F070FEB9
S3150802D19000BF80BDF8E7002080B582B000AF40210D
S3150802D1A040480FF0FBFB0346012B0CBF012300236B
S3150802D1B0DBB2BB710023FB713B4B1B78BA799A42EF
S3150802D1C01BD13A4B1B78012B02D9BB79FB7128E09C
S3150802D1D0364B1B780133DAB2344B1A70FEF780FBF2
S3150802D1E003461846FFF719FD0346012B02D1012310
S3150802D1F0FB7116E00023FB7113E02B4ABB7913700F
S3150802D2002A4B00221A70FEF76BFB03461846FFF7F5
S3150802D21004FD0346012B02D10123FB7101E0002321
S3150802D220FB71FB79002B1CD0FEF75AFB0346012142
S3150802D2301846FFF7E2FC1E4B1B78FA799A422CD065
S3150802D2400AF07CFF0346042118460BF06EF80346E3
S3150802D250002B02D017480DF035FB154AFB791370DF
S3150802D2601BE0FEF73DFB034602211846FFF7C5FC05
S3150802D2700F4B1B78FA799A420FD00AF05FFF0346E2
S3150802D280042118460BF051F80346002B02D00A482F
S3150802D2900DF018FB064AFB79137000BF0837BD4626
S3150802D2A080BD00BF00100242E8D30020E9D3002067
S3150802D2B0EAD30020008505083885050880B582B0BE
S3150802D2C000AF0346FB710021094815F0D1FD042180
S3150802D2D0074815F02DFF064B1B68FA795A63044B6B
S3150802D2E01B6800229A6300BF0837BD4680BD00BF8F
S3150802D2F0F8E7002080B582B000AF0346FB7104212F
S3150802D300094815F0B5FD0021074815F011FF064B2F
S3150802D3101B6800225A63044B1B68FA799A6300BF9A
S3150802D3200837BD4680BD00BFF8E7002080B500AFCC
S3150802D3300021084815F09CFD0421064815F098FDC1
S3150802D340044B1B6864229A63024B1B6864225A6365
S3150802D35000BF80BDF8E7002080B500AF002108486D
S3150802D36015F0E6FE0421064815F0E2FE044B1B689A
S3150802D37000229A63024B1B6800225A6300BF80BDD3
S3150802D380F8E7002080B483B000AF78600B46FB70E4
S3150802D3907B68FA7883F8322000BF0C37BD465DF801
S3150802D3A0047B704780B483B000AF78607B6893F8DB
S3150802D3B03230012B01D1012307E07B6893F8323022
S3150802D3C0022B01D1022300E0002318460C37BD4682
S3150802D3D05DF8047B704780B483B000AF78600B4673
S3150802D3E0FB707B68FA7883F8332000BF0C37BD469A
S3150802D3F05DF8047B704780B483B000AF78607B68C1
S3150802D40093F83330012B01D1012307E07B6893F8A7
S3150802D4103330022B01D1022300E0002318460C37D1
S3150802D420BD465DF8047B704780B582B000AF012126
S3150802D43040480FF0B3FA0346012B14BF0123002319
S3150802D440DBB2BB710023FB713B4B1B78BA799A425C
S3150802D4501BD13A4B1B78632B02D9BB79FB7128E0A7
S3150802D460364B1B780133DAB2344B1A70FEF738FAA8
S3150802D47003461846FFF796FF0346012B02D10123FE
S3150802D480FB7116E00023FB7113E02B4ABB7913707C
S3150802D4902A4B00221A70FEF723FA03461846FFF7AC
S3150802D4A081FF0346012B02D10123FB7101E0002310
S3150802D4B0FB71FB79002B1CD0FEF712FA03460121F9
S3150802D4C01846FFF75FFF1E4B1B78FA799A422CD053
S3150802D4D00AF034FE0346042118460AF026FF0346DC
S3150802D4E0002B02D017480DF0EDF9154AFB79137097
S3150802D4F01BE0FEF7F5F9034602211846FFF742FF3D
S3150802D5000F4B1B78FA799A420FD00AF017FE034698
S3150802D510042118460AF009FF0346002B02D00A48DE
S3150802D5200DF0D0F9064AFB79137000BF0837BD46DD
S3150802D53080BD00BF00140242EBD30020ECD30020CA
S3150802D540EDD30020008505083885050880B582B028
S3150802D55000AF202140480FF021FA0346012B14BFE1
S3150802D56001230023DBB2BB710023FB713B4B1B7803
S3150802D570BA799A421BD13A4B1B78632B02D9BB79EB
S3150802D580FB7128E0364B1B780133DAB2344B1A703A
S3150802D590FEF7A6F903461846FFF72DFF0346012BA9
S3150802D5A002D10123FB7116E00023FB7113E02B4A1B
S3150802D5B0BB7913702A4B00221A70FEF791F90346BB
S3150802D5C01846FFF718FF0346012B02D10123FB7108
S3150802D5D001E00023FB71FB79002B1CD0FEF780F9D2
S3150802D5E0034601211846FFF7F6FE1E4B1B78FA7909
S3150802D5F09A422CD00AF0A2FD0346042118460AF0E4
S3150802D60094FE0346002B02D017480DF05BF9154A23
S3150802D610FB7913701BE0FEF763F9034602211846ED
S3150802D620FFF7D9FE0F4B1B78FA799A420FD00AF008
S3150802D63085FD0346042118460AF077FE0346002BA9
S3150802D64002D00A480DF03EF9064AFB79137000BF6C
S3150802D6500837BD4680BD00BF00140242EED3002043
S3150802D660EFD30020F0D30020008505083885050889
S3150802D67080B483B000AF78607B681B7818460C3795
S3150802D680BD465DF8047B704780B483B000AF78600E
S3150802D6900B46FB707B68FA781A7000BF0C37BD46DA
S3150802D6A05DF8047B704780B483B000AF78607B680E
S3150802D6B05B7818460C37BD465DF8047B704780B424
S3150802D6C083B000AF78600B46FB707B68FA785A70B5
S3150802D6D000BF0C37BD465DF8047B704780B483B043
S3150802D6E000AF78607B681B7818460C37BD465DF834
S3150802D6F0047B704780B483B000AF78600B46FB703A
S3150802D7007B68FA781A7000BF0C37BD465DF8047B51
S3150802D710704780B483B000AF78607B685B78184640
S3150802D7200C37BD465DF8047B704780B483B000AF02
S3150802D73078600B46FB707B68FA785A7000BF0C3724
S3150802D740BD465DF8047B704780B483B000AF78604D
S3150802D7507B681B7818460C37BD465DF8047B704714
S3150802D76080B483B000AF78600B46FB707B68FA78AA
S3150802D7701A7000BF0C37BD465DF8047B704780B44B
S3150802D78083B000AF78607B685B7818460C37BD4675
S3150802D7905DF8047B704780B483B000AF78600B46AF
S3150802D7A0FB707B68FA785A7000BF0C37BD465DF885
S3150802D7B0047B704780B483B000AF78607B681B78BF
S3150802D7C018460C37BD465DF8047B704780B483B0B3
S3150802D7D000AF78600B46FB707B68FA781A7000BF58
S3150802D7E00C37BD465DF8047B704780B483B000AF42
S3150802D7F078607B685B7818460C37BD465DF8047B13
S3150802D800704780B483B000AF78600B46FB707B68C4
S3150802D810FA785A7000BF0C37BD465DF8047B70472C
S3150802D82080B483B000AF78607B689B7818460C3763
S3150802D830BD465DF8047B704780B483B000AF78605C
S3150802D8400B46FB707B68FA789A7000BF0C37BD46A8
S3150802D8505DF8047B704780B483B000AF78607B685C
S3150802D8601B7818460C37BD465DF8047B704780B4B2
S3150802D87083B000AF78600B46FB707B68FA781A7043
S3150802D88000BF0C37BD465DF8047B704780B483B091
S3150802D89000AF78607B685B7818460C37BD465DF842
S3150802D8A0047B704780B483B000AF78600B46FB7088
S3150802D8B07B68FA785A7000BF0C37BD465DF8047B60
S3150802D8C0704780B483B000AF78607B681B781846CF
S3150802D8D00C37BD465DF8047B704780B483B000AF51
S3150802D8E078600B46FB707B68FA781A7000BF0C37B3
S3150802D8F0BD465DF8047B704780B483B000AF78609C
S3150802D9007B685B7818460C37BD465DF8047B704722
S3150802D91080B483B000AF78600B46FB707B68FA78F8
S3150802D9205A7000BF0C37BD465DF8047B704780B459
S3150802D93083B000AF78600B46FB707B6802337A6867
S3150802D94012881344FA781A707B681B8801339AB2D4
S3150802D9507B681A807B681B88DBB218460C37BD4683
S3150802D9605DF8047B704780B582B000AF7860396095
S3150802D9704FF481720021386823F0F8FD6021386877
S3150802D980FFF7D5FF7868FFF773FE0346194638682E
S3150802D990FFF7CDFF7868FFF786FE03461946386813
S3150802D9A0FFF7C5FF3B681B88DBB218460837BD463A
S3150802D9B080BD80B584B000AF786039600023FB7300
S3150802D9C002220021386823F0D1FDFB7B5A1CFA7328
S3150802D9D01A467B6813441B7819463868FFF754FEC3
S3150802D9E0FB7B5A1CFA731A467B6813441B78194642
S3150802D9F03868FFF764FEFB7B18461037BD4680BDC4
S3150802DA0080B582B000AF786039604FF48172002128
S3150802DA10386823F0ABFD60213868FFF788FF3B685A
S3150802DA201B88DBB218460837BD4680BD80B582B072
S3150802DA3000AF786039604FF481720021386823F0AC
S3150802DA4095FD61213868FFF772FF7868FFF746FE91
S3150802DA50034619463868FFF76AFF7868FFF759FEE2
S3150802DA60034619463868FFF762FF3B681B88DBB234
S3150802DA7018460837BD4680BD80B584B000AF7860C9
S3150802DA8039600023FB7302220021386823F06EFDF9
S3150802DA90FB7B5A1CFA731A467B6813441B78194691
S3150802DAA03868FFF727FEFB7B5A1CFA731A467B680F
S3150802DAB013441B7819463868FFF737FEFB7B18466E
S3150802DAC01037BD4680BD80B582B000AF7860396038
S3150802DAD04FF481720021386823F048FD61213868C5
S3150802DAE0FFF725FF3B681B88DBB218460837BD4699
S3150802DAF080BD80B582B000AF786039604FF481721C
S3150802DB000021386823F032FD62213868FFF70FFFDB
S3150802DB107868FFF719FE034619463868FFF707FFC4
S3150802DB207868FFF72CFE034619463868FFF7FFFEAA
S3150802DB303B681B88DBB218460837BD4680BD80B5F0
S3150802DB4084B000AF786039600023FB73022200219B
S3150802DB50386823F00BFDFB7B5A1CFA731A467B685E
S3150802DB6013441B7819463868FFF7FAFDFB7B5A1CE3
S3150802DB70FA731A467B6813441B7819463868FFF706
S3150802DB800AFEFB7B18461037BD4680BD80B582B0BB
S3150802DB9000AF786039604FF481720021386823F04B
S3150802DBA0E5FC62213868FFF7C2FE3B681B88DBB2D8
S3150802DBB018460837BD4680BD80B582B000AF78608A
S3150802DBC039604FF481720021386823F0CFFC702146
S3150802DBD03868FFF7ACFE7868FFF7ECFD034619468E
S3150802DBE03868FFF7A4FE7868FFF7FFFD0346194673
S3150802DBF03868FFF79CFE7868FFF712FE0346194657
S3150802DC003868FFF794FE3B681B88DBB2184608376C
S3150802DC10BD4680BD80B584B000AF78603960002308
S3150802DC20FB7303220021386823F0A0FCFB7B5A1CF5
S3150802DC30FA731A467B6813441B7819463868FFF745
S3150802DC40C5FDFB7B5A1CFA731A467B6813441B787C
S3150802DC5019463868FFF7D5FDFB7B5A1CFA731A4634
S3150802DC607B6813441B7819463868FFF7E5FDFB7B8A
S3150802DC7018461037BD4680BD80B582B000AF7860C1
S3150802DC8039604FF481720021386823F06FFC7021E5
S3150802DC903868FFF74CFE3B681B88DBB21846083724
S3150802DCA0BD4680BD80B582B000AF786039604FF45A
S3150802DCB081720021386823F059FC71213868FFF710
S3150802DCC036FE7868FFF7C7FD034619463868FFF738
S3150802DCD02EFE7868FFF7DAFD034619463868FFF71D
S3150802DCE026FE3B681B88DBB218460837BD4680BD50
S3150802DCF080B584B000AF786039600023FB730222D6
S3150802DD000021386823F032FCFB7B5A1CFA731A4648
S3150802DD107B6813441B7819463868FFF7A8FDFB7B16
S3150802DD205A1CFA731A467B6813441B7819463868D4
S3150802DD30FFF7B8FDFB7B18461037BD4680BD80B598
S3150802DD4082B000AF786039604FF48172002138687A
S3150802DD5023F00CFC71213868FFF7E9FD3B681B8844
S3150802DD60DBB218460837BD4680BD80B582B000AF23
S3150802DD70786039604FF481720021386823F0F6FB27
S3150802DD8072213868FFF7D3FD7868FFF79AFD0346D4
S3150802DD9019463868FFF7CBFD7868FFF7ADFD0346ED
S3150802DDA019463868FFF7C3FD3B681B88DBB218467D
S3150802DDB00837BD4680BD80B584B000AF786039604B
S3150802DDC00023FB7302220021386823F0CFFBFB7B7A
S3150802DDD05A1CFA731A467B6813441B781946386824
S3150802DDE0FFF77BFDFB7B5A1CFA731A467B681344C2
S3150802DDF01B7819463868FFF78BFDFB7B18461037E8
S3150802DE00BD4680BD80B582B000AF786039604FF4F8
S3150802DE1081720021386823F0A9FB72213868FFF75E
S3150802DE2086FD3B681B88DBB218460837BD4680BDAF
S3150802DE3080B582B000AF78600B467B800D481BF038
S3150802DE404FFA02467B889A420FD34FF0FF310A48AF
S3150802DE501AF066FC7B881A46796806481BF029FC84
S3150802DE6005481AF09FFC012300E0002318460837EC
S3150802DE70BD4680BDF4D3002084A5002080B5C4B079
S3150802DE8000AF024607F58873A3F209131A70002336
S3150802DE9087F80F314AE007F10C034FF4807200212C
S3150802DEA0184623F063FB4FF0FF3129481AF038FC75
S3150802DEB007F10C03194627481BF072FC034687F83C
S3150802DEC00F3123481AF06EFC4FF0FF3120481AF042
S3150802DED027FC07F10C0319461E481BF0FBFB0346F9
S3150802DEE087F80F311A481AF05DFC4FF47A711A480E
S3150802DEF01AF016FC0346002B0DD1F7F720F897F80F
S3150802DF000F319AB207F10C031946F7F706FA1248C7
S3150802DF101AF048FC02E011480CF0D4FC07F58873A5
S3150802DF20A3F209131B7818460CF00AFE09481BF0DF
S3150802DF3035FA034683F00103DBB2002B03D0084B04
S3150802DF401B78002BA7D000BF07F58877BD4680BD92
S3150802DF5084A50020F4D30020A0A50020F492050889
S3150802DF6004D5002080B483B000AF78600B467B806E
S3150802DF7000BF00BF0C37BD465DF8047B7047000042
S3150802DF8080B582B000AF0023FB712D4B1B78002BA6
S3150802DF904ED02C4B1B780133DAB22A4B1A70294B16
S3150802DFA01B78092B47D9274B00221A70244B5B781A
S3150802DFB0012B1FD8224B5B780133DAB2204B5A70F9
S3150802DFC04FF47A7120481AF0ABFB0346002B0DD1A9
S3150802DFD0F6F7B5FF03461A4A92F883201B491846F4
S3150802DFE0F7F79BF918481AF0DDFB24E018480CF0FD
S3150802DFF069FC20E00023FB7102E0FB790133FB7127
S3150802E0000F4B93F88330FA799A42F6D34FF0FF31E1
S3150802E01010481AF085FB0D490F481BF05BFB0D48AB
S3150802E0201AF0C0FB84220021054823F09FFA02E079
S3150802E030044B00221A7000BF0837BD4680BD00BFD8
S3150802E04004D5002088D50020A0A5002007D50020E9
S3150802E050F492050884A50020F4D3002080B500AF09
S3150802E0604FF48072024903481BF00EF900BF80BDC7
S3150802E07004D40020F4D3002080B500AFFFF7EEFFEA
S3150802E08000BF80BD80B582B000AF786039603B685A
S3150802E090DBB21946786800F04BF800BF0837BD4670
S3150802E0A080BD80B582B000AF786039603B689BB2AC
S3150802E0B019467868FFF7BCFE00BF0837BD4680BD23
S3150802E0C080B582B000AF78603960064B1B683A6843
S3150802E0D092B2796818461AF0D1FE00BF0837BD46D3
S3150802E0E080BD00BF9016002080B582B000AF786070
S3150802E0F03960054B1B683A68796818461AF058FF62
S3150802E10000BF0837BD4680BD9016002080B500AF17
S3150802E110044B1868044B054A00211AF074FE00BF26
S3150802E12080BD00BF90160020A3E0020885E0020821
S3150802E130B0B584B000AF78600B46FB7009F0FEFFFD
S3150802E140F860FB789BB219467868FFF70BFF7B6885
S3150802E1501B78013B712B00F2068501A252F823F0C7
S3150802E16029E3020867EB020867EB020867EB020875
S3150802E17075E3020867EB020867EB020867EB020819
S3150802E18067EB020867EB020867EB020867EB02080F
S3150802E19067EB020867EB02084DE3020867EB020821
S3150802E1A067EB020867EB020867EB020867EB0208EF
S3150802E1B067EB020867EB020867EB020867EB0208DF
S3150802E1C067EB020867EB020867EB020867EB0208CF
S3150802E1D067EB020867EB020867EB020867EB0208BF
S3150802E1E0A1E3020879E4020845E5020867EB02089A
S3150802E1F067EB020867EB020867EB02084DE50208BF
S3150802E20095E5020867EB020867EB020867EB020866
S3150802E21067EB020867EB020867EB020867EB02087E
S3150802E22067EB020867EB020867EB020867EB02086E
S3150802E23067EB020867EB020867EB020867EB02085E
S3150802E24067EB020867EB020867EB020867EB02084E
S3150802E25067EB020867EB020867EB020867EB02083E
S3150802E26067EB020867EB020867EB020867EB02082E
S3150802E27067EB020867EB020867EB020867EB02081E
S3150802E28067EB020867EB020867EB020867EB02080E
S3150802E29067EB020867EB020867EB020867EB0208FE
S3150802E2A067EB020867EB020867EB020867EB0208EE
S3150802E2B067EB020867EB020867EB020867EB0208DE
S3150802E2C067EB020867EB020867EB020867EB0208CE
S3150802E2D067EB020867EB020867EB02089DE502088E
S3150802E2E0CFE60208A7E7020867EB020867EB02080F
S3150802E2F067EB020867EB020867EB020867EB02089E
S3150802E30067EB020867EB020867EB020867EB02088D
S3150802E31067EB020867EB020867EB02087FE8020868
S3150802E32061E902088FEA0208C549C6481EF035FBAC
S3150802E330C3481EF080FB0446C1481EF088FB03460C
S3150802E34019462046FFF7BCFE00F00EBCBE4B012262
S3150802E3501A70BB49BC481EF043FBB9481EF06BFB5A
S3150802E3600446B7481EF073FB034619462046FFF7D4
S3150802E370A7FEF9E3B5480CF0A5FAF86809F04AFFD2
S3150802E380AF481EF046FBAE481EF055FB0446AC48A5
S3150802E3901EF05DFB034619462046FFF791FEE3E3AE
S3150802E3A0AB480CF08FFA7B680133AA4918461AF073
S3150802E3B07FFC1AF069FB034618461AF092FB0346DD
S3150802E3C01C46A4481AF0C6FB03469C4211D1A14832
S3150802E3D01AF0C0FB03461C461AF056FB03461846BB
S3150802E3E01AF07FFB03461A4621469B480CF06AFA46
S3150802E3F031E098481AF0AEFB96481AF0ABFB034692
S3150802E4000F2B1ED893481AF0A5FB03461C469148C3
S3150802E4101AF0BBFB03461A46214690480CF052FAFC
S3150802E4201AF032FB04468B481AF094FB0346194647
S3150802E43020461AF062FBFB7819467868FAF728F93B
S3150802E44009E084481AF086FB034619460F23002280
S3150802E45083480CF037FA7A497E481AF050FC784815
S3150802E4601EF0E9FA044676481EF0F1FA0346194602
S3150802E4702046FFF725FE77E37A480CF023FA7B68F5
S3150802E4800133794918461AF06EFC1AF0FDFA03466A
S3150802E49018461AF026FB03461C4673481AF090FBE8
S3150802E4A003469C4211D170481AF08AFB03461C4661
S3150802E4B01AF0EAFA034618461AF013FB03461A46F6
S3150802E4C021466A480CF0FEF92BE067481AF078FBF9
S3150802E4D065481AF075FB03460F2B18D862481AF0DE
S3150802E4E06FFB0346194662480CF0ECF91AF0CCFAAF
S3150802E4F004465D481AF064FB0346194620461AF09C
S3150802E500FCFAFB7819467868FAF7C2F809E0564821
S3150802E5101AF056FB034619460F23002255480CF0FB
S3150802E520D1F9474950481AF03AFC45481EF083FA91
S3150802E530044643481EF08BFA034619462046FFF75F
S3150802E540BFFD11E34C480CF0BDF90DE34B480CF046
S3150802E550B9F9012200214A4823F008F81AF094FA78
S3150802E560034618461AF0BDFA0346194644481AF0F5
S3150802E5704EFB334942481AF028FC31481EF05BFA32
S3150802E58004462F481EF063FA034619462046FFF74B
S3150802E59097FDE9E23B480CF095F9E5E23A480CF0BA
S3150802E5A091F97B68013339491846FFF702FA1AF0DE
S3150802E5B06BFA034618461AF094FA03461C46334881
S3150802E5C0FFF756F803469C4211D13048FFF750F838
S3150802E5D003461C461AF058FA034618461AF081FAF8
S3150802E5E003461A4621462A480CF06CF95EE027488B
S3150802E5F0FFF73EF82548FFF73BF803460F2B4BD8A3
S3150802E6002248FFF735F803461C462048FFF74BF821
S3150802E61003461A4621461F480CF054F91AF034FAF2
S3150802E62004461A48FFF724F80346194620461AF004
S3150802E63064FAFB7819467868FAF72AF836E000BFD2
S3150802E640B8E50020C0E60020BCE6002014930508C1
S3150802E65030930508C4E600204C930508789305080C
S3150802E660A8930508D8930508C8E60020F893050874
S3150802E670289405085094050884940508A09405086A
S3150802E680CCE60020BC940508DC940508D0E60020F8
S3150802E690FC94050828950508C648FEF7E9FF0346CF
S3150802E6A019460F230022C4480CF00CF9C349C14885
S3150802E6B0FFF7A6F9C1481EF0BEF90446BF481EF088
S3150802E6C0C6F9034619462046FFF7FAFC4CE2BC484F
S3150802E6D00CF0F8F87B680133BA491846FFF7CCF90B
S3150802E6E01AF0D2F9034618461AF0FBF903461C46F5
S3150802E6F0B448FEF7F3FF03469C4211D1B148FEF730
S3150802E700EDFF03461C461AF0BFF9034618461AF0EF
S3150802E710E8F903461A462146AB480CF0D3F831E02D
S3150802E720A848FEF7DBFFA748FEF7D8FF03460F2BDC
S3150802E7301ED8A448FEF7D2FF03461C46A148FEF798
S3150802E740E8FF03461A462146A0480CF0BBF81AF021
S3150802E7509BF904469B48FEF7C1FF03461946204625
S3150802E7601AF0CBF9FB7819467868F9F791FF09E0B0
S3150802E7709448FEF7B3FF034619460F23002294482E
S3150802E7800CF0A0F88D498F48FFF79DF98B481EF0CB
S3150802E79052F9044689481EF05AF903461946204694
S3150802E7A0FFF78EFCE0E18B480CF08CF87B680133AE
S3150802E7B089491846FFF7C3F91AF066F90346184657
S3150802E7C01AF08FF903461C468348FEF7BDFF034637
S3150802E7D09C4211D18048FEF7B7FF03461C461AF041
S3150802E7E053F9034618461AF07CF903461A46214697
S3150802E7F07A480CF067F831E07748FEF7A5FF7648C5
S3150802E800FEF7A2FF03460F2B1ED87348FEF79CFF9E
S3150802E81003461C467048FEF7B2FF03461A462146CF
S3150802E8206F480CF04FF81AF02FF904466A48FEF7BB
S3150802E8308BFF0346194620461AF05FF9FB781946FC
S3150802E8407868F9F725FF09E06348FEF77DFF034676
S3150802E85019460F23002263480CF034F857495E48DC
S3150802E860FFF794F955481EF0E6F8044653481EF099
S3150802E870EEF8034619462046FFF722FC74E15A4889
S3150802E8800CF020F87B68013358491846FFF7C2F99D
S3150802E8901AF0FAF8034618461AF023F903461C46F4
S3150802E8A05248FEF787FF03469C4211D14F48FEF7AE
S3150802E8B081FF03461C461AF0E7F8034618461AF083
S3150802E8C010F903461A46214649480BF0FBFF36E083
S3150802E8D04648FEF76FFF4548FEF76CFF03460F2BC7
S3150802E8E023D84248FEF766FF03461C463F48FEF712
S3150802E8F07CFF03461D463D48FEF792FF03462A461D
S3150802E90021463C480BF0DEFF1AF0BEF804463748AB
S3150802E910FEF750FF0346194620461AF0EEF8FB7832
S3150802E92019467868F9F7B4FE09E03048FEF742FF5F
S3150802E930034619460F2300222F480BF0C3FF1F492F
S3150802E9402A48FFF799F91D481EF075F804461B4830
S3150802E9501EF07DF8034619462046FFF7B1FB03E190
S3150802E96026480BF0AFFF7B68013325491846FFF7A7
S3150802E970BFF91AF089F8034618461AF0B2F80346A0
S3150802E9801C461F48FEF767FF03469C423CD11C48BB
S3150802E990FEF761FF03461C461AF076F80346184648
S3150802E9A01AF09FF803461A46214616480BF08AFFC4
S3150802E9B05CE000BFD0E6002058950508B8E50020BF
S3150802E9C08C950508D4E60020AC950508D895050867
S3150802E9D0089605083C960508D8E6002060960508BC
S3150802E9E090960508C4960508FC960508DCE60020FC
S3150802E9F01C970508489705087C970508B0970508E7
S3150802EA00E0E60020D09705085948FEF724FF584843
S3150802EA10FEF721FF03460F2B1ED85548FEF71BFFAC
S3150802EA2003461C465248FEF731FF03461A4621465C
S3150802EA3050480BF047FF1AF027F804464C48FEF7F1
S3150802EA400AFF0346194620461AF057F8FB78194674
S3150802EA507868F9F71DFE09E04548FEF7FCFE03460D
S3150802EA6019460F23002244480BF02CFF434940481D
S3150802EA70FFF765F941481DF0DEFF04463F481DF0E1
S3150802EA80E6FF034619462046FFF71AFB6CE03C48A8
S3150802EA900BF018FF7B6801333A491846FFF78BF9E2
S3150802EAA019F0F2FF034618461AF01BF803461C46ED
S3150802EAB03448FEF706FF03469C4211D13148FEF759
S3150802EAC000FF03461C4619F0DFFF034618461AF0F4
S3150802EAD008F803461A4621462B480BF0F3FE31E0A6
S3150802EAE02848FEF7EEFE2748FEF7EBFE03460F2BF5
S3150802EAF01ED82448FEF7E5FE03461C462148FEF7C3
S3150802EB00FBFE03461A46214620480BF0DBFE19F0A7
S3150802EB10BBFF04461B48FEF7D4FE034619462046A9
S3150802EB2019F0EBFFFB7819467868F9F7B1FD09E0A9
S3150802EB301448FEF7C6FE034619460F230022144858
S3150802EB400BF0C0FE0D490F48FFF75CF90B481DF0A4
S3150802EB5072FF044609481DF07AFF03461946204605
S3150802EB60FFF7AEFA00E000BF00BF1037BD46B0BDE2
S3150802EB70E0E60020FC9705082C980508B8E5002071
S3150802EB8060980508E4E6002084980508B498050804
S3150802EB90E898050880B500AF224BD3F8F430002B6D
S3150802EBA003DA21480BF08EFE39E01E4BD3F8F43017
S3150802EBB003F08043002B03D01C480BF083FE2EE0A3
S3150802EBC0184BD3F8F43003F00053002B03D018483F
S3150802EBD00BF078FE23E0134BD3F8F43003F080539E
S3150802EBE0002B03D013480BF06DFE18E00D4BD3F83B
S3150802EBF0F43003F00063002B03D00F480BF062FEDB
S3150802EC000DE0084BD3F8F43003F08063002B03D0F1
S3150802EC100A480BF057FE02E009480BF053FE00BF04
S3150802EC2080BD00BF000C0244209905083C990508DE
S3150802EC30589905087499050894990508AC99050820
S3150802EC40C499050880B500AF034815F0EBFF0248E2
S3150802EC5015F0A8FE00BF80BDDCE8002080B500AF35
S3150802EC6000F07AFB0BF01EFE00BF80BD80B500AF38
S3150802EC70264B274A9A6062B600BF0CF07BF800F072
S3150802EC8057F800F0B5FB00F005F900F025F900F099
S3150802EC90B9F800F029F900F0E3F900F045FA00F0B6
S3150802ECA05BFB00F0BDFA00F009FB09F047FA1948C8
S3150802ECB0F6F73EF80BF0F6FDFFF728FA00F04AFEE3
S3150802ECC020F0F6FB0BF080FE134813F0CBFF134837
S3150802ECD013F0C8FF01224FF4004111480DF076FEE9
S3150802ECE0012201210F480DF071FE02F03DF90821BB
S3150802ECF00D4814F01DFA04210B4814F019FA0B48B2
S3150802ED000BF0E0FDF5F7A2FB00BFFDE700ED00E022
S3150802ED1000000208E8E6002044E8002090E8002007
S3150802ED200004024200100242ACE70020E0990508FE
S3150802ED3080B59CB000AF07F1200350220021184687
S3150802ED4022F014FC07F1080300221A605A609A603E
S3150802ED50DA601A615A612A4B1B69294A43F0300361
S3150802ED601361274B1B6903F030037B607B6800BF86
S3150802ED70234B5B6903F00803082BF9D109233B628D
S3150802ED804FF480337B624FF08063BB630223BB641C
S3150802ED900323FB6403233B657D237B650223BB6553
S3150802EDA00223FB6502233B6608237B660023BB66B8
S3150802EDB00023FB6607F1200318460DF0F7FE03460B
S3150802EDC0002B01D000F060FC1F23BB600323FB600D
S3150802EDD000233B6100237B610023BB610023FB61A7
S3150802EDE007F10803052118460EF018FB0346002B07
S3150802EDF001D000F049FC00BF7037BD4680BD00BF98
S3150802EE000008024480B500AF204B214A1A601F4B06
S3150802EE1000225A601D4B4FF440729A601B4B002227
S3150802EE20DA601A4B00221A74184B00225A74174BCE
S3150802EE3000229A74154B05225A61144B0A229A61CA
S3150802EE40124B2722DA61114B0A221A620F4B05224C
S3150802EE505A620E4B02229A620C4B0722DA620B4B5B
S3150802EE6002221A63094B01225A63084B01229A634A
S3150802EE70064B0022DA6305480CF07AF90346002BA2
S3150802EE8001D000F001FC00BF80BD00BFE8E600200B
S3150802EE9000A4004080B500AF0D4B0E4A1A600C4B19
S3150802EEA005225A600A4B40F2ED22DA60084B40F21C
S3150802EEB0ED229A60064B00221A6105480DF0DEFD26
S3150802EEC00346002B01D000F0DFFB00BF80BD00BF68
S3150802EED04CE700200030004080B400AF00BFBD46BA
S3150802EEE05DF8047B7047000080B59CB000AF07F15F
S3150802EEF0600300221A605A609A60DA6007F15403C6
S3150802EF0000221A605A609A6007F1380300221A60D2
S3150802EF105A609A60DA601A615A619A613B1D342214
S3150802EF200021184622F022FB4B4B4C4A1A604A4BE8
S3150802EF3046F2A7125A60484B00229A60464B632251
S3150802EF40DA60454B00221A61434B00225A61424B52
S3150802EF5000229A61404813F02DFE0346002B01D089
S3150802EF6000F092FB4FF480533B6607F160031946A3
S3150802EF70394814F0F3FB0346002B01D000F084FB5A
S3150802EF80354813F01DFF0346002B01D000F07CFB29
S3150802EF9000237B650023BB650023FB6507F1540349
S3150802EFA019462D4815F0D6FA0346002B01D000F073
S3150802EFB06BFB6023BB630023FB6300233B640023D4
S3150802EFC07B640023BB640023FB6400233B6507F1D3
S3150802EFD0380308221946204814F0ACFA0346002BD7
S3150802EFE001D000F051FB07F138030C2219461A48E2
S3150802EFF014F0A0FA0346002B01D000F045FB0023CB
S3150802F0007B600023BB600023FB6000233B61002377
S3150802F0107B614FF40053BB610023FB6100233B6213
S3150802F02000237B624FF00073BB620023FB6200235E
S3150802F0303B6300237B633B1D1946074815F05AFBC1
S3150802F0400346002B01D000F01FFB034808F012FC10
S3150802F05000BF7037BD4680BD60E70020002C014026
S3150802F06080B58AB000AF07F11C0300221A605A6005
S3150802F0709A603B4600221A605A609A60DA601A6100
S3150802F0805A619A61274B4FF080421A60254B46F225
S3150802F090A7125A60234B00229A60224B6322DA6037
S3150802F0A0204B00221A611F4B00229A611D4813F059
S3150802F0B087FE0346002B01D000F0E6FA0023FB6127
S3150802F0C000237B6207F11C031946164815F042FA1B
S3150802F0D00346002B01D000F0D7FA60233B600023D9
S3150802F0E07B600023BB6000233B613B460422194632
S3150802F0F00C4814F01FFA0346002B01D000F0C4FA9C
S3150802F1003B4608221946074814F014FA0346002B10
S3150802F11001D000F0B9FA034808F0ACFB00BF283763
S3150802F120BD4680BDACE7002080B58AB000AF07F1C6
S3150802F1301C0300221A605A609A603B4600221A6033
S3150802F1405A609A60DA601A615A619A61324B334A96
S3150802F1501A60314B46F2A7125A602F4B00229A6068
S3150802F1602D4B6322DA602C4B00221A612A4B0022AD
S3150802F1709A61294813F024FE0346002B01D000F0B9
S3150802F18083FA0023FB6100237B6207F11C031946FD
S3150802F190214815F0DFF90346002B01D000F074FA76
S3150802F1A060233B6000237B600023BB6000233B6136
S3150802F1B03B4600221946184814F0BCF90346002BB0
S3150802F1C001D000F061FA3B4604221946124814F0AF
S3150802F1D0B1F90346002B01D000F056FA3B46082245
S3150802F1E019460D4814F0A6F90346002B01D000F083
S3150802F1F04BFA3B460C221946074814F09BF903467C
S3150802F200002B01D000F040FA034808F033FB00BF98
S3150802F2102837BD4680BD00BFF8E70020000400403D
S3150802F22080B588B000AF07F1100300221A605A6051
S3150802F2309A60DA603B1D00221A605A609A601D4B7A
S3150802F2401D4A1A601B4B40F6C3125A60194B00221C
S3150802F2509A60184B6322DA60164B00221A61154B24
S3150802F26000229A61134813F0A5FC0346002B01D02D
S3150802F27000F00AFA4FF480533B6107F1100319466E
S3150802F2800C4814F06BFA0346002B01D000F0FCF987
S3150802F29000237B600023FB603B1D1946054815F0D9
S3150802F2A059F90346002B01D000F0EEF900BF2037CA
S3150802F2B0BD4680BD44E800200008004080B588B0FD
S3150802F2C000AF07F1100300221A605A609A60DA60EA
S3150802F2D03B1D00221A605A609A601D4B1D4A1A602D
S3150802F2E01B4B40F6C3125A60194B00229A60184B00
S3150802F2F06322DA60164B00221A61154B00229A61C4
S3150802F300134813F057FC0346002B01D000F0BCF952
S3150802F3104FF480533B6107F1100319460C4814F069
S3150802F3201DFA0346002B01D000F0AEF900237B60DC
S3150802F3300023FB603B1D1946054815F00BF90346E9
S3150802F340002B01D000F0A0F900BF2037BD4680BDD2
S3150802F35090E80020000C004080B500AF224B234AFB
S3150802F3601A60214B4FF4E1325A601F4B00229A6011
S3150802F3701D4B0022DA601C4B00221A611A4B0C2222
S3150802F3805A61194B00229A61174B0022DA61164B11
S3150802F39000221A62144B00225A62134B00229A6206
S3150802F3A0114815F0AFFA0346002B01D000F06CF9AC
S3150802F3B000210D4817F01FFB0346002B01D000F071
S3150802F3C063F90021084817F054FB0346002B01D0C5
S3150802F3D000F05AF9044817F0D5FA0346002B01D073
S3150802F3E000F052F900BF80BDDCE800200038014079
S3150802F3F080B58EB000AF07F1240300221A605A6066
S3150802F4009A60DA601A61854BD3F88C30834A43F0E6
S3150802F4101003C2F88C30814BD3F88C3003F01003FA
S3150802F4203B623B6A7D4BD3F88C307C4A43F020031F
S3150802F430C2F88C30794BD3F88C3003F02003FB6189
S3150802F440FB69764BD3F88C30744A43F08003C2F8D2
S3150802F4508C30724BD3F88C3003F08003BB61BB69E6
S3150802F4606E4BD3F88C306D4A43F00403C2F88C30E5
S3150802F4706A4BD3F88C3003F004037B617B69674BD4
S3150802F480D3F88C30654A43F00103C2F88C30634BDB
S3150802F490D3F88C3003F001033B613B695F4BD3F829
S3150802F4A08C305E4A43F00203C2F88C305B4BD3F8C9
S3150802F4B08C3003F00203FB60FB68584BD3F88C30A0
S3150802F4C0564A43F00803C2F88C30544BD3F88C30B2
S3150802F4D003F00803BB60BB68504BD3F88C304F4A25
S3150802F4E043F04003C2F88C304C4BD3F88C3003F00F
S3150802F4F040037B607B6800224FF4004148480DF0C8
S3150802F50065FA00224FF4806146480DF05FFA002240
S3150802F510012145480DF05AFA41F27C037B62002329
S3150802F520BB620023FB6207F1240319463E480DF02D
S3150802F53027F83F237B620023BB620023FB6207F1A5
S3150802F5402403194639480DF01BF802237B62384B0F
S3150802F550BB620023FB6207F12403194635480DF006
S3150802F5600FF824237B620023BB620023FB6207F1A8
S3150802F570240319462F480DF003F821237B62002342
S3150802F580BB620023FB6207F1240319462A480CF0E2
S3150802F590F7FF4FF400437B620123BB620023FB6241
S3150802F5A000233B6307F1240319461D480CF0E8FFC4
S3150802F5B04FF4F8537B620023BB620023FB6207F118
S3150802F5C0240319461D480CF0DBFF4FF480637B6267
S3150802F5D00123BB620023FB6200233B6307F124037A
S3150802F5E0194610480CF0CCFF01237B620123BB624B
S3150802F5F00023FB6200233B6307F1240319460A48EA
S3150802F6000CF0BEFF002200210C200BF0D5FC0C20CA
S3150802F6100BF0ECFC00BF3837BD4680BD000C024437
S3150802F620000402420018024200100242001402427A
S3150802F630000031100008024200000242000C024299
S3150802F64080B582B000AF78607B681B680B4A93422C
S3150802F65001D10BF0B5FB7B681B68094A934201D1BD
S3150802F660FCF7DAFC7B681B68064A934201D1FCF771
S3150802F67065FD00BF0837BD4680BD00BF00200040BB
S3150802F68000080040000C004080B400AF72B600BF0C
S3150802F69000BFFDE7B0B596B000AF786039600023C9
S3150802F6A07B6573E0764B774A402178680BF0DCFF7E
S3150802F6B00346002B03D074480BF004F966E0F5F70D
S3150802F6C01BFC0346002B03D06E4B1B687B6502E0CE
S3150802F6D06C4B1B687B65F5F729FC02467B6D9342EA
S3150802F6E004D168216748F5F7E1FA4FE01AF0A6F95E
S3150802F6F002467B6D93423BD01AF03EFA02467B6D78
S3150802F700934235D01AF042FA02467B6D93422FD0C5
S3150802F7101AF046FA02467B6D934229D01AF09CF9F2
S3150802F72002467B6D934223D01AF044FA02467B6D59
S3150802F73093421DD01AF0D0F902467B6D934217D038
S3150802F7401AF098F902467B6D934211D01AF076F9AF
S3150802F75002467B6D93420BD01AF0DAF902467B6DAC
S3150802F760934205D01AF0ECF902467B6D93420DD10D
S3150802F7701AF0E6F9434BDB681846F5F744FC0346EC
S3150802F780DBB21A463E49786D1FF0C8FE40217868FA
S3150802F7900CF0D8F80346002B84D17868F5F726FBD7
S3150802F7A003461A46394B9A607868F5F7E5FA03462E
S3150802F7B0364A13607868F5F7FAFA0346334A53600D
S3150802F7C0324B9B68002B12D0304B1A682F4B5B6862
S3150802F7D007F10C002E4921F035FE07F10C031846F5
S3150802F7E00BF070F8294B9B681846F5F753FB0C2269
S3150802F7F02649284821F0AAFE0346002B36D0234B79
S3150802F8001B68DAB207F15003114618461AF037F8A0
S3150802F8101E4B5B68DAB207F15003114618461AF016
S3150802F82049F81A4B9B68DAB207F150031146184693
S3150802F8301AF05BF807F10C0207F150031146184655
S3150802F8401AF095F81AF02EF9044607F10C03184631
S3150802F8501AF05AF8054607F10C0318461AF060F82A
S3150802F86003461A46294620461FF01EFF094B074A39
S3150802F87007CA83E8070000BF5837BD46B0BD00BFB8
S3150802F88098E9002070E90020F0990508B4C800201C
S3150802F890109A0508C0C8002080B58AB002AF786001
S3150802F8A00B467B8013463B800023BB600023FB602C
S3150802F8B07B683B6101237B617B88BB613B88FB617B
S3150802F8C007F10803194607480BF0ACFD012300931C
S3150802F8D001230222022103480BF0FEFD00BF203756
S3150802F8E0BD4680BDE8E6002080B58CB002AFF86060
S3150802F8F0B9607A604FF080433B6100237B61FB6805
S3150802F900BB610123FB61BB683B627B687B6207F1D3
S3150802F9101003194607480BF085FD012300930123BE
S3150802F9200222022103480BF0D7FD00BF2837BD4645
S3150802F93080BD00BFE8E6002080B500AF04480BF0A2
S3150802F940FCFD0022012102480CF01AF800BF80BD16
S3150802F950E8E6002080B500AFF5F7CEFA0346002B9D
S3150802F96009D0F5F7E3FA03461A466FF0604102201A
S3150802F970FFF7BAFF09E0F5F7D9FA03469BB21A462A
S3150802F9804FF6FF710220FFF787FFFFF7D5FF00BF8B
S3150802F99080BD000080B58EB000AFF860B96013462E
S3150802F9A0FB71FB79002B02D0FB79402B01D900238E
S3150802F9B03FE007F1140324220021184621F0D6FD60
S3150802F9C0FB687B61F5F798FA0346002B03D04FF0E4
S3150802F9D08043BB6101E00023BB610023FB61FB7925
S3150802F9E09BB21846F5F7B8FA03463B6200237B62D8
S3150802F9F04FF48013BB624FF40013FB6200233B6390
S3150802FA0000237B634FF47A710C4818F089FE03468B
S3150802FA10002B0AD107F11403BA6819460848F4F705
S3150802FA2071FE064818F0BEFE02E006480AF04AFFD2
S3150802FA30012318463837BD4680BD00BF30A50020D1
S3150802FA40E8E60020349A050880B590B000AFF8635E
S3150802FA5087ED0C0B87ED0A1B87ED082B87ED063B16
S3150802FA6087ED044B87ED025BB9637A603B60FB6BFB
S3150802FA70BA6B1A66FB6B7A68DA67FB6B012283F844
S3150802FA807920F96BD7E90223C1E90E2397ED041B06
S3150802FA9097ED060BF86B00F0F9F8012197ED082BA4
S3150802FAA097ED0A1B97ED0C0BF86B00F04BF83968CB
S3150802FAB0F86B00F056F9F96B4FF000024FF00003AD
S3150802FAC0C1E91623F96B4FF000024FF00003C1E9B2
S3150802FAD01423F96B4FF000024FF00003C1E910231B
S3150802FAE0F96B4FF000024FF00003C1E9122300BF81
S3150802FAF04037BD4680BD80B483B000AF7860796870
S3150802FB004FF000024FF00003C1E9162379684FF05F
S3150802FB1000024FF00003C1E9142379684FF000028E
S3150802FB204FF00003C1E9102379684FF000024FF045
S3150802FB300003C1E9122300BF0C37BD465DF8047BFA
S3150802FB407047000080B58AB000AFF86187ED040BF4
S3150802FB5087ED021B87ED002BB9614FF000024FF0CB
S3150802FB600003D7E90401F1F7E7F80346002B40F052
S3150802FB7086804FF000024FF00003D7E90201F1F741
S3150802FB80DBF80346002B7AD14FF000024FF0000350
S3150802FB90D7E90001F1F7D0F80346002B6FD1BB690C
S3150802FBA0012B0CBF01230023DAB2FB6983F8782004
S3150802FBB0F969D7E90423C1E90023F969D7E90223D8
S3150802FBC0C1E90223F969D7E90023C1E90423FB69DC
S3150802FBD01B6E1846F0F7C4FD4FF000022A4BF0F7E9
S3150802FBE063FF02460B46C7E90823F969D7E90423E6
S3150802FBF0C1E90623D7E90823D7E90201F0F72AFE65
S3150802FC0002460B46F969C1E90823D7E90823D7E969
S3150802FC100001F0F749FF02460B46F969C1E90A23D2
S3150802FC20FB691B6B012B2BD1FB69D3E906234FF02A
S3150802FC3000004FF00001F0F755FC02460B46F96941
S3150802FC40C1E90623FB69D3E908234FF000004FF008
S3150802FC500001F0F747FC02460B46F969C1E9082399
S3150802FC60FB69D3E90A234FF000004FF00001F0F7D1
S3150802FC7039FC02460B46F969C1E90A2300E000BFCE
S3150802FC802837BD4680BD00BF00408F4080B586B08C
S3150802FC9000AF786187ED020B87ED001BD7E90023D9
S3150802FCA0D7E90201F1F75CF80346002B55D17969C9
S3150802FCB0D7E90223C1E91A237969D7E90023C1E9F9
S3150802FCC01C237B6993F87930002B47D07B69D3E9EB
S3150802FCD012017B69D3E91C23F1F74CF80346002B82
S3150802FCE006D07B69D3E91C237969C1E9122310E09E
S3150802FCF07B69D3E912017B69D3E91A23F1F71CF868
S3150802FD000346002B05D07B69D3E91A237969C1E931
S3150802FD1012237B69D3E914017B69D3E91C23F1F722
S3150802FD2029F80346002B06D07B69D3E91C23796997
S3150802FD30C1E9142312E07B69D3E914017B69D3E98B
S3150802FD401A23F0F7F9FF0346002B07D07B69D3E99C
S3150802FD501A237969C1E9142300E000BF1837BD46A2
S3150802FD6080BD80B582B000AF786039607B6893F851
S3150802FD707930002B2ED07B681B6B3A689A4229D0C1
S3150802FD807B68D3E906234FF000004FF00001F0F735
S3150802FD90A9FB02460B467968C1E906237B68D3E9C3
S3150802FDA008234FF000004FF00001F0F79BFB0246D4
S3150802FDB00B467968C1E908237B68D3E90A234FF021
S3150802FDC000004FF00001F0F78DFB02460B467968FA
S3150802FDD0C1E90A237B683A681A6300BF0837BD4639
S3150802FDE080BDB0B58CB000AF78604FF000024FF01E
S3150802FDF00003C7E908234FF000024FF00003C7E9E2
S3150802FE0006234FF000024FF00003C7E904234FF020
S3150802FE1000024FF00003C7E90A237B68DB6FFB6029
S3150802FE207B6893F8793083F00103DBB2002B01D0AB
S3150802FE300023F0E07B681B6EFA689A42C0F0EA80FB
S3150802FE407B68D3E91023C7E908237B68D3E90E0147
S3150802FE50D7E90823F0F746FB02460B46C7E906230D
S3150802FE607B68D3E91623D7E90801F0F73BFB02467C
S3150802FE700B46C7E904237B68D3E914457B68D3E9B3
S3150802FE800801D7E90623F0F7E5FC02460B462046A9
S3150802FE902946F0F729FB02460B467968C1E914237D
S3150802FEA07B6893F8783083F00103DBB2002B14D019
S3150802FEB07B68D3E914457B68D3E90601D7E90423AD
S3150802FEC0F0F7C8FC02460B4620462946F0F70AFB1D
S3150802FED002460B467968C1E914237B68D3E9140103
S3150802FEE07B68D3E91C23F0F745FF0346002B06D0AF
S3150802FEF07B68D3E91C237968C1E9142310E07B687F
S3150802FF00D3E914017B68D3E91A23F0F715FF0346F0
S3150802FF10002B05D07B68D3E91A237968C1E9142333
S3150802FF207B6893F87830002B0BD07B68D3E90623DD
S3150802FF30D7E90601F0F78EFC02460B46C7E90A2303
S3150802FF4005E04FF000024FF00003C7E90A237B6879
S3150802FF50D3E914457B68D3E90A01D7E90423F0F704
S3150802FF6079FC02460B4620462946F0F7BBFA0246BA
S3150802FF700B46D7E90A01F0F7B7FA02460B46C7E974
S3150802FF800A237B68D3E91C23D7E90A01F0F7F2FEB4
S3150802FF900346002B05D07B68D3E91C23C7E90A234D
S3150802FFA00EE07B68D3E91A23D7E90A01F0F7C4FE03
S3150802FFB00346002B04D07B68D3E91A23C7E90A2330
S3150802FFC07968D7E90A23C1E912237968D7E90823A8
S3150802FFD0C1E916237B68D3E90E014FF000024FF000
S3150802FFE00003F0F79FFE0346002B11D04FF00002E4
S3150802FFF04FF00003D7E90601F0F794FE0346002BFB
S3150803000006D079684FF000024FF00003C1E91223C6
S31508030010012300E0002318463037BD46B0BD80B43F
S3150803002083B000AF78607B68D3E90E2343EC172BC4
S31508030030B0EE470AF0EE670A0C37BD465DF8047B57
S31508030040704780B485B000AFF86087ED000BF96898
S31508030050D7E90023C1E90E2300BF1437BD465DF86F
S31508030060047B704780B485B000AFF86087ED000B5A
S31508030070F968D7E90023C1E9102300BF1437BD4641
S315080300805DF8047B704780B483B000AF78607B6803
S31508030090D3E9122343EC172BB0EE470AF0EE670AAF
S315080300A00C37BD465DF8047B7047000080B500AF8A
S315080300B0074B1B78DBB2002B07D1054B01221A70BD
S315080300C004220021034821F051FA024B184680BD49
S315080300D0DAE90020DCE9002080B483B000AF786059
S315080300E00B46FB707B68FA781A7000BF0C37BD465F
S315080300F05DF8047B704780B483B000AF78607B6893
S315080301005B7818460C37BD465DF8047B704780B4A8
S3150803011083B000AF78600B46FB707B68FA785A7039
S3150803012000BF0C37BD465DF8047B704780B483B0C7
S3150803013000AF78600B46FB70054B00221A807B687C
S31508030140FA78DA7000BF0C37BD465DF8047B704752
S31508030150D8E9002080B500AFFFF7A8FF03460021C2
S315080301601846FFF7B9FFFFF7A1FF03460021184614
S31508030170FFF7CDFF00BF80BD80B500AF074B1B78E7
S31508030180DBB2002B07D1054B01221A701822002176
S31508030190034821F0EBF9024B184680BD71ED0020A8
S315080301A074ED002080B483B000AF78607B68DB7C95
S315080301B018460C37BD465DF8047B704780B483B098
S315080301C000AF78600B46FB707B68FA78DA7400BF79
S315080301D00C37BD465DF8047B704780B483B000AF27
S315080301E078607B689B7C18460C37BD465DF8047BB4
S315080301F0704780B483B000AF78600B46FB707B68AA
S31508030200FA789A7400BF0C37BD465DF8047B7047CD
S3150803021080B483B000AF78607B685B6818460C3798
S31508030220BD465DF8047B704780B485B000AF78603F
S315080302307B685B68FB60FB680133FB607B68FA6875
S315080302405A6000BF1437BD465DF8047B704780B417
S3150803025085B000AF78607B685B68FB60FB68013B31
S31508030260FB607B68FA685A6000BF1437BD465DF8C1
S31508030270047B704780B483B000AF786039607B68CD
S315080302803A685A6000BF0C37BD465DF8047B704771
S3150803029080B483B000AF78607B689B6818460C37D8
S315080302A0BD465DF8047B704780B483B000AF7860C1
S315080302B039607B683A689A6000BF0C37BD465DF8BB
S315080302C0047B704780B483B000AF78607B681B7B80
S315080302D018460C37BD465DF8047B704780B483B077
S315080302E000AF78600B46FB707B68FA781A7300BF19
S315080302F00C37BD465DF8047B704780B483B000AF06
S3150803030078607B685B7B18460C37BD465DF8047BD3
S31508030310704780B582B000AF78600B46FB707B6888
S31508030320FA785A730221786800F031FC00BF08375F
S31508030330BD4680BD80B483B000AF78607B68DB7B45
S3150803034018460C37BD465DF8047B704780B483B006
S3150803035000AF78600B46FB707B68FA78DA7300BFE8
S315080303600C37BD465DF8047B704780B483B000AF95
S3150803037078607B689B7B18460C37BD465DF8047B23
S31508030380704780B483B000AF78600B46FB707B6818
S31508030390FA789A7300BF0C37BD465DF8047B70473D
S315080303A080B483B000AF78607B681B7D18460C3732
S315080303B0BD465DF8047B704780B483B000AF7860B0
S315080303C00B46FB707B68FA781A7500BF0C37BD4677
S315080303D05DF8047B704780B582B000AF07F0AEFEC8
S315080303E003460121184608F05FFC0346FB71002308
S315080303F0BB7100237B7107F0A1FE03460221184651
S3150803040008F052FC03461A46FB79934204D2FB7959
S31508030410002B01D00123BB7102237B7126E007F071
S315080304208DFE02467B791946104608F03DFC0346C5
S315080304301A46FB79934216D907F080FE02467B7962
S315080304401946104608F030FC0346002B0BD007F07C
S3150803045075FE02467B791946104608F025FC0346C5
S31508030460FB717B79BB717B7901337B717B79052BB7
S31508030470D5D9BB7918460837BD4680BD90B597B020
S3150803048000AF0346FB71FB79012B02D0FB79022BE4
S3150803049022D107F053FE0346184608F023F803460D
S315080304A0194665480AF00EFA07F048FE0346184649
S315080304B008F035F80346194660480AF003FA604B14
S315080304C01B7819465F480AF0FDF95F4B1B781946F6
S315080304D05E480AF0F7F93EE0FB79072B27D1FFF7C9
S315080304E04BFE03461846FFF7EDFE034619465848E2
S315080304F00AF0E8F9FFF740FE03461846FFF7E2FE5F
S3150803050003461A465349544820F09CFF5349524818
S3150803051018F08BFA514818F055FA04464F4818F064
S315080305205DFA034619462046FDF7CAFD13E04C4813
S315080305300AF0C8F949494B4818F077FA474818F0BA
S3150803054041FA0446454818F049FA0346194620462F
S31508030550FDF7B6FD6CE0FA7907F10C031146184668
S315080305601AF08CFE07F0EAFD0346184607F0BAFFB1
S3150803057003461A4607F10C03114618461AF099FE64
S3150803058007F0DCFD0346184607F0C9FF03461A467B
S3150803059007F10C03114618461AF0A6FE284B1A78DB
S315080305A007F10C03114618461AF0B9FE264B1A78BA
S315080305B007F10C03114618461AF0CCFE07F114028C
S315080305C007F10C03114618461BF05FFB002387F857
S315080305D0573025480AF076F9002387F857300EE096
S315080305E097F8573058333B4413F8433C19461F488A
S315080305F00AF068F997F85730013387F857303B7D87
S3150803060097F857209A42EBD319480AF05BF94FF04B
S31508030610FF31184818F084F819F002FA3A7D07F101
S315080306201403013319461FF03FF8124818F0BAF8B5
S315080306305C37BD4690BD00BF549A0508789A0508ED
S3150803064095EC00209C9A050896EC0020C09A0508AC
S31508030650E49A0508089B0508E8EB0020E4E900206E
S31508030660349B0508549B05087C9B0508909B050845
S31508030670989B0508F8A4002098B500AF07F05EFD1F
S315080306800346184608F0F0F90346042B21D107F070
S3150803069055FD03460521184608F0F3F9D3480AF031
S315080306A011F9D349D34818F0C0F9D14818F08AF993
S315080306B00446CF4818F092F9034619462046FDF733
S315080306C0FFFCFFF759FD034607211846FFF774FE9B
S315080306D060E007F033FD0346184608F0C5F90346FC
S315080306E00C2B11D1C4480AF0EDF8FFF745FD034674
S315080306F007211846FFF760FE07F020FD03460D2184
S31508030700184608F0BEF945E007F018FD03461846F3
S3150803071008F0AAF90346142B07D107F00FFD034681
S315080307201521184608F0ADF934E007F007FD03462E
S31508030730184608F099F90346162B11D1AF480AF063
S31508030740C1F8FFF719FD034607211846FFF734FEDC
S3150803075007F0F4FC03460521184608F092F919E058
S3150803076007F0ECFC0346184608F07EF903460E2B01
S3150803077010D1A3480AF0A6F8FFF7FEFC03460721A3
S315080307801846FFF719FE07F0D9FC03460F2118464A
S3150803079008F077F907F0D2FC0346184608F064F91F
S315080307A00346092B31D107F0C9FC03460021184635
S315080307B008F067F9FFF7E0FC034600211846FFF740
S315080307C0FBFD90480AF07EF807F0B8FC03460021C3
S315080307D0184608F02DF98C480AF074F884498B48B2
S315080307E018F023F9824818F0EDF80446804818F003
S315080307F0F5F8034619462046FDF762FC07F09EFC0A
S3150803080003460121184607F0F6FFFFF7B5FC034632
S315080308101846FFF7C5FD0346022B38D17C480AF074
S3150803082051F80220FFF72AFEFFF7A6FC034600212C
S315080308301846FFF7C1FD6E49764818F0F6F86C4876
S3150803084018F0C0F804466A4818F0C8F8034619466B
S315080308502046FDF735FC704B1B78092B40F0C48006
S315080308606E480AF02FF86C4B05221A7060496C48DB
S3150803087018F0DBF85E4818F0A5F804465C4818F04B
S31508030880ADF8034619462046FDF71AFCACE0FFF718
S3150803089073FC03461846FFF783FD0346012B1DD158
S315080308A060480AF00FF80120FFF7E8FDFFF764FC3C
S315080308B0034600211846FFF77FFD4D495A4818F0AD
S315080308C0B4F84B4818F07EF80446494818F086F8F9
S315080308D0034619462046FDF7F3FB85E0FFF74CFC74
S315080308E003461846FFF75CFD0346052B56D1FFF76B
S315080308F043FC044600F0A8F8034619462046FFF7CA
S31508030900EDFC4A4809F0DEFF494809F0DBFF07F02A
S3150803091015FC03460221184607F048FFFFF72CFC8F
S31508030920034600211846FFF747FD07F007FC034671
S315080309300021184608F07CF8FFF71EFC0346002141
S315080309401846FFF71EFD3B4809F0BCFF28493A48FD
S3150803095018F06BF8264818F035F80446244818F0BA
S315080309603DF8034619462046FDF7AAFB20493348B6
S3150803097018F05BF81E4818F025F804461C4818F0CA
S315080309802DF8034619462046FDF79AFB07F0D6FBD2
S3150803099003460021184607F095FD25E0FFF7ECFB13
S315080309A003461846FFF7FCFC0346072B1CD12448CD
S315080309B009F088FFFFF7E0FB034600211846FFF717
S315080309C0FBFC0720FFF75AFD09491E4818F02DF8C6
S315080309D0074817F0F7FF0446054817F0FFFF0346D5
